:20000000004B00205D4C0100FDC90110FDC90110FDC90110FDC90110FDC90110FDC90110C1
:1C002000FDC90110FDC90110FDC90110FDC90110FDC90110FDC901103BCA0110A4
:20003C00BD0400214D040021810400218504002121050021A10500215106002179060021DA
:20005C00F8B51047F8B50E4600210125AD0430470A48037800F00FF89B070BD0124C2078D9
:20007C00FF2807D0FF2121700E490F24240220436031C882F8BDF8B5014800476B02002147
:20009C00E54C0000094801E00848000C064C05492278FF2A01D1CA7A22706031C8827046E9
:2000BC00801C004700620840C8060021070F0808F0B4084710B501480047000089090000A8
:2000DC0070B503461546012906D0002906D0114A2846FFF7B5FF70BD0F4800E00F480524E5
:2000FC00834203D84008641E002CF9DCE340012040031818820B012907D006490023803111
:20011C002846FFF79FFFE0B270BD0249044B6C31F6E70000835C0000A0BC862300830D2357
:20013C0098060021F8B51A4E0546716B1948CC09E401002D11D01849097802290FD0007B18
:20015C00044372B60120154F4002B847114820380088C109C90704D016E0C07AF0E7407BE5
:20017C00EEE70F497463CC61400AC0070CD001208003316B002D01D0014300E081430846D1
:20019C0031630749403948630020B84762B6F8BD80020021880000219B0200217B3F00008B
:2001BC004040044010B5224A0021516121498968C90009D42149204BCA0598424B6B01D84D
:2001DC00134300E093434B631D49FFF771FF10BD38B51A4D287F002827D11A480088C009E2
:2001FC00C00722D1124C606900281ED1684600F04FF868460078012817D168464078102831
:20021C0013D208206061686A4009400120600E4A0021D1620D4A0221116001210843206094
:20023C00032108436862206038BD0948804738BD00400440180000210000930880020021EC
:20025C00CF680000680000210011044080E200E0C33B00000749002800D00420064A72B649
:20027C000978C90701D0105800E0802062B640B2704700006B0200215860044010B5034CF9
:20029C00FFF718FF20680028FAD110BD0011044003B40148019001BDA56F00000000000035
:2002BC00010003000A001F005900EB003902EA04F9099712EB1FA132784A0A66FA828C9E28
:2002DC0063B617C964D6EDDEC1E3E0E5FF000000A36100007F1407134D00F1242E1F133FEA
:2002FC00B00A3F0007FF0000304000400140034007400F404F40CF40CF41CF43CF47CF4F25
:20031C00CF3FCF2FCF1FCF0F000000000F00080000003F00000040003F00000004006800A8
:20033C000E00DC00060043001A00050000000000020000003F00000000000400C00000004A
:20035C000400C0000000070050C00091007070C00091007082312100319110B1007001812B
:20037C0001B100A18231329110B101911110418141224F40F106007051C0019130181039D5
:20039C00833108D01831416F3100319110B1831414165B680070251050C00091F4C3C0C007
:2003BC002014036F3110410422C082312100319110B163393110410482C0823121003191C2
:2003DC0010B163393110A2C082312100319110B1501015310514059200703F6452C03110EE
:2003FC0031066131C102426412C13110213971065131E102426400708A65996588C0208278
:20041C0050398039001E9F4041C001301814181A89C0308260398039001EA94041C001306B
:20043C001914191A3C64369110B1349110B154B0007154A064B0F0800022AF404012B09002
:20045C0032B053825339533985643F6411C122C1426470C1C26811C1C2C0426470C1C76815
:20047C0050C00091277298921516141642105310F0C12182313131398139313151B070B293
:20049C0072652772999270B262107310F0C331822131213981391B107265E2C08231608289
:2004BC0080318039020061B00071329110B151A061B0277230C2F36800008012B09032B012
:2004DC00007050C000912772999262107310F0C3318221312139813951B070B27E652772CB
:2004FC00989270B242105310F0C1218231313139813931311A107E6551A061B02772B0C08B
:20051C0018693F6401C122C1426401C1C2C04264151A3C64359110B153828564C012B09040
:20053C0032B000703F6472C281C0426422C111C1426402C011C1426462C031C3426462C319
:20055C0011C1426402C311C14264538253398564E2C347641122404142C281C8426452C275
:20057C0011C1426472C2E1CE426402C281C8426402C201C84264B0C0546900703F6442C234
:20059C0001C8426452C211C0426472C2E1C0426402C001C1426462C001C3426422C101C16F
:2005BC00426462C301C1426402C301C1426453828564007061B000711214231C7A4D33911F
:2005DC0010B10070329110B17269007061B000711318321C8649329110B10070339110B1BC
:2005FC007E690070C2C047641510C2C01216476441311514C0C0803105145410A078040478
:20061C000070E6C0863101CC161467106182F0C3010417140070067305720B720E7250B060
:20063C000071818060B050A092804122C3458080F1C11004301601110114016CD661D761A0
:20065C00D861D961DA61DB61DC61DE61E061E261E461366339639180F2C0210421318280DE
:20067C00422A1214321601112114016CEE610B62F4613963EE610B62F4613963E661E661E8
:20069C00E661E661E661E6619464E661F964E6612A65E6615665E6614667E6611012B09011
:2006BC000E720673057210123090A761F0CF3C67D4C103C0C0C354644078509150781092CC
:2006DC00607820927078309280784092907860923078909110824039F006011010311014C6
:2006FC0000924267E661BCA0E2A054A0F08050221546408000222B470D6240A02D828D313D
:20071C008D391082F1C0100409101A824A391A041082803910040E10AB10BC10C2106364AD
:20073C002972E0CF3C6713B003B0C86653B050B054B064B013B0A5661082E0223846AE66FD
:20075C000071418001222B47F08010224B46F022184764B03122384263B0CE661082E02256
:20077C0038467066386264B06F818F318F3DD0DFFF923C670071418001222B4764B0F080B1
:20079C005022654263B01182C1226046CE6605671182D12252467066526261817281813126
:2007BC00813D8231823DC0EFF19202933C670B62B081C091D381978290A2D3187F4EF30B3F
:2007DC001316E31CA44AC391E3813B149062BA1C8B46231E8B4AE31C8B4E90B207228B4221
:2007FC0090A21B1A9662E31CA44AC391E3813B18AB1CA04E9B1CA24ABC1CA442B21010821C
:20081C00D0229D42F0801022A4466364A566A462AB1094629B10946200703082F1C010044E
:20083C0063B00071A86ABC10E0B00070B281C291D281018212185181121841828131813D85
:20085C00121CBF4AE2B032B0B0DFF2923C67F1C72114C34E12C86291729131B0E1B000706B
:20087C0008C006C000C86091709100700182B081C091D0811018518110180614E1804282ED
:20089C008231823D201CE44AE2B02122E84632B00510A0DFF5923C672122E842E2A032B0EC
:2008BC0031824139F0C00104011EF642181610C01030081C04476010103C0610F1C7611437
:2008DC00FA4E16C8669171818131813D161C014B769131B006C008C0007061818131813DC7
:2008FC00408280390118F11C174B0114B080C0221747BCB033B090EFF1920F933C6700704E
:20091C0003A063B064B0EFB056650071408000222B4764B02A65EFA00071408000222B47DB
:20093C0064B003B03862018262818231823D80EFF19202933C6703A05665E661A2806364AA
:20095C00E66150B00071E661E092D08200223D47C0B20070A080F022594330B002C162312C
:20097C0001C0A080001E5243F0225343A0F56031603953632010101A136F236E11161216EE
:20099C00546B00702DC300000DC1000051A20000000000000000000001A90000797C0100BB
:2009BC00451B0100B1770100DD700100C1700100152301000000000000000000DD0D0100ED
:2009DC00893C0100314F01003DD60000037901000E3FA70C18B80BDA500AD33809CD2C0800
:2009FC00CB2407C92006C71C05C61804C51803C41402421001C310004100F6C0080E3FAB55
:200A1C000C2BBC0BE5900AD85809D24008CE3207CB2A06C92405C82004441803C61C02C502
:200A3C001801C41600C312F6C0040500DF3B0100196501004DC90000617C0100417D0100C6
:200A5C00511A010041650100B97C0100C57C0100BF7C0100050000007D7D010000000000B3
:0E0A7C006D160100EC0900000F190A00000FB2
:200A900000FD00000F15B14E0100700A7F0000A00900004800705D8000351E002000314604
:200AB00001B0C708010104EF16027FCD10887BB80BEC003301B5BBAA8A6FFC0D949C06FB0A
:200AD00000C8FFE0070000320FEEFC2038C40D00F2810000631405FD2001F800F2952B014C
:200AF000F3952201F1028EDFF802018F6BFFEEC5FF7401004D330100752D7D91F50208FF91
:200B1000EFF2010AA35510D9DAA4200300FA9803FFE50538BF000074150020FFE183FE01D7
:200B30005019AD00008002035704401F01B33C01B48201BC59030370AA270810FFE084FF52
:200B5000E1D74E9055FFE20701FA2103FF0F008000230798E0EF08003FA7FFE1930300EB25
:200B70008005FFE0040478800188FD6A03F5F40110580000BFFC0400C42264FFEFFC02FFC8
:200B9000FDFFFFE1E9EE000089534F01003D5F3A8F0DFFEF31AD3EB0DF736B0100515D804E
:200BB00015CEFEFFEF003002002087F9013300DB0030FFEF06E9F70A7F50FFEDCB488DDB31
:200BD000B7B200B8FFEF2A0718FE6D30403700A3840600FF2040007F64404000FF0305079E
:200BF000B123053305FF8305480A0306B87AFF02009F84020044C7FF03040102638410008F
:200C1000FF4302B0040200DF7DFF838803008460F135FF88601A418C602382FFA388FB005F
:200C30004309000025630030FF0000FFE5FE0096EC1F35B078C0787178514972C50DED5085
:200C500040BF00011B0000C800B002EF002A0002EE60180C0EEEFFE02600027870440D0E18
:200C7000AEEF901200024A90E00170028F000C000379F07AF17AD1606F8A0100054EC005C7
:200C90006227FF344F441A00200031F71904FFE5768170D02B523307C2014EB17CFA1F0944
:200CB000FFEB0D2005800E0030F5FEFFDF31C553920000C9783E725600841D00200175021E
:200CD0007D3E017D0608808007003008BF22FD30001C60005000A0007F40018002F004E0EE
:200CF0002430F6FFEF0E40117E3D0100B81B130020003101BF02D401B0003128AF229E2C1F
:200D1000970000CC356DB3357F0F087A9FCF14304EEF1D9C1C0020003155A40034AC0034A4
:200D3000B40034BC003435C40034CC0034CD0990077271480C4D02F1FFE1FC05F0003104B4
:200D50002070AA00310C00341400341C0034247C0034FFED1C08C0801D21700D1E21749C12
:200D7000010AF00030987198297B8B325E7F14756E010085C1C7FF001417F3819099819874
:200D90001E268633B80600F3FFEF0CF0003448B0323381C036AF100560006531700031A99F
:200DB0001006B0003118003420003428AA0034300034380034400034482A003450003458C0
:200DD00000346000346FD20D7F3F3F00EC18263B4474FFF0007D000000941E0020880030DD
:200DF000598C007000F1004B00700500927F2001010000D8300174000044FFF000F3010006
:200E1000000700B9FC1C0020EC01A80252901E0133340100052000313C0034FFF0009D0078
:200E300000016CDC02007200C0C0EF1B00200300C48D60011F0049770100FFF000FD0000BA
:200E500004D81A0020CC1CC70020010100003100294C1D0300200031FFF0007B0100000F0A
:200E7000009C1C0020016100FFF000006D290100D77A0100797B0100003D000000D81A002C
:200E900020FFF000000000000200000069170000000F08000000FFF00001000000FFF000BB
:200EB00001000004FFF00001000004FFF0000000900A000008020020E40D00004401002020
:200ED0000C0E0000000100202D0E0000A40100204C0E0000780100206A0E0000C801002073
:200EF000880E0000E4010020980E0000981E0020A00E000000020020A80E0000EC01002038
:100F1000AF0E0000F0010020B60E0000F801002026
:201000003C000000000000000000000034100000000000000000000001000000000000004F
:1C10200000000000000000000000000001000000000000000800000000000000AB
:20103C003400000000000000000000006810000000000000000000000100000000000000E7
:14105C00010000000000000000000000080000000000000077
:2010700030000000000000000000000098100000040000000000000001000000FFFFFFFF87
:10109000FF00000001000000080000000000000048
:2010A0002C0000000000000000000000C4100000040000000000000001000000FFFFFFFF2F
:0C10C000FFFFFFFF080000000000000020
:2010CC0038140000E410000095A1011091A70110A1C2011009B2011041B8011000000000EA
:0810EC00000000002D000000CF
:2010F400280000000000000000000000141100000000000000000000FFFFFFFF0000000093
:081114000800000000000000CB
:20111C00341400003011000065C2011069C101101BC2011091BA011000000000000000006D
:04113C002F00000080
:20114000341400005411000071C20110A5B6011099BF011045B601100000000000000000BD
:04116000300000005B
:201164002400000000000000000000008011000000000000000000000000000008000000AE
:041184000000000067
:20118800240000000000000000000000A41100000000000000000000000000000800000066
:0411A8000000000043
:2011AC00240000000000000000000000C8110000000000000100000000000000080000001D
:0411CC00000000001F
:2011D00000000000101E0020040000000000000000000000200000007010000030000000DD
:2011F0001C110000181E00200400000000000000000000000C0000003013000018000000F1
:2012100040110000201E002004000000000000000000000024000000481300001800000074
:2012300000000000281E002004000000000000000000000010000000A01000002C00000048
:20125000CC100000301E002004000000000000000000000020000000641100002400000077
:20127000FFFFFFFF381E002004000000000000000000000028000000881100002400000003
:20129000FFFFFFFF401E0020040000000000000000000000580000003C10000034000000E8
:2012B000FFFFFFFF481E0020040000000000000000000000100000006013000018000000FD
:2012D000FFFFFFFF501E00200400000000000000000000001C000000AC1100002400000073
:2012F000FFFFFFFF581E002004000000000000000000000038000000F410000028000000E4
:20131000FFFFFFFF601E002004000000000000000000000054000000001000003C0000007F
:1813300018000000000000000000000040130000080000000000000032
:1813480018000000000000000000000058130000080000000000000002
:18136000180000000000000000000000701300000800000000000000D2
:081378000200000000910100D9
:041384000100000064
:0413880000000E0053
:04138C0000000F004E
:041390003200000027
:041394000100000054
:04139800841D002090
:04139C00000200004B
:0413A000E97C0100E3
:0413A400FDC901106E
:0413A8000000000041
:0413AC00000000003D
:0413B0000800000031
:0413B4000000220013
:0413B800A41B002052
:0413BC00010000002C
:0413C0009C1D002050
:0413C400080000001D
:0413C8000000000021
:0413CC00000000001D
:0413D0000000000019
:0413D400080000000D
:0413D8000000000011
:0413DC00000000000D
:0413E0000100000008
:0413E400CC1C0020FD
:0413E80006000000FB
:0413EC0001000000FC
:0413F000441A00207B
:0413F40000000000F5
:0413F80000000000F1
:0413FC0000020000EB
:0414000000000000E8
:021406002900BB
:021408000100E1
:02140A002500BB
:02140C002F00AF
:02140E003000AC
:021410002D00AD
:021412000100D7
:0114140001D6
:0814180003000000BC9001007C
:081420000000000000000000C4
:0414280000000100BF
:04142C0000000300B9
:0414300083C4011060
:041434003C14000064
:041438003C14000060
:04143C0000000000AC
:041440008000000028
:041444008000000024
:0414480000000000A0
:04144C009C1D0020C3
:041450005D790100C1
:041454002000000074
:041458006C90010093
:04145C00B08F01004C
:0414600009C30110AB
:04146400AF4D010087
:041468002F510100FF
:04146C0095C801100E
:0414700097C8011008
:041474000000000074
:041478006B90010074
:04147C00808E01005D
:04148000988E010041
:04148400688E01006D
:0214880008005A
:02148A00090057
:02148C0001005D
:02148E0000005C
:01149000015A
:041494000000000054
:041498000000000050
:04149C00000000004C
:0414A0000000000048
:0414A400817D010045
:0414A8008158010066
:0414AC00096B0100C7
:0414B000015C0100DA
:0414B400CB5C01000C
:0414B800BD60010012
:0414BC0031220100D8
:0414C000E57A0100C8
:0414C40011380100DA
:0414C8000DC801103A
:0414CC001DC8011026
:0414D0000800000010
:0414D40024000000F0
:0414D80018000000F8
:0414DC0028000000E4
:0414E00020000000E8
:0414E4003C000000C8
:0414E8000C000000F4
:0414EC0034000000C8
:2014F000CA482DE9F04F0C4601210170DFF82493DFF82483DFF824A3DFF824B3C4494FF0EC
:20151000000C2027ADF14C0D65461F4081F800C0C7490E9391F838600D9205EA020008BF05
:2015300000287AD10D984FF0E047194662460F4002EA000008BF002843D10E9E0D9B4FF441
:201550008601B9F8B200DFF80CC3CDF8289012EA060701EA030108BF002919D1BC4912EA9B
:20157000060701EA030108BF00296FD0374643460D9E1C8103F130015881002F81E8C0008C
:2015900004BF311CB1F1806F60D102285ED111E0374643460D9E1C8103F130015881002FA4
:2015B00081E8C00004BF311CB1F5803F4ED1B0F5505F4BD1186A674643693868214698472D
:2015D00042E04646C449B6F9087091F90000BC42A0F10100087017D1728906F1300003C8B2
:2015F000002904BFB0F5803FB2F5505F08D0002904BFB0F1806F022A02D011F013FD03E0EF
:2016100012F058FF15F0C2FF524692F90000401E10706FF00101318114E043466FF00100AA
:2016300003F1080108806EB1B4480078832802D08120594608704646316919B160468847E8
:201650002146E8E7CDF82890B9F8B2000D9A0E9E02212F461140374008BF002900F07C83D2
:20167000A84A43F201418142119200F04F83C91C814200F04B8398490A4691F9001047460B
:20169000491E1170B7F908108C4205D043F60401814240F04A8346E3654890F838C007F19B
:2016B000300090E800034FF482062F4617EA090706EA080008BF002810D15748303003C88C
:2016D0004FF400322F4602400F4008BF002A02D111F0A8FC29E312F0EDFE26E30020BCF147
:2016F000010F4FF081045D460F9003D0287808B116F04EF92C70824C002067786081119E52
:20171000E770054635702069DFF8FC91017A457A05F0070201EB022135F07F05A1F10401FE
:201730001FFA81F840F0D982B8F5006F80F2D5820A3041460FF0CCFEE16904F11400052293
:20175000083115F05FFFA8F1030305201FFA83F8E27DA57D6081217E354B0C96C2F301109C
:20177000109093F83800617105EB022518B91099022900F0B2821099022900F3AE8260B13C
:2017900015F0070F00F0A9825C480078862804D105F00700022840F0A082281300F0020AB5
:2017B000BAF1020F58DAA37805F00700022841D14E46D6F804B0002B3CD1E16909A801226C
:2017D0000D3115F01FFF06206081D84780460B96C24F4A48B6683A680078862822D122B9B4
:2017F00016F0D6F848463A6886689DF9240016F0B7FA9DF924705077002090774046D7778A
:20181000B04705F0100010F0EDFD0DE0EA1D0020E01D00200C15002048190020E61D0020BC
:20183000FC3500204046B04715F04CFD59E2C046C8160020314800780026862808BF01268A
:20185000CDF82C905EB1002012F0A6FEE77805E000000C8C181C0020CDF82C90A37887B11E
:201870007BB9012F00F03682022F03D115F0070F40F03082032F04D105F00700032840F0EC
:201890002982280908D315F4405F00F02382C2480778002F00F01E82BAF1020F02DAA80AB2
:2018B00080F01882BE480078C0F3810B8611BBF1010F00F00F82012E00F00C821099B74828
:2018D00002290BD010F80B10805D4018C7B20EB3E8091FD3BF1E0EE0E71D002000EB0B0197
:2018F0008019097900794018C7B2E8090ED25BEA06030FD0BF1CFFB20CE0C04600360020A1
:2019100058350020FE350020001800205BEA060308BF0227C5F30029A7EB09008045C0F24E
:20193000D981A8EB07002909484480B2208124BF25210F910F994018743080B215F0EAFD87
:2019500094F80280E060002800F0C4810021742210F0B7F80020B8F1000F207103D10C9984
:2019700005F0200008700C9803784FF00008002B53D0B9F1000F50D1D548008805F007019A
:2019900003291ED18108424609D3544991F82E30A3B90B681BB15B7E33F07F030ED16AB990
:2019B0008008C24607D3D6498B68887813B1984794F8048010B9BAF1000F02D004202071DE
:2019D0008046D14890F8383013B11098022824DACC490220002301F10A0AB8F1000F8AF8FA
:2019F00000006279CB72AAF1020007D000F1020A9AF8001041F010018AF8001002710A9AC1
:201A10000521A2F87810C2F8840014F0C1FF504603210FF05DFD94F80480E16801F174009A
:201A30004860886523890B812089A1F85C0028090ED3C9F1030082B2A1F85C20886DD54900
:201A500015F0E0FDE1688A6DB1F85C00801888655348D04B0078C0F3011218788D81B9F18E
:201A7000000F00F0780040EA020048EA00050D744FF0FF038B730CBF6079002081F83060EF
:201A900081F83AB081F849006089002FA0EB090085B2658100F01381E0693A46E780291853
:201AB0000831684615F0AEFD3D48EE19B5B26581E16800780A7C6E46C0F38103C0F3011AA6
:201AD000C0F38108002B02F0400949D0C0F301100023022804D1D0090ED201E0A8100020E3
:201AF0009DF801209DF8000000EB0220A1F844000DF10206A1F84200AE4AB1F84400B2F831
:201B10005220824203D04FF6FF72824222D1B8F1030F12D072783078A64B00EB022082B2DE
:201B30004A86B3F85010B61C0120914211D04FF6FF71914218BF00200BE0E0683146323088
:201B500016F0EEF8E0689B493230473115F0C8FB08360346002B00F0B5802046E168C07DF8
:201B7000831125D0BAF1020F03D0087CC00903D309E059EA080206D172783078B61C00EBBE
:201B90000220A1F84200032B0CD07078327802EB00220A850CE0C046A4120020C8900100DD
:201BB0006F350020E0683146283016F0B9F8E16888890009C0F08380886D3A46694615F044
:201BD00021FDE068816D79188165E669B0F85C1001227F18A919A0F85C7008310DF125008B
:201BF00015F010FD6F1CBDB26581E1689DF82500896D0870E2689DF825609DF82530906D27
:201C1000401C9065B2F85C00401CA2F85C0006F0070082F82400C3F3C10182F825102089A0
:201C300092F824708046002F4CD0604F7F183E78361D8642E68045DCE0692918324608318C
:201C500005A815F0DFFC3A789DF817C0111D481980B29DF81450608105EB0C60E3689DF8F2
:201C7000165000EB05409DF81550042900EB052098610BDDE06806A9521E1C3015F0C2FC30
:201C90003878E3686844C07D83F82600986D05A9324615F0B7FCE068816D71188165B0F87F
:201CB0005C10A8EB06077118A0F85C10791E89B22181B0F85C2001818918A0F85C1000F0CC
:201CD00067FC0EE015F068FF11F0ACF909E0C0469418002015F0D2FD03E015F0CFFDCDF889
:201CF0002C90DDF82C80D8F804008047E1690A68002313710968E161D8F80810884714E03B
:201D1000EC1D00203C1C0020C816002040462A4F80784146401C887097F900003946401ED5
:201D3000087011F07FF915F05DF826480A99214F00226FF0010690F83800A1F8B2203E8155
:201D500010B11198007808B915F020FC1B481B4990F90000401E0870174890F9000010B9D8
:201D7000134800210170154890F90000A0B10D9A0E9F02214FF0E0401140384008BF0029A0
:201D90000ED00E4890F90000002809DC15F000FE06E0C0466E3500200020014604F034FE2A
:201DB0000749002013B00870BDE8F08FB0900100DE1D002048190020E71D0020E61D002020
:201DD000EA1D0020C81600202DE9F04F0320ADF1940D14F07BF8BD494FF00008022001F13F
:201DF0001C0242F80C8F401EC2F80880F9D18B4606270BF1400001467F1E21F80C8BFBD1DC
:201E100008210180B34AB449121D22F00303CD1ACBF82050CBF81830AD4FCBF81C30DBF8C4
:201E3000184087600E460BF11C071846A14200F28C83A910E82500EB810121F8048C4FF67D
:201E5000FC741D8004EA020100F1E803761A2546CBF8103005EA0601EC39A0F8E810404669
:201E70001DF000FACBF81400C84E3868D04CCBF81000316804F10C05296070686860C449FA
:201E90000822284614F0F0FD20B9C2480168296040686860C048C149C0F8B410C0F8BC80E2
:201EB000C04EC0F8C060C0F8CC80BD4FC0F8D080BD4CC0F8B870BD4BC0F8C440D0F8B410DB
:201ED000C0F8C83000F1B40609B1404688471DF045FADFF8E0924146382209F118000FF001
:201EF000F0FD02270820ADF830001024ADF83270DBF824100D940CA8884700280CBF0E9F79
:201F1000474608200124ADF83C00DBF82410ADF83E400FA88847A6499DF84000119C0A4685
:201F30000870546087B1D021397087F80180B87087F8038087F804803946C7F8088002207E
:201F5000C7F80C8013F098FBB349182001221DF03FF9284615F00CFD18201DF023FC944937
:201F70000F4648707868494688600EF0BFFDAB4C4D464846394650308860A8682662414615
:201F9000A060F52015F0FAF9A54D05F1180005F10C010EF04BFBA8600D2015F0F7FB002889
:201FB0000CBF082646460E2015F0F0FB08B946F010069C49A86815F0B9FD9B49C82205F1ED
:201FD000240012F057FCCC48102E686011D1206A78B1C2686AB1FF204FF6FC778DF8080020
:201FF000F81CADF80A0002AEADF80C0096E803009047BDA015F06AFCC04F07F1140007F17A
:2020100008010EF013FB7860404615F0A7FD4646BD1E824605F8028F02206870304615F062
:2020300003FE014678685246C9B213F05DFB761C022EEFDBB24907F120004FF4FA7212F0AA
:2020500019FC552040F2EE2115F08CF9E0200E2115F094F9AB4904F12800642212F00AFCBB
:20207000A949E0604FF47A7204F1B80012F002FC4E46E0610121301D15F044F8A34D4D4838
:2020900080884108C0F0E4804A49206A4F78002F40F0D88041460028159131D007697FB338
:2020B00006208DF810000646ADF8126015ABADF8148004AA009392E8030004234246B8478D
:2020D00060B9159819301590206A1BE00018002049F9010001360020004B00203746404677
:2020F0008DF81070236A169004AAADF812605E69ADF8148092E8030016AB0422B047206AEE
:2021100041461591002800F091800769002F00F08D8006208DF818000126ADF81A6018ABF1
:20213000ADF81C8006AA009392E803000E234246B84700287AD115980FF0D0FA12F0E6FA0B
:20215000071C39D0F80000EB071080B214F018FA2490002808BF474630D00646C14606F187
:20217000040A484631460FF0F7FA308871887369524611F003FA0AF1180A183609F10100C3
:202190005FFA80F94F45ECDC18E0C046C8FF0100E8900100F012005008020020F14E010006
:2021B000D5520100C5640100C156010085EA0000B41D00206817002040462490249E022088
:2021D00015F098FAFFB2BDF860009DF86D30E883012B1CBF9DF86C00287702D119A815F0B5
:2021F000C7FBBDF86210532015F0BCF89DF86D000FF0CCFD47B106F10C013046424610F0F6
:20221000E5FC18367F1EF6D1249808B114F0BAFCC3490120087015E0B5890000EC150020F3
:20223000901A0020C95A010095740100BC4880F8008015980FF052FA012015F05BFA012006
:2022500015F01CFAC248012114F08CFDB4488088810807D309F088FCBD48022114F082FD0B
:20227000AF488088C00859D3C44832220C3830F80C1F4FF6FF738B420BD041894B0808D30D
:2022900001F44073B3F5407F03D14FF6FF4319404181521EEBD14FF440704FF4807114F052
:2022B00017F8002836D1B54E32200C3E36F80C2F4FF6FF7191422BD071894B0828D311F4F8
:2022D000407F25D102208DF88400ADF87C201FA80BF088FAF0B970894FF6FF5140F480702E
:2022F00070810840708115E0544920436F6C6C6563746F7200C046C02D760100201B002086
:20231000B5110100B972010081720100DC0A0020401ECBD18E48042114F024FDA988480825
:2023300005D39748012114F01DFD28468188880805D39348022114F015FD2846818895F89F
:2023500023000A0967D3AF68401E5BD0401E57D0401E39D0401E58D187490DF16E000E227E
:202370000EF030F8384650BBC5F8088081498DF87B800DF17A031820E1221CF029FF5020B5
:202390000DF16E0115F0ECFA7A490DF172031820E2221CF01DFF1CA9532015F0E1FAE868D3
:2023B00020B1016811B10DF16E00884795F82200022814BF0320042015F09CF925E00668D6
:2023D00014F0E0FB3046CEE72A7FE88B02E0401C80B2E8833B4606E0997C8A4202D1D9896F
:2023F000884203D01B68002BF6D141468142EED0298C532014F0B6FF40460FF0C7FC04E0A6
:20241000404600E0012010F015FC5D48082114F0A9FC28468188C8080AD34120414614F08D
:2024300095FF062015F066F95548042114F09AFCA08840083BD3A07800090ED310F02AFD6B
:202450004FF6FF71ADF88600814206D002208DF88E000DF1860013F0BBF8A078400920D330
:20247000207850B9012020703AA015F02FFA4120012114F06BFF052009E084F8008039A01E
:2024900015F024FA4120414614F060FF062015F031F93C4815F09CFA012802D1394815F0C8
:2024B00059FC394884F80280012114F05BFC1C48808800287FF4E3AD08200A27ADF8200006
:2024D0004FF0FF36ADF82270DBF82410099608A8884700287FF4D3AD08200727ADF84800BE
:2024F000DBF82410ADF84A7012A88847149E00289DF84E209DF84C0017967FF4C0AD234926
:202510000978914211D12149497881420AD01F4989684B6C4BB141463246984705E0C046D8
:2025300068170020304601F0C9FB179800283FF4A6AD0820ADF8280003270B96DBF824109D
:20255000ADF82A700AA8884799E524F8028B6DE46C1700205065726D69744A6F696E2D4F13
:202570004E2000C05065726D69744A6F696E2D4F464600C0AD470100608C0100800B0020C7
:20259000E00A002080160020F0150020B41D00202DE9F04FB94C0C3CE0686189E269258988
:2025B000806DADF13C0D0E46891808312A4615F029F8A81986B2E068816D6D188565E0698C
:2025D0000122311808310EA815F01CF8E069761CB5B2042265812918083104A815F012F8F4
:2025F0009DF813109DF8100000EB0160E3689DF812102D1D00EB01409DF81110658100EB23
:202610000120049015F0EAF8D863049814F0DCFDA3F84000EA2014F07EFE0221B648E2688A
:202630000170117C2079084310749DF9380015F097FB82F846009DF93800118982F84800D5
:20265000002082F8470002F174009065B2F85C00401A5168091851609089830A18D20309A6
:2026700057D310F0070F07D000F00700032812BF081C5068401C48E05068C17801F00703F4
:20269000491001F0380101EB43014018001D3CE0171C02D115F07CF9E268B889800A2ED350
:2026B00079684878C6112AD13E89796600204D780B7805F07F056D0005EBE3157E2D0DD033
:2026D0007F2D09D003F07F031818801C5B1880B2991C8642EBDC08E0002100E00121801C94
:2026F00087F8601080B2864201DA002005E07968411879603989091A3981A7F86800506E8A
:2027100010B1B2F86800B0B1506850619089000916D292F86000002800F0FC80104611F02D
:20273000FBFBE268D06C002800F0F480B2F85000002840F0EF8015F01DFA0020E06024E23E
:202750004FF0000B1546104605A9CDF814B007ABCDF818B095F82470CDF81CB006AA04F0A2
:202770004CF8002840F0CB80059A6E6968682B89311A581A1FFA80F80AB915F009F9B5F8A3
:202790005C0000900196CDF808800698001D03900598A969AB6D3A4615300AF0ABFB0028B7
:2027B00040F0AD80AD4895F860302E89C15D701A288113B1284611F0AFFBAE8906F007067B
:2027D000032E02D168680078E87395F80F90732009A913F0FDFE83200DF13A0107F084FC80
:2027F000DFF8D082DA4651460AE0C278012A03D1002F08BFDC2027D0001D491C0990C9B247
:202810009DF83A00884279DD09988278032E07D00378B3420DD098F800300BB1022E08D045
:20283000032EE9D10378032BE6D103465B784B45E2D1BB10B3EBA20F05DA02F0030207F0F7
:2028500003039A42D1DD50468146059895F80FC090F814E0514601E0491CC9B28E4549DDB5
:2028700007694B00032E03EB070209D1FB5C032BF2D152786245EFD10BE0C0466435002068
:202890001278B24205D098F80020002AE4D0022EE2D10698077D002F08BFB9F1DC0F2DD0BA
:2028B000A869B0F1FF3F23D0712008A913F090FE5346089AA9690598824206D106989A464F
:2028D00000EB8A00C068884210D85B1C2C32022BF1DB0698491CB1F1FF3F00EB8A00C16052
:2028F00002D1079801218170584608E0DB2007E0DB2004E0DC2002E0FC350020DD206870F8
:20291000E26850709069577850651FB1F22014F002FDE2689F4DDFF8849295F8381000291A
:2029300000F0AD8090899C4EDFF874B200F00700022858D1A078002855D15078002852D1A7
:20295000E1684FF000080CA88DF83980283115F0E7F906F11C01E7680888EB6D401C088078
:20297000786E0DF139020421984704F10C0A30B94846006818B19DF8391080F8681014F09F
:20299000BDFD90B1E76897F8300002280ED1DAF80000594602222031283014F065F828B995
:2029B0000BF116010CA815F0BBF9E7680DF12E0000906D6E786E0CA942460BABA847794818
:2029D0000078862808D1F08BE768401CF083B88900F010000FF006FD15F0CCF84046E0607D
:2029F00014F070FCD3E0704B1A78002702B101277248026827B12F7817B114F07FFD28B989
:202A10001878002831D014F079FD70BB53782779002B40F0BA809DF83800318C02F12803A0
:202A3000002F207002F11C0201F10100308414BF082600265D490020086014F077FD0146FB
:202A5000009658460192263006881A460D20334604F0DEFB20B913F09BFF03E0B49001004A
:202A700014F0CEFB1348E268017841B1D5F880702FB13946104688470E48E26801780A9273
:202A900051B1907BFF287AD01046C17B042976DC40680078072872D0938913F0070040D0D0
:202AB000401E56D0801E6AD1C3F30130022808D102E0C046001700205068007807282ED043
:202AD000FFE7108900285AD0104641684A1C42600F788446C7739CF824607EB9002F4ED0E7
:202AF0000A2F4CDA0189324EF01910F8010C884209D0082F43D1082905D040E0C07B0028C8
:202B10003DD00A283BDA60460189491E0181C17B0B3101700A99C87B401CC8731BE0322085
:202B300018E0244E96F8A1000F280CD014F07EFE48B9181300F00200022804DA0A984D46FE
:202B500008352968884796F8D7000A9A1074152000E0162010700A994D4605F1280013F019
:202B700013F8154E7068804795F83010491C85F83010B1688847202014F04AFF02E00AA840
:202B900012F06EFA4FF0000828E710F04BFA0FB0BDE8F08FC81600206C1C0020A8100020BF
:202BB0006C12002000360020FE350020401C0020DC8C0100D81100200018002064350020DF
:202BD0002DE9FE4FE54980460122A1F130000260DF480768002FFCD0DE4ADF4EC027E04852
:202BF000E04B17603268920808D2324652F8042C03F14104120C42F0F00222704FF0000ACD
:202C10008346C1F800A0DFF864C3DBF80810D64D0191880E43D2480E41D3802018744FF65E
:202C3000D802A3F8512018702868C0F30464162CA8BF203C1F460F3F387800F01F001628B6
:202C5000A8BF2038844223D0624602F1980EDA4ACEF800A0261A022E05DC16F1020FB8BF41
:202C70006FF0010600E002263018166800F01F06844246F4F856A7F866604FF0010616608C
:202C9000E8D11068374617601068CEF80060106828460068C0F30420162808DB06E0A5F19F
:202CB000D0000068C0F30460162800DB203800EB2170401C162805DA10F10A0FB8BF6FF05F
:202CD000090000E01520DE4F00F01F0040F4F850A3F85900386880083ABFEA48C0F800A06F
:202CF00041F04061019E6246A5F13804C80E8F0E80F0010000F00100106087F0010000F02C
:202D1000010090602068C0F38367C0F38F21B00C23D2304640F3072000280BD54242504687
:202D3000490805D17F0806BF0127391C4FF6FF71521EF5D1002810DD4FF6FF72490041F063
:202D500001018A4207D27F0047F001070F2F92BF01210F27111C401EF0D141EA0741182020
:202D700012F028FE2068D24E2768C94CA6F10409C0F3870107F0030041EA0021D9F80400D5
:202D900040F2FF3253468FB22C21466800972746A7F14000B0470C3D2868C0F30D011C2042
:202DB00012F008FEB84955F8080C014000F07C400143142012F0FEFD55F80C1C01F47C0051
:202DD0000904090C0143102012F0F4FD624955F8042C0968C2F30350C2F30345490813D286
:202DF000DBF800100B0510EB237003D41028A8BF0F2000E05046090415EB217503D4102D70
:202E1000A8BF0F2500E0554645EA001502F47F4002F0FF01B8F1220F40EA054041EA00012C
:202E300024BF02F0804211430C2012F0C3FD974DB8F1220F32BF01202868C0F30070B8F17D
:202E5000220F4FEA400040F0200084F8090126BF2868C0F3407001208E4EB8F1200F40F005
:202E7000100084F8090138BF514606D33168C80C00F44070C1F384510143282012F09AFD86
:202E9000B8F1200F26BF3068C0F301505046B8F1220F4FEA400040F0600084F80C0126BFE2
:202EB0002868C0F3C0605046B8F1220F4FEAC00040F0800084F8010126BF2868C0F345504B
:202ED0005046B8F1200F4FEA800040F47C40A4F89C0138BF70490AD3306801038A15920533
:202EF00001F47C1100F00F00114341EA0031082012F060FD4FF48000A5F1D0012060674AAF
:202F1000886D40F21E236FF31F40834216D90868030E13F00F0F03F00F01C0F3034018BF52
:202F3000491E072805D006280EBF0720801C00F00F0041EA0011A2F108000170DDF804C078
:202F5000CCF381477F1E13D07F1E3BD036E0C0469402224300600C40B03F00504010094017
:202F7000AC3F005015620840881300500000204328460068810C21D24FF480412160D2F854
:202F90000210430AC0F3033703F0800321F08F010B4347EA0301C2F80210D2F80130060A64
:202FB00066F30303C2F80130116800F0E70721F0E70147EA010004E02C2009404FF000403D
:202FD000224610603B480068C0F3C0070FB94020A0624FF40070206428684027C0F3C14098
:202FF00040F0300084F8C800CCF3815050B3401E03D0401E1FD002211EE0012013F010F9BE
:2030100006460420314610F039F9042013F008F98642FAD12248066826F07F4012F03EFFE0
:20303000D9F81400036807214FF06022300E98474FF4806020600321042010F01FF908E03F
:20305000000009400420012110F018F9154812F025FF203D2868144947F6180600F03F0069
:2030700084F8CB0F144B0E80D9F800201868D1680220884711480D4D076001212960BDE8F8
:20309000FE8FC04694042A43FCFCFC008C13005040A00C409813005000803F400A600840CD
:2030B000A83F0050BD37860070B00C4094046042A4010010B03F00502C20094000600C4074
:2030D0002DE9F04FADF18C0D1C911E93CC491D920A6806460DF156000260496841603046F6
:2030F000694612F0FDFB00281F9004BF0020229000F0F78102200027B61CDFF84CB32090A2
:20311000D34D2297304602A910F0ADFF5FEA000900F0E48122990EA816220EF0D2FC9DF848
:2031300009707F1E00F082807F1E40F0CF81B9F10A0F40F3D681B61C316804A80160361D42
:20315000318805AF42F20B0039800DF1160111F03FF9BDF81600BDF81410884200F3C18109
:20317000B61C16F8010B16F8017B16F8014B8DF8380016F8011B8DF839700EAA8DF83A40A3
:20319000304605F05BFABF4909780028064400F0A8811F9C012904F1020400F091814FF426
:2031B00000500DF14E0111F013F90DF14E000DF15601082213F058FC40B11C990DF14E0041
:2031D000082213F051FC002840F07A8142F2010004A905F063FE42F20B0005A905F05EFE9C
:2031F00042F205000EA905F059FE0DF1390142F2060005F053FE0DF13A0142F2070005F062
:203210004DFE0DF13B0142F2090005F047FE9DF83B0028B1022840F0538142F2030001E0B3
:2032300042F20D000FA905F039FE49E1B9F1040F40F35781B61C16F8010B16F8017B16F8E3
:20325000014B8DF8380016F8011B8DF839700EAA8DF83A40304605F0F1F90028064400F08F
:2032700040811C9806A905F075FC9DF83600002840F00A819DF83B0000287AD195F8317095
:20329000002F00F0FD8095F83300874207D095F88C000A2801D10AF011FBA86B1EE0AF6BD4
:2032B0004FF400500DF15E0111F092F813F0FAFC4FF0FF08229C2190A24695F83100A0424D
:2032D00040DCA86BB8F1FF0F08D008EB88040019007912F053FDA86B071923D195F83130A8
:2032F0000746002B08BF229C19D05846229C40681946D8467F1F7F1DFA782AB1491E04F174
:203310000104F8D17F1D0AE0804795F83310491C85F83310D8F80810884795F83130A34203
:2033300000F094801C980CF0FFF938710120F870FC788DF8364038798DF83700229B8DF881
:203350002330A1E0387911F0F9FB014608220DF15E0013F089FB40B138880104219814F01C
:20337000EBFC82453CBF8246A046641C7F1DA4B2A3E795F83070002F00F0828095F83200DD
:20339000874207D095F88C000A2801D10AF096FA686B1EE06F6B4FF400500DF1660111F032
:2033B00017F813F07FFC4FF0FF08229C2190A24695F83000A0424DDC686BB8F1FF0F08D0A9
:2033D0004FEA48140019C07F12F0D8FC686B071925D195F830300746002B08BF229C1CD05B
:2033F000DBF80400229C1946D846203F2037BA7F42B1491E04F10104F8D120370DE0C04655
:20341000D8900100804795F83210491C85F83210D8F80810884795F83030A34216D022994F
:20343000384620220EF04DFB1C980CF07DF9F8770123FF2039462022BB770446787206A8C9
:20345000FC720CF0BFFF1FE000180020612055E004140020F87F11F071FB014608220DF1BC
:20347000660013F001FB38B17968219814F064FC82453CBF8246A046641C2037A4B297E7D5
:2034900064203BE0C81600209DF836000EA9162240F004008DF8360008A80CF093FF1F9CDD
:2034B0009DF83B00A41C40B19DF84D700FA8394610F002FA3F1A8DF8357006A80FF022FCA9
:2034D00020984844801C80B2209003E01F9C4E44B61CA41C209884423FF714AE2098022800
:2034F00003DC229A6720114604E01F9A911C121A2298921C1D9B19801E990A8023B0BDE85B
:20351000F08F70472DE9F843C74C0F460646F80B80F0DD81E07AB90F80F06B81B80880F0E1
:203530005881F80A80F03181207A10B1380980F02981206C002840F093803809C0F09380CD
:20355000002501262570B948A67114F0D1FA284613F0E8FBB64904F170002A4614F0E3FB89
:2035700004F1580090E8000314F006F92379B0EB08004FEA103071EB09010905012B40EAEE
:203590000100606606D194F86810B0EBC12F01D8E07860B340F60900A08294F82100267105
:2035B00000F0F00040F0010084F8210094F82000E57000F0F00084F82000A56114F092FC38
:2035D000D14A131D196821F0020119606FF00203136004F1140642F8106C11688908FCD30D
:2035F0001360516841F00201516014F077FC2E4604F1580080E86000666611F045FE6078C2
:20361000012803D0E068403014F064FCC6480660022012F01DFA11200BF08AFAE068007C5F
:2036300010B90E200BF084FAA07A18B1A572052012F00EFABD49A5710878E57128B10D7099
:2036500004F1EC00042114F03DF8B4F95000B4F95210884214BF022007200CF0B9F88EE00E
:20367000380980F08C80B80B77D2780B29D2380CC0F0518104F13C0014F068FBF0B1C168CB
:2036900049680978022919D190F82700400915D2206C90F82700400910D3206C8068408851
:2036B0000028FAD0206C806840880128F5D0206C0026A0641920266414F0BAF927F400474C
:2036D00029E111F0B3F838B1B56930466FF4807100224FF00073A847954904F1700000222B
:2036F00014F021FBB16800254FF0010840F602026572088884F8008082420AD0B0F5C15F14
:2037100007D00A8B4FF61F60104040F43470088306E00A8A4FF61F60104040F434700882C6
:20373000757414F029F8D4F85421E36804F5AA719A4208BFA846266E46B1864226BF301AB8
:20375000401E801B01EB8801000B88602566192014F06EF927F48057DDE004F1400014F0E1
:20377000F5FA061C08D0706830B17568F068B6F9241000222023A84727F40057CBE027F0F7
:203790000807C8E000202072F9E714F0ABFB054604F13C0014F0DAFA061C15D0E06810B1C2
:2037B000783013F06FFBF068E060284614F096FB13F0E2FF20665F4814F09AF94FF40061FD
:2037D00004F1EC0013F07EFF002027F480672072A1E004F14C05284614F0B8FA06F0DEFF06
:2037F000284614F0B3FA27F0020708B147F0020791E020B1042012F02BF90020E07214F07F
:2038100071FBB1688046088840F60202824211D0B0F5C15F0ED00A8B4FF61F60104040F45E
:20383000347008830DE0C046D80D002051BA0000050801000A8A4FF61F60104040F43470B8
:20385000088204F1580090E80C00002B08BF002A18D0042012F0E4FCA0B1A56D13F08CFF02
:20387000854226BF401B401E401B000BF060F168708A401840F6C411F06081422CBFB0F5C4
:20389000FA7FF160404614F029FB10F0CFFF98B1B56930466FF4807100224FF00073A847DE
:2038B00004F13C0014F052FA002808BF47F0020702D0192014F0BCF875692DB10021304632
:2038D0004FF080630A46A84727F0005723E014F009FB014604F1440014F038FA0646B569DE
:2038F000A80813D296B125EA0500B061084614F0F5FA706868B165B12A46F068B6F92410C4
:2039100075680023A84704E010100440084614F0E5FA27F4804727B104F1EC00394613F012
:20393000D1FEBDE8F883C04600000460F735002039C4000051AA00002DE9F04FDFF8E0C20C
:2039500092F808B009AF88460646ADF1240D049338F07F05039206BF604600884FF6FF70F5
:203970000590F08A800934BF002008203076F08AC00834BF102080207076F08A400903D23B
:2039900060460E30007800E00020B076F08A41082CBF20240024000928BF44F0100475686A
:2039B000002108F07F08307D06916D1E02280EDB0C2808DC0C2803D1022044F40854069009
:2039D00044F0030404E00D280CBF02200120044396F8880008B144F00804210900D328B149
:2039F000DFF8C89299F8CC3013B908B1DF2051E121096DD396F88950DFF8B4A206F1240129
:203A100033891AF8052007910AEB0001097908908918491DC9B2C918B1F5006F80F23C8154
:203A300000284CD0049A039906F180000AF06AFD0799002808603FD0806AB0F1FF3F39D00F
:203A500070680023401E8DB196F88A10524600F80119515D491EC9B241B1721892F87F20B8
:203A7000491EC9B2002900F80129F6D1079970660968896AB162090E00F8011996F82A1064
:203A900000F8011996F82910089A00F8011996F8281005F0030500F8011902F0070141EA8F
:203AB000C501017071683289091AC9B270608918318105E0DB2700E0F3277770EDE00023B2
:203AD000F08A7370C00828BF44F0100475686D1E336DA3B9B36D93B999F8E510012903D12E
:203AF0003089B0F5EE7F06DA200904D202290AD144F4005401E044F48054012002E044F452
:203B1000085402200690DFF8ACA19AF8000001280FD013F0F3FC60B19AF8380048B196F86F
:203B30006B00042805D1022024F48054069044F4005444EA8834B8F1020FA4B20AD0B8F15B
:203B5000030F10D1ED1F09F1D801284614F0E8F86D1E08E0B9F8BE00001205F8010999F8A5
:203B7000BE0005F80109069802280CD0B8F1000F15D0BBF1000F0CD004990598814208D1C2
:203B900044F040040BE0BBF1000F08D1B8F1000F05D00599081205F8010905F8011944EA8D
:203BB0008B24BBF1020FA4B209D0BBF1030F0ED10399ED1F284614F0B3F86D1E07E00399EA
:203BD0000888001205F80109087805F80109BBF1000F05D00498011205F8011905F8010948
:203BF0003878F8B934480178307D0D2814D068B9306D28B999F8A800411C89F8A8100AE041
:203C100099F8CD00411C89F8CD1004E099F8B600411C89F8B610014605F8011904E0C04664
:203C30009212002044F48074201205F801092C7070683189401B7560C0B240183081200949
:203C500027D3B06D00B130629AF8380010B1307D0D281ED1726A12F1150002D113F098FE3E
:203C7000726A916A481C9062306A3289B162471B0092D21B019090B20290706A96F8882049
:203C90002B46153008F0AEF900281CBF7070071C07D10020707005E0E5277770F32013F0F3
:203CB0003AFBF8B209B0BDE8F08FC046D8110020B0900100C81600205D350020B0B5044689
:203CD000BC480768ADF1480D002F00F0AC812078401E112800F2A781DFE810F06E0156014C
:203CF0003C0127011F010801F100E300C300B2008D005D0053004200A5012A001C00120060
:203D1000F86B002800F08F81684621460DF0C0F9F96B86E1386C002800F0858168460021E1
:203D300001220DF0CEFE60788DF80000396C78E1F86A002800F07781684600210E220DF0BE
:203D5000C0FEA11C684613F0C1FBA57BA1890022ADF80A1005B101228DF80C20F96A61E111
:203D7000B86B002800F05F816846002102220DF0A8FEA5788DF8015060788DF80000B96B0E
:203D90004FE1786B002800F04E81684621460DF07FF9796B45E1386B08B368460021142222
:203DB0000DF08FFEA5788DF80150A3680193A289ADF80820A17B8DF80A1060788DF80000C7
:203DD000E57B8DF80B50237C8DF80C3094F911208DF80D2061690491396B6846884760687B
:203DF000002800F020810146F22008700020487011F042FC17E1B86A002800F0148168469D
:203E1000002124220DF05DFE6078A11C8DF800000DF1020013F05AFB04F10C0103A813F0B1
:203E300055FB257EE08A04F119018DF818500B22ADF816000DF119000CF0C4FAB96AF0E06D
:203E5000786A002800F0EF806846002102220DF038FEA5788DF8015060788DF80000796A90
:203E7000DFE0386A002800F0DE806846002112220DF027FE658862796078ADF80250237903
:203E90008DF80520E11D8DF80000A5798DF804300B220DF107008DF806500CF093FA396AD5
:203EB000BFE0F869002800F0BE806846002101220DF007FE60788DF80000F969B1E0B86937
:203ED00010B1204610F052F8A07D002800F0AB80A07820B9A069002800F0A58003E0A069DE
:203EF000002800F0A08012F08DFE9CE07869002800F099806846002113220DF0E2FD6D46CC
:203F1000A01C0168406829600B22686004F10A0102A80CF057FA796983E03869002800F051
:203F3000828020460BF054FB7DE0F86800287AD0684600210E220DF0C4FD6078A11C8DF8B9
:203F500000000DF1020013F0C1FAA089ADF80C00F96866E0B868002865D068460021142290
:203F70000DF0AFFDA01C01686D46296040686860A07A0B2204F10B018DF808000DF10900DB
:203F90000CF020FAB9684CE0786800284BD06846002110220DF095FD60786588211D8DF873
:203FB00000000B22ADF8025001A80CF00BFA796837E0C046BC1D00203868A0B3684600216A
:203FD00019220DF07EFDA01C01686D46296040686860A07A410824BF01218DF808108108BF
:203FF00024BF01218DF80910C10824BF01218DF80A10010924BF01218DF80B10C10924BF45
:2040100001218DF80C1030F07F001CBF01208DF80D000B220DF10E0004F10B010CF0D2F99F
:2040300039686846884712B0B0BD70472DE9F04FC54C27688246ADF12C0D17B913F0A8FC61
:204050002768DFF8148308F10300DFF814930678002E3FD0002638897968BC4B0796C500ED
:20407000097818781035890906D340F6485191FBF0F1491901F5AF753B7D68438500352B6F
:204090000CBF371C4FF4FA570DF12601E82010F085FB9DF82600032808BF44F620672068BB
:2040B000007D7D19352807D112F096FB014620686C300FF001FC454302204F468DF82000CA
:2040D00007F10C000068069506A909F05DF9AE480C3806709E4901209E4F087039780129D3
:2040F00002D0002102F090FC20680589466813F011FEDFF868823088000936D398F83870A6
:20411000216897B34A6A4F6E906AC346B0F1FF3F25D027B3431C93628862030E07F8013912
:20413000206890F82A0007F80109206890F8290007F80109206890F8280038702268106A06
:2041500000950190801B281A80B20290916A506A92F888203346153007F044FF00E0DB20CE
:20417000DBF87C10002840F0E280294630460DF0AFF9642009A910F011FB494698F8387083
:20419000087837B9774800780BF06CF8012805D0C9E00BF067F8012840F0C580724CA81CE8
:2041B0002D1D761EA9B2A4F87800C1F3022040F0080006F80109022731709DF82450C4F8FD
:2041D0008460002D4FF00006A4F86A600CBF67486748C4F8C000674DC4F8800068688047E7
:2041F000AB460A90BAF1010F54D0BAF1040F51D0BAF1000F4ED094F84000BAF1050F04F10E
:204210003005C0F3C0002CD0E8200DF1250110F0C5FA98F8380000B39DF8250003281CD1B2
:20423000687B2B7C00F0F00005F1110140F00300687343F018002874F42010F0AFFAD8F87A
:204250009C00804704968DF814706686A064B0468DE88001D9F80C004EE0474B04F168056D
:204270000EE028B9687B00F0F00040F0010004E0687B00F0F00040F003006873404B66863F
:20429000049638468DF8147031468DE80300D9F80C0032E094F83D0000F0F00040F0030033
:2042B00084F83D0094F8400004F130010D46113140F0180084F84000F42010F06FFA98F89D
:2042D0003800002808BF4FF4FA5002D0D8F89C008047A064049620498DF81470D9F80C0028
:2042F0008B78002B06BFA4F84E6004F14C056686324639468DE806001F4B294604AA01F055
:20431000EDFB1E490880DBF80810002809D41D4A92F900001C4F6834401C10700A983C60B3
:204330000DE00A9888471A200DF056F908E0002908BFE420F8D0154A00201070E420884713
:204350000BB0BDE8F08FC046A81000206C1D0020DF1D0020EA1D00206C1C0020C8160020FE
:204370000C1C0020AF1200200C1500204E9055550E7A555500180020999F00003C1C002021
:20439000F5CF0000E61D002054190020003600202DE9F04FC24D4FF0000AADF1140DDFF800
:2043B0001C83E868CDF808A000288DF80CA040D1CC4CBC49843C2068814210D0BA49814259
:2043D0000DD0BA4981420AD0B949814207D0B949814204D0B849814201D013F0D9FA12F0AE
:2043F00021FE21684FF0FF32012805D1C1F30330083806D0C01F01D0012A02D10120E87072
:2044100001E085F803A011F0BBFF4446206A00F1200118B913F0BCFA216A2031096805F1DD
:20443000140088474FF4FA70E884A54FAF620626EE624446E26992F82670E7B9A14892F8E7
:20445000257001788F4216D05046342404FB002C9CF8267037B99CF82530401C9942C0B2C2
:20447000F4D103E09CF82500884204D1604611F057FBD8F81C20DFF850B2D8F824001BC877
:204490008BE81B00E878012814BF50460520DFF83C928F4C8BF8000099F8157127B9906974
:2044B0000068C4F8A40005E0D0690068C4F8A40012F098FE632004A910F070F999F8E72075
:2044D000104611F063FDB4F896C007462CF0070C4CF0010CA4F896C0D4F8980004F1880675
:2044F000812A40F00F00C4F8980001DB842A05DB397B052914BF2421292100E0212184F822
:204510009C10717D812A01F03F01717501DB842A18DBBB7A6BB99DF810203F3262F30501C8
:204530007175F28A4FF6C07303EA020141F0180113E09DF8102001F0C00102F03F020A436D
:20455000114603E021F03F0141F002017175F28A4FF6E071114041F02001F182FA7A397B56
:20457000491D5143D8F81C200A230CF0010C91FBF3F1C9044CEA1141F181F97A192389037D
:2045900091FBF3F161F31C203061308B92F824104FF6F77361F3020003EA0001308392F8D1
:2045B000240000F008000843308399F9D6000EF025FFA4F8A20079683B68D8F81C203889B8
:2045D000401E414303EB51004FF47A71B0FBF1F0A4F8A800106A0078A4F88AA084F8AC00CC
:2045F000C4F88CA0707B00F0F00040F00100707313F0C6FAA0B9F87A364A99F8E740B1FB72
:20461000F0F01070F87A022CB1FBF0F0C0B2B1FBF0F0687004D1304802214170A8270770C1
:20463000EF68D8F820402FB3504610F0D7F9287999F8E710884211D1697999F81521E868CD
:2046500091420CD10221524653468DE80600314602AA01F043FAC8F80C6017E0E868D8F837
:20467000201049688847D8F8207001201B493C68087000E024681A4805F114035946324687
:20469000A047E860D8F82400C8F8280099F8E70099F81571287105B06F71BDE8F08FC04618
:2046B0000C1C002000F0022000F0012000F00020008002200080012000800020481900200B
:2046D00059690100BF120020CC350020D81100200C1500206C1D00206C1C0020EB1D002032
:2046F00010300020181300502DE9F04F09AFADF13C0D08900A92388809911E46ADF818002C
:20471000101C08BF002000F08481002700F101094FF0FF3A4FF0010BB8466CE1252940F0D3
:2047300063811078521C0A922D2818BFADF8068005D15846551CADF8060010780A9530288D
:204750001CBF4246434605D10A9908785A465B46491C0A912A28CDF80080554616D1306872
:2047700004930A99CDF808A0C01C4B1C20F00300001D306050F8044C0A93002C087800940A
:2047900018D5ADF806B06442009413E044460AE0610001EBC40140180A99A0F130040878CE
:2047B0000094491C0A91302801DB3A28F0DBCDF808A004932E282BD10A9908782A2801F137
:2047D00001010A9111D13068CDF80880C01C20F00300001D306050F8045C002D48BF454662
:2047F00008782B46491C0A9111E0454643460AE0690001EBC50140180A99A0F1300508786D
:204810002B46491C0A91302801DB3A28F0DB02930AB1224604926C2804D04C2818BFADF810
:20483000048005D10A990878ADF804B0491C0A910BA9CDF80C800FAB07916428059300F027
:204850008B80692800F08880BDF818C0752872D078286ED06F286AD0702850D063283DD049
:2048700073281ED009980A990128A1F101010A9115D96B490C68B5F1FF3F03D0A84288BF05
:204890006D1C00D8099D029508A80AA932466B46A047C7190A99039801F1010974E0404603
:2048B0002AE030680A99C01C20F00300001D306050F8040CBCF1000F01F10109014608B9EF
:2048D00055A00146079112F0CFFF0390B5F1FF3F5BD0A842C4BF281C039056E03068C01C94
:2048F00020F00300001D306010F8040C5D468DF82C000A990395584601F1010945E008205A
:2049100035680490E81C20F00300001D306050F8041C082210230FA80DF00CFE401E07901A
:20493000402101700A99079801F1010929E0082302E0102300E00A230A99306801F10109CA
:20495000C01C20F00300001D306050F8041CAA42BCBF2A1C049210E00A99306801F10109D9
:20497000C01C20F00300001D306050F8041CAA42BCBF2A1C04926FF009030FA80DF0DAFDEA
:204990000790059D281A0390009C241ABDF8065000945DB906E008A8202109AA11F09FFD43
:2049B000009C7F1C641E0094F5D503980546401E039075B9BDF80600E8B10098401E0090F1
:2049D00019D408A8202109AA11F089FD00987F1CF4E70798411C0791017809AA08A811F030
:2049F0007EFD03987F1CE1E708A809AA11F077FD7F1C09F101094A460A9812F8011C401C02
:204A100000290A907FF48AAE089808B14146017038460FB0BDE8F08F286E756C6C2900C09A
:204A3000249101002DE9F04F002898461546ADF12C0D00F0158111F47C1F40F00E8111F03D
:204A50000F0F00F00D8107460591002006900A904FF0000A0990544608944FF0010BCDF84F
:204A700010B0044650460790059805990BEA000021EA0B014FEA4B0B401E059100F0CD80E8
:204A9000401E7BD0801E68D0001F40F0E08005B12F660720152642F2D002022307F8010BF5
:204AB00001A907F8016BA2F1CF0007F8013B0FF08FFC684603A90BF01DF99C4801783E465E
:204AD000812907DB9848B0F8B600842905DA49F6D05104E09448B0F8B60042F2D0010818CD
:204AF0000099019A4FF47A6390FBF3F040180090824206D8801ABDF80C300090581CADF826
:204B10000C00009B50085146814609041804030C19430004534610EB090041EB0A0102F0CA
:204B300073FCBF1D0090BDF80C309DF80C009DF8002006F8010B181206F8010B9DF801105F
:204B500006F8012B9DF8023006F8011B9DF8032006F8013B0934327078E00220152607F8B5
:204B7000010B042307F8016BB8F1000F07F8013B0CBF099898F80000241D65E01DB1EF65F0
:204B900095F86B0006900520152642F2D002049B07F8010B0DF10E01DDF8189007F8016B72
:204BB000A2F1CC0007F8013B0FF012FC02A810F0F3FA5E4801783E46812907DB5A48B0F82E
:204BD000B600842905DA49F6D05104E05648B0F8B60042F2D001081802994FF47A6390FBD8
:204BF000F3F09DF80E209DF80E3040183F1D0290000206F8019B00EB6300B0FBF2F00290DD
:204C10009DF808009DF8091006F8010B9DF80A3006F8011BE41D337018E00320152607F84D
:204C3000010BB8F1000F07F8016B034607F8013B04BF0A9807F8010B05D098F8000007F8DD
:204C5000010B98F80100641D07F8010BA4B2059800287FF409AF264661E011F00F0F01D038
:204C700000205DE080468A4602264FF4803908F1020509EA0A002AEA090A4FEA4909B0F5B9
:204C900080301AD0B0F5803014D0B0F500300ED0B0F5802009D0B0F5002004D0B0F5801092
:204CB0002AD1072404E0062402E0052400E00424002704E00224012701E001242746A81C0D
:204CD000214600F073FC47B104F00F04C0F30A0141EAC42141F4004105E004F07F0400F06F
:204CF000FF0141EA042105F8011B36180912B61C2970B6B245196D1CBAF1000FB9D1022EA4
:204D1000D8BF00260BDDB01E4FF6FE7708F8010BB819C0F3022040F0A00088F800003046DE
:204D30000BB0BDE8F08FC046A0310020BF120020BA482DE9F84F0025B94CB749056094F822
:204D5000E200002800F06381012800F02F81B54E02283CD0032840F05A8151F8250CD4F8E7
:204D7000B8100029A0F5C060C4F8D400B8BF49420028B8BF4042814226DA4FF08057D7F822
:204D9000A4014568B4F8BC0030214FF47F42082300903046A847D7F8A4014568B4F8C00047
:204DB00004214FF4F802122300903046A847D7F8A401B4F8D070456820214FF440620A23F7
:204DD00030460097A847012584F8D8501AE151F8258C12F099FE2F4600B901273946924FB9
:204DF00038680028FCD0B146012609F10409D9F82CA03E6009B112F08DFECAF30720C4F8C8
:204E1000BC0012F081FEAA4600B9B2463B68002BFCD0D9F800B0BAF1000F3E6001D012F05E
:204E300079FECBF38440C4F8C00012F06DFEAA4600B9B2463B68002BFCD0D9F81C90BAF11D
:204E5000000F3E6001D012F065FEC9F38120C4F8D000B8F5C061C4F8B81000F09C8094F88C
:204E7000D80068B9C4F8D410D4F8C000C4F8C800D4F8BC70C4F8C470D4F8D030C4F8CC300D
:204E9000D4F8D410D4F8BC30002954BF02206FF0010004F1C802176801EB410140184110C7
:204EB00000EB917107EBA1001060D4F8C810C4F8C43000291CDD1E293CDDD4F8CC0030B99B
:204ED0003429B4BF15391E21C4F8C81025E02A29BABFD4F8C8000B381E20C4F8C800D4F89B
:204EF000C4003F28B4BF401C3F20C4F8C4001FE0D4F8CC00032812D011F10B0FC6BFD4F8B8
:204F1000C8000B30301CC4F8C800D4F8C4000028C4BF401E051CC4F8C450032508E011F112
:204F3000150FC6BFD4F8C8001530301CC4F8C800C4F8CC504FF08057D7F8A401B4F8C4300D
:204F500030214FF47F424568364800930823A847D7F8A40104214FF40032112345683148AC
:204F70000096A847B4F8C860D7F8A40104214FF4F802122345682B480096A847D7F8A401A4
:204F900020214FF440620A23B4F8CC60456825480096A84701E084F8D85040F2FF504045AC
:204FB00002D8801C40452DD208202EE051F8251C1E4F4BF2F5204843060A3868C0F38140B9
:204FD00001280AD111F018FB10F040F912F0A8FD3111C010484306EBE03694F8E50030B9CB
:204FF0001348006820F07F408019460801E084F8E5501048310C0660012741600E4D876090
:20501000287808B90B2000E0052084F8E40004F0E1F8BDE8F88FC0462D400C402C500C400F
:20503000F012002000A00C4000800C40B43F0050102009403C600C409E9001002DE9F04F5E
:20505000AC4C04F128000068ADF1240D0FF0E8FE08B111F0CBFFA248DFF89CA2DFF888B27B
:205070000068A24E089011F08FFB11F0DBFDE569A769B5F57A7F13D0C01B4FF47A720023BB
:20509000A5FB000102F0C0F980464FF47A72002312F0DCFA2A46002302F0B6F9C01901E0D6
:2050B000A0EB0708A0618D488C49006820F00200086070688047DBF80010DBF804304546A5
:2050D0006918B1F57A7F0DD34FF47A72B1FBF2F2D2184FF47A73CBF804201F46B1FBF7F206
:2050F0005A43891ACBF80010B168884770688047DAF8041002466818B168CAF80400104623
:205110008847DAF8000000285FD007464FF00009706880474FF000081FFAA5F3079083B988
:205130005FFA95F36BB93979E8B2884204DD79682846884209D20AE03879E9B2401A387136
:2051500008E079682846884201D3414601E07968091A7960B88878B9FB8853B9FB6843B1CE
:205170003B8933B1B87A19460AF022FDF8687860B88808B9FB880BB13B896BB9B9F1000FB4
:2051900004BF3868CAF8000003D03868C9F800003868B846074601E0B9463F68B16807987C
:2051B0008847B8F1000F0ED0B8F8043043B9B8F806302BB998F80A00B8F808100AF0F8FC80
:2051D000404611F00FFD002FA2D144484349006840F002000860E06828B3804723E015F876
:2051F000060C2169A5F10C07032819D0E16A9DF816000978884210D115F8080C10F0F6FE0F
:20521000B979012903D0022908BFA87000E02870002029460EF052F905E011F0E7FE02E048
:2052300009B12846884708200727ADF81000716AADF8127004A88847069D0028CFD0294804
:2052500000680088C8B1706880472649096800220D880A80B1688847089A0020294620706C
:2052700090470546FF202070706880471D4909680A8815430D80B168884711F085FA0746AB
:20529000B7F1FF3F1CD0706807B9194F216AB94238BF0F1C80471C230546626AADF8023090
:2052B0000820ADF80000716A019268468847A16A3846491CA1620FF0ABFFB1682846884736
:2052D00008200A27ADF808004FF0FF35ADF80A70716A039502A88847C5E6C04610E000E0B9
:2052F000109101000C300020F81D0020001800208EC2F528DC1B0020DC3500202DE9F04F29
:20531000A54C064600200F46ADF13C0DDFF89092ADF80C002068A44D017D252900F0108174
:205330006C3005A903F016FC002818BFC0B240F0308120460068C18AC9080DD3007D03284A
:205350000AD09DF81F0038B99DF820004C463870B534207000201CE101A804A90AF0CAFC23
:20537000A5F12F018B4691F82F30019A3468DBF808104FF47A7A504641F208155843891A21
:205390000AFB12000AFB01F1001B091B8D42C8BF002965DC854205DD002803DD346804F5AA
:2053B000915434609DF81F00002857D042F204000DF135010FF00CF811F084FC0446069889
:2053D0000DA9241A42F206000FF002F89DF834109DF81D00FF2904BF0A218DF83410FF2805
:2053F00008BF0A209DF834206C499DF81C30D046B4FBF1F1801880B24843991008FB01F193
:20541000814298BF081C2D1805A811F0F8F99DF81C203468B0FBF2F15143411A8BB251469C
:205430004B4308FB02F1CA1AC91A121B091B8D4201D9002908D56942914216D2002A14D598
:20545000B5FBF8F109B203E06900B1FBF8F189B232684FF4916303FB012405E0002004E0EF
:20547000306841F630342418346005460DF1120102A80AF03FFC0298DBF80810B4FBFAF2BE
:2054900010180290814203D99BF82F30834204D94B4603F15804267836BB9DF81C00551980
:2054B0000004A84298BF2D1A9DF81F00002808BF9DF8200016D09DF81C00B5FBF0F084B29B
:2054D0009DF833000FF03AFB9DF83120014620460FF0CCFA044611F07FF9024608A9204646
:2054F0000FF0A6F84C460DE0814204D8BDF81200401CADF812004C46BDF8120094F85B10B7
:205510000CF0C8FE3870244E84F8B5003068007D05287FF41FAF2348007820B111F0EEFF49
:2055300000283FF417AF387803A9ADF80C0042F20C0003F0B3FCBDF80C00A4F8B00009E74E
:2055500068460DF10E010AF0D5FB3068009A2B7841F208144FF47A7101FB02020092594336
:205570008A1A944210DCA1F5FA619142BCBF00F5FA6030604C4694F85B10208F0CF08AFEDB
:2055900001460020397002E039784C46652084F8B5100FB0BDE8F08FA8100020A08601001E
:2055B000A0310020951200208B320020F0B504460846ADF16C0D401E6BD0401E0DD0801E80
:2055D00000F00381401E00F0E980401E00F0DB80401E00F0A88000203CE142F2010007A94F
:2055F0000EF0F6FE42F20B0008A90EF0F1FE42F206000DF165010EF0EBFE42F207000DF10E
:2056100066010EF0E5FE42F2050019A90EF0E0FE04A80AF085F905460DF1670142F2090049
:205630000EF0D6FE9DF86700002808BF002303D0022010F0C8FD034607A8006808A920602F
:205650000988271D3C46B81C218005F007079DF865609DF864109DF8662000F8011B9DF844
:20567000674000F8016B03F0030600F8012B620747EA926104AC41EA8611012700F8011BB4
:205690009DF8672000942946019707F0D3F90A3099E042F206000DF165010EF099FE42F266
:2056B00007000DF166010EF093FE42F2040019A90EF08EFE04A80AF033F905460DF16701D8
:2056D00042F208000EF084FE9DF86700002808BF002303D0012010F076FD03469DF8640047
:2056F0009DF8657004F8010B9DF8666004F8017B9DF867209DF86770790704F8016B03F0F2
:20571000030705F0070646EA916004AE40EA8710294604F8010B002700962046019707F0B0
:2057300089F9001D4FE042F2150011A90EF050FE13AD42F2160029460EF04AFE15AE42F286
:20575000170031460EF044FE17AF42F2180039460EF03EFE11A801682160406860606A68C3
:2057700004F108035A6028681860306803F10801086074684C60386801F1080528607A68C9
:205790006A60202066E042F214000DF122010EF01FFEBDF8221002200A1258E009A80021F6
:2057B00020220CF08EF942F2130009A90EF010FE09A812F059F8024609A920460AF002FEB1
:2057D00009A812F051F880B244E042F20E0002A90EF0FEFD0DF10A0142F20F000EF0F8FD42
:2057F0000DF10B0142F20A000EF0F2FD03A942F210000EF0EDFD0DF10D0142F211000EF03D
:20581000E7FD0DF10E0142F212000EF0E1FDBDF808009DF80B209DF80C709DF80D609DF840
:205830000E509DF80A1004F8010B02F00102001204F8010B07F0010042EA400206F00100D7
:2058500042EA800205F0070042EA4012042004F8011B22701BB0F0BD2DE9F04F06469E4843
:20587000001D0068ADF1340D80470B900AA9822004F03AFC9DF8280018BB00248DF8284032
:205890004FF6FF75ADF804509DF82800ADF80650FF2108228DF8000002A812F065FA8DF82F
:2058B0001840D420694602F08FF89DF82800401CC0B28DF828003228E4DB82200AA902F0CC
:2058D00083F80020DFF808A2DFF808828DF8280081469DF828008DF8019069468DF80000C0
:2058F000D02004F001FC01274D46E8B99DF80B30012B07D19DF80A0020B90DF1020011F00E
:2059100075FE88B9747B002C0CBF052209224F469C4209D10DF1020006F10E0111F072FACB
:20593000002818BF012507D1002F40F0BF801DB9707F002800F0BA804C469DF828008DF8D1
:20595000214008A98DF82000D12004F0CDFB002832D19DF82200FF282ED08DF80000694698
:20597000D42004F0C1FB002833D102A8311D082211F048FA00B330887788ADF80400ADF82A
:20599000067045B1307B9DF82810B7698DF818000DEB81010F61D420694602F015F875B1A4
:2059B000307F9DF82310884209D08DF8230008A9D12002F009F802E0641C322CBDDB322CCA
:2059D00074D14F468DF80070D420694604F08CFB28B1DAF808100B988847192074E002AB5B
:2059F000184611F003FE4C4600B101242046341D30B918462146082211F004FA00284AD0FF
:205A100030887388327BADF804009DF82810ADF80630002D8DF818200DEB810000F1100061
:205A30000CBF4946B1690822016002A8214611F0E9FD98F8380030B1D8F888201AB19DF8DE
:205A50000010204690474C469DF828008DF8214008A98DF82000D12004F046FBE82807D051
:205A70009DF82200FF2803D0641C322CECDB10E09DF800008DF82490337F8DF822006946FA
:205A90008DF82330D42001F09FFF08A9D12001F09BFF322C02DB7F1C322F93DB322F05D192
:205AB000DAF808100B9888471A200DE09DF82800401CC0B202288DF82800FFF60AAFDAF871
:205AD00008100B98884748460DB0BDE8F08FC04600180020C8160020001800202DE9FE4FE6
:205AF0009B4692468946054612F0FCF902908C48353801680CAFA94208BF416801A84A4641
:205B100053460090284603F089FE834C061C13D194F8880140F0040084F888010298C4F8EB
:205B30007C5112F0DBF99DF8040002280CBF6FF002086FF00108ECE005F1780011F0A2F97D
:205B5000B08CA4F85000B6F92480C6F808909AF80400C6F804B086F82600A6F824806F48BF
:205B7000F56097E80C00202106F110071940104087E80300002786F82770F0684068007817
:205B9000022809D19AF80500012805D196F8270040F0100086F82700029812F09FF994F801
:205BB0008901042807D1D4F88001B4F9841194F8862112F059F812F095F9814694F88901C5
:205BD00030F004033ED104F13C000368D3B931460FF058FF38B3A5F8C08096F8270040F0DD
:205BF000800086F8270085F8C270E07920B1207810B101202072E771484612F06FF94848AB
:205C100000781FE004F13C0031460FF03BFF50B1A5F8C08096F8270040F0800086F8270034
:205C300085F8C27048E0B4F9500000F6FF706FF31F30A4F85000484612F050F96FF0010045
:205C5000BDE8FE8F02280ED196F8270040F0800086F8270085F8C270484612F03FF9B6F9C9
:205C70002400BDE8FE8F012811D104F1C80011F009F996F8270040F0800086F8270085F86C
:205C9000C270206C0028E7D1484612F027F9206C00282AD12078A76400BB6079012838D08F
:205CB00012F020F98146A079A0B9B0680DF08EF858B9607A012803D1484612F00FF928E05D
:205CD000484612F00BF904211FE004F1C80012F0FDF8F1E7134901200870EDE7012011F085
:205CF00003FA192011F0A4FE13E0206CC0684068007802280DD1F06840680078022808D171
:205D10009AF8050028B94FF4004104F1EC0011F0D9FC4046BDE8FE8FD80D0020FDEFFF9F79
:205D3000610F0020F73500202DE9FE4F0646307D01280AD196F916000DF060FB4FF6FF7165
:205D5000814208BFE82000F00281F07B814A20B91146491C0978022908DB012803D1104681
:205D70000078022802DBF120BDE8FE8F346AB6F8289096F8347096F835B0B58B4FF0000821
:205D90005FEA040A17D0744890F83830002B2ED0016D00292BD004F0FF0088476E49096D5F
:205DB00004B20AF47F008847001900B2001D00B2C43084B200E0C4240DB12D1DADB267482F
:205DD0000078012809D147B16548C11991F8048010F80B002418641DA4B205EB0900201855
:205DF0004044801C80B210F02DFE071C02D11A20BDE8FE8F08EB09002B193881002D07EB9C
:205E1000030078600EBF0020E019801C00217422C7F8A00007F10C0011F0A6FF4C442D197F
:205E300007F13C00FF211022A7F84C5011F09CFF07F12C000F21102211F096FF00243C7009
:205E50007C707868716A328D0AF0BCFA07F1800006F12C010B220AF0B5FA07F18C003146AF
:205E700011F04CFA7089A7F89600307B87F89800707B06F10E0587F899002A6869460A6023
:205E9000AB888B80AA798A719DF800102046012908BF01209DF80110012908BF40F00400AE
:205EB0009DF80210012908BF40F008009DF80310012908BF40F010009DF80410012908BF8F
:205ED00040F020009DF80510012908BF40F040009DF80610012908BF40F08000A7F89A00D2
:205EF000707D87F89C00B07D87F89D00B28BA7F8A42022B1D7F8A000B1690AF063FAB07FBF
:205F100087F8A600306AC7F8A800B7F8A400C0B1D7F8A000A8B17868401E7860F82101701F
:205F30007868401E78600470B7F8A410B7F8A4607868401A786039897018801C3881786820
:205F5000B8650848007839460DF0B8FA2046BDE8FE8FC046D6100020C8160020A4120020A6
:205F7000B0900100881800202DE9F047DFF80CA20746AAF13500DFF8F8810068800880F071
:205F9000E78010F039FB814908310B6800261C17641C990D0AD2C0F13E0110F10A0F4FEA42
:205FB000E101D8BF08218C42B8BF0C1CDFF8C4C1990E0FD2590E0DD36246143A1168C1F374
:205FD00004211629A8BF20391268C2F30462162A0EDB0CE0634AD2F87C11C1F30461162987
:205FF000A8BF20391268C2F30442162A00DB203A61189146162905DA11F10A0FB8BF6FF088
:20601000090100E01521584C584D01F01F0242F4F85222802A6812F0030F18BF0126D20855
:2060300028BF46F002060FB146F00406424692F90740041B052C04DA9479B44208BF9188C0
:2060500066D00F28A0F10F0827DB08EB0014A4F1F0084FEA282EBEF1070F88BF4FF0070E96
:206070007546062D88BF06255CF82570042404EB850465462C59E41B04F0FF05F70824BF1E
:20609000C4F307273D44B70824BFC4F307473D44770828BF05EB146501E00025AE465CF845
:2060B0002EC0F7080CF0FF0424BFCCF307273C44B70824BFCCF307473C44770828BF04EB10
:2060D0001C64ADB2A9EB0101A8EB0E277D43002905F1800504EB1524D8BF012103F0FF0339
:2060F00034254D43A9B259434FF6FF73B1FBF4F18B4238BF191C802889B2918005DA10F19B
:20611000800FB8BF6FF07F0000E07F20D0719671194800681F2910604FF0000008D340F2F7
:20613000FF128A4206D24908401C8A42FBD301E01F219180124F0F39090940EAC10047EA4A
:206150000001CAF8FB1F0026CAF8FF6FBDE8F0870C490D4F424608200F60921D1070BDE83C
:20617000F087C0463C1100506E62084024220840EC3500209C130050082009403500094020
:2061900000E7A48030100940FDFDA400AC3F00502DE9F04F0128ADF1140D40F0EE80DFF8D0
:2061B00014B2DBF8DC00012840F0E4800220CBF8DC0011F087FE029001200EF08BFD5FEAD4
:2061D000000806D00120CBF8DC00029811F076FED5E011F06FFE6C490390002008600120EE
:2061F00010F01EF8012818BF002003D100200DF0A5F80120654900900020654F0860386890
:20621000112011F09FFC00280CBF00240124102011F098FC08B144F002040F2011F092FCEF
:2062300008B144F004040B2011F08CFC28B159480068594E016B308888470A2011F082FC80
:20625000002600B101264FF0805A0AF5DC75301C04D02868514E016B3088884750480126C6
:2062700006602868816944F0200088474D48066011F062FC00F001010191400814D24A486D
:2062900011F013FC8146B9F1040FF8D0B9F1010F05D1DAF8D801426843480321904743499B
:2062B000086820F0030008600020FFF75DFE2B683868986B8047019801280DD0B9F1010F1C
:2062D00005D1DAF8D80142683748314690473749086840F0030008602C4806602868416917
:2062F000204688470B2011F02DFC20B128682A4BC16A188888470A2011F024FC20B12868E8
:20631000264BC16A188888472548032206602549CBF8DC2000230B602868416B204688473E
:206330000128F9D1386804200EF0D4FC044616481F490660386808688009FCD30098012829
:2063500002D130460CF0FAFF11F0E4FB08200EF0C1FC07460398CBF8DC6011F0A7FD0DF0A3
:206370003BF9029811F0AAFD57EA040018BF4FF0FF3804E06FF0040801E06FF001084046E7
:2063900005B0BDE8F08FC0460C400940000222432C200940B80100104A8E0100468E010006
:2063B0002820086080010443004003402422084014100940F0120020804A2DE9F04F13681B
:2063D0000546ADF13C0D0DF12A000360526842607B4C94F8B30005F1280105F12807002822
:2063F00000F0E8806878002840F0E48011F086F8DFF8D091DFF8D48100B3042046466A6881
:20641000A873301D12780068042A00F0958095F83000022812D14846007801280ED06A4955
:2064300005F1280002220E46203110F01DFB28B906F1160105A811F073FC05AF686E00288F
:2064500000F0B880012102AA0AF008FD002840F0B1809DF80800A873E86C40B139460DF134
:206470001E0208ABFCF72CFE002840F0A38008A80090686E39460DF11E0306F013FF0028BD
:2064900040F0988048460078012851D04FF400500DF122010DF09CFF0DF122000DF12A01BF
:2064B000082210F0E1FA38B10DF122003946082210F0DAFA00283BD194F85900002837D0F9
:2064D000A66CB4F8445042F2010004A90DF080FF049A4FF000410020E2FB0610061C206D1C
:2064F00011F0FEF986190498B04202D86D1C361AADB24746786880475FFA80F8206CB042D2
:2065100004D1208FA84208BF002608D026642587002084F8350010F0D5FB0126E064B968D5
:20653000404688470EB10BF0E5FC012084F85800002084F859003DE08B468047264C0D90AD
:2065500095F8307022480A264FF00009804610F807A0207AB84206D152462046594610F09F
:2065700051FC012804D0761E04F10C04F1D100E0A1465FEA09070FD198F80601164F461C08
:20659000810088F8066101EBC001F0B27F180A2804BF002088F80601384659460A2211F0B7
:2065B00031F80C48094900788968B8720D9888470420A8730FB0BDE8F08FC046D09001006C
:2065D000A0310020C81600206C12002000180020041400200C1C0020921400202DE9F04357
:2065F000002B08BF002A10D10029BCBF00204FF0004106DB50EA01071CBF6FF000006FF08E
:2066100000410AF072FCBDE8F0835FEA530898EA610803D50026404266EB01015FF00009EF
:2066300013F0004E03D00026524266EB03031C461546002C08BF8D429CBF2C1C0025070CBB
:2066500047EA01470E0CB44208BFBD429EBF240444EA15442D04070A47EA01670E0AB442E6
:2066700008BFBD429EBF240244EA15642D02470847EAC1774E08B44208BFBD4200F292801D
:20669000870847EA81778E08B44208BFBD427BD8C70847EA4177CE08B44208BFBD4265D806
:2066B000070947EA01770E09B44208BFBD424FD8470947EAC1674E09B44208BFBD4239D84A
:2066D000870947EA81678E09B44208BFBD4223D8C70947EA4167CE09B44208BFBD420DD892
:2066F000E60146EA5566EF01B14208BFB84201D3C01BB14159EB09094EEB0E0EA60146EAF1
:206710009566AF01B14208BFB84201D3C01BB14159EB09094EEB0E0E660146EAD5666F017C
:20673000B14208BFB84201D3C01BB14159EB09094EEB0E0E260146EA15762F01B14208BF7D
:20675000B84201D3C01BB14159EB09094EEB0E0EE60046EA5576EF00B14208BFB84201D38B
:20677000C01BB14159EB09094EEB0E0EA60046EA9576AF00B14208BFB84201D3C01BB141AC
:2067900059EB09094EEB0E0E660046EAD5766F00B14208BFB84201D3C01BB14159EB090943
:2067B0004EEB0E0EA14208BFA84201D3401BA14159EB09094EEB0E0EA34208BFAA423EBF8F
:2067D0002D0A45EA0465240A8AD373464A465FEA080803D50026404266EB01015FEA480841
:2067F00003D50026524266EB03031E4617460B46024631463846BDE8F0832DE9F0430446A6
:2068100094F830900F46984615468B20ADF1340D0DF10A0103F068FC8A20694603F064FCF8
:2068300094F8250000283ED1B9F1000F19D1BDF80A104FF6FE70884205DCBDF80A108842F7
:206850002FD1694615E0B4F844009DF80A608DF80C0000128DF80D00BDF80A008DF80E60AE
:206870001BE0B9F1020F09D0B9F1030F19D104F1280103A811F054FA092612E0207CC00935
:2068900034BFB4F84200B4F844008DF80C0000128DF80D00208D8DF80E00001205268DF8E0
:2068B0000F00002013E002280CBF05260926012818BF04F11C0104D1892006A903F014FC15
:2068D00006A9324603A810F09DFE94F8260006EB0D01C8723A4603A831460BF0CFFA0028C2
:2068F00040F08E80B9F1000F19D1BDF80A104FF6FE70884205DCBDF80A1088422FD1694632
:2069100015E0B4F844009DF80A608DF8200000128DF82100BDF80A008DF822601BE0B9F1BB
:20693000020F09D0B9F1030F19D104F1280108A811F0F6F9082012E0207CC00934BFB4F8DB
:206950004200B4F844008DF8200000128DF82100208D8DF8220000128DF8230004203E68C0
:2069700081460BA9822003F0BFFB9DF82C10307B8142D8BF9DF82C00002841D007460024FC
:20699000722029460FF024FEB0689DF82C102018C8F80000007881422EDD2B68C10001EB5E
:2069B0000011D8F80000C91829604278012A1FD0807828BBB9F1040F06D0091D08A810F064
:2069D0008FFC012816D017E008884B888DF82800042208A98DF82A3000128DF82900181266
:2069F0008DF82B000AA810F00DFA012802D003E0807828B9002004E07F1E04F10304BFD13A
:206A1000F3200DB0BDE8F0832DE9F04F7C4C074660688946ADF11C0D8047A046714E724D8B
:206A30006F4C8346012F68D010F0BCFD00285FD06348007800285BD162480078002857D161
:206A500061480078002853D16048007800284FD15F48007800284BD15E480078002847D190
:206A70005D480078002843D15C48007800283FD100200BF061FB00283AD12746387800286A
:206A900036D1286A436CF068022104AA98479DF8100068B32C46B9F1010FBA4635461ED041
:206AB000524F226AE86897F9001011F1020F05D0926B97F900109047E868226A4C4E96F948
:206AD000001011F1020F05D0926B96F900109047E868226A6FF001013170397001E0E86883
:206AF000226A01218AF80010D169884700206070D8F80810584688475EE001200BF01CFB87
:206B1000D8F80810584688473A4800780F2842D12078012842D1384F97F8C2000028FBD12C
:206B3000286A436CF068022105AA98479DF8140068B197F8C20050B9207801282ED10020FF
:206B5000B9F1010F207029D010F038FD26E0D8F80400804702222270002302938DF80C20ED
:206B7000284F7B8181468DE80C00274BF0680837394602AAFEF7B2FF002C01D510F008FF67
:206B9000224991F90000401C0870D8F80810EF604846884702E0484607F04AFA2078174DE1
:206BB000022803D1287808B110F0F2FE2878012802D020780228FCD007B0BDE8F08FC04674
:206BD000FC350020FE35002000360020FD350020FF350020DE1D0020DF1D0020E01D0020B1
:206BF000EB1D00200C1C002048190020DC1D0020DD1D00207912002010300020EA1D00202F
:206C1000001800200C150020D53E0100E61D00202DE9FE437B4E80460F46B8F1450F06D1A5
:206C30003046342210F0EEFCC6F89C60E7E010F086F93B2808BFF42000F0E280724C04EB51
:206C50008004A07810B9E178002938D0E178814208BFFB2000F0D480B8F1580F25D0B8F145
:206C7000600F1BD0B8F1E00F0FD0B8F1E80F05D03A78904220DC91421EDB20E006F1E70094
:206C90003978007881421AD1B9E097F900000CF0B5FB4FF6FF7181420ED010E038880A2800
:206CB0000ADBB0F5804F07DA09E038888F2803DB46F2B041814202DAE820BDE8FE83544DB5
:206CD0006868804781462078627839468019943010F098FCA968484688474046503800F0F8
:206CF0008C80801E73D0401E00F084808D387CD0401E63D0401E75D0801F1BD00D387ED1E2
:206D10000E2096F815718DF8000017B11B208DF8000096F9D6109DF90000884203D0E0206C
:206D30006946FFF775FF10F05DFA96F81501002841D164E0032096F8E7108DF801008129D9
:206D50004FF005008DF8020006DB842904DA8DF8010008208DF802009DF8010096F8B910CA
:206D7000884204D04F200DF10101FFF751FF9DF8020096F8C510884204D057200DF10201A0
:206D9000FFF746FF214C94F83800A0B110F0B6FB88B1E26E7AB1022000278DF803000DF1F2
:206DB00003018DF8047042F21B009047E26E42F21C0001A990470CF0ABFD20E096F8D70076
:206DD0000DF042FA01281AD01A20BDE8FE8396F8BD0018B902200EF00BFB10E0022010F0A3
:206DF0000FFE0CE010F0AEFB09E096F9D60010F009FD04E010F0B2FB01E010F0F9FC002006
:206E1000BDE8FE83D811002004880100C81600200018002030B50546EC6B00214422ADF1C4
:206E3000440D68460AF04DFE14F8010B8DF8000021680DF10100016061680834416020783A
:206E5000617810F01DFFA41CADF80A0041080FD32078617810F014FFA41CADF80C00207806
:206E7000617810F00DFFADF80E00BDF80A00A41C810808D32078617810F002FFADF8100060
:206E9000BDF80A00A41CC1080FD32078617810F0F7FEA41CADF812002078617810F0F0FE7C
:206EB000ADF81400BDF80A00A41C01097FD32078617810F0E5FEA41CADF8160020786178EE
:206ED00010F0DEFEA31CADF818001878597810F0D7FE9A1CADF81A001078517810F0D0FE80
:206EF000931CADF81C001878597810F0C9FE9A1CADF81E001078517810F0C2FE931CADF80C
:206F100020001878597810F0BBFE9A1CADF822001078517810F0B4FE941CADF82400207896
:206F3000617810F0ADFEA41CADF826006178207810F0A6FEA31CADF828001878597810F030
:206F50009FFE9A1CADF82A001078517810F098FE931CADF82C001878597810F091FE9A1CF2
:206F7000ADF82E001078517810F08AFE931CADF830001878597810F083FE9A1CADF8320062
:206F90001078517810F07CFE931CADF834001878597810F075FE9A1CADF8360010785178D8
:206FB00010F06EFEADF83800BDF80A00941C40090ED320786178A278E37810F07DFD241D3E
:206FD0000F906178A2782078E37810F075FD10900E490F4C086B401C0863207800280CBF93
:206FF0000121002101200BF0B5FB298804A010220DF068FB28460CF091FA11B030BDC046E2
:2070100053656E736F7220307800C04668170020221B00202DE9F047064637680C465FEA49
:207030000208ADF1180D14BF00214FF0FF3107F14800814610F036FF002808BF0B2000F0CA
:20705000DF80002565707148FC60B8F1010F057004D065700220FC600EF038FF2078012867
:2070700040F29080801E012857D9801E01282CD9801E012800F2B88010F034FF8246A078F7
:20709000009021782846062908BF0120019001200290A068228A6368E16807F001F90746E8
:2070B000504610F01BFF002F40F0A080B8F1000F02D010F017FA02E030460FF0B3FB0028C9
:2070D00000F0878010F040FE21E010F00BFF012782460097A168A278606824782B46042CB1
:2070F00008BF3B1C08F06EFC0746504610F0F6FE002F7BD1B8F1000F02D010F0F3F902E056
:2071100030460FF08FFB002863D00EF07FFE3E49C1F8B0510D60074668E010F0E3FE82469E
:20713000E08A0090E0680190208B0290A0780390207D04900121059122782846022A08BFA0
:20715000081CA368E178626802F0E8FC0746504610F0C4FE002F49D1B8F1000F02D010F07F
:20717000C1F902E030460FF05DFB002831D00EF07DFE071C3AD1E078A168E28A23690AF073
:2071900029FBC8E710F0AEFE8246E08A0090E0680190208B0290A0780390207D049001208B
:2071B0000590277807B90546E1786268A368284602F072FD0746504610F090FEB7B9B8F1F9
:2071D000000F02D010F08EF902E030460FF02AFB08B9142014E00EF031FE071C06D1E07853
:2071F00021690CF0B9FF96E74FF0FF37B8F1010F02D002200EF02CFC484610F06BFE384607
:2072100006B0BDE8F087C04650450240FA3500202DE9FE4F0CAF89469A4604467D680292D0
:20723000294604F0B3F9061C00F0D9803888F082DFF8CC81347598F8380018B1012C04BF44
:207250001520307506F1800029460B2210F0DAF9012C04D00D2C1CBF7068401C00D170686C
:207270003062002598F8380035650028B5654CD0052C18BF012C43D14FF0040B86F86BB057
:20729000F08A86F86950C00932BF57485D4816300078029986F86A000A6806F16C073A6078
:2072B0004B687B600889388110F028F940BB06F16C0010F035FD4D4F07EB8407386810F478
:2072D0007F0F0CD086F82CB0386806F12C01012200F47F003063304602F0DEF9386810F00E
:2072F000FF0F4FF003090BD02A2086F83C00386806F13C0100F0FF003064304607F0CEF9BB
:2073100098F8380008B10D2C13D00095029A534630464946FCF710FB071C61D1E41F012C6E
:2073300003D8707E40F020007076304607F0E0FA56E010F0E3F8294600B101212B483430CD
:2073500009B94FF00309052186F86B10016811F0F70F12D02A2186F83C1098F80020006872
:2073700006F13C01012A00F0FF0030641CBF20F008003064304607F091F90095029A5346D3
:2073900030464946FCF7D8FA071C29D1184806603489756801A964200DF000FA154E6D1E83
:2073B000231DA01C99B2A6F87800C1F3022040F0080005F801090A1F297091B2AA1CC6F8C2
:2073D000845010460AF084F89DF8040000280CBF09480A48C6F8C000C6F8800000E01A27F1
:2073F000F8B2BDE8FE8FC04691120020108D0100401C00200C1500204E9055550E7A5555C3
:20741000C8160020A41200202DE9F0411C4615468C4208BF854282BF00230022E5E0002CB1
:2074300008BF002D0AD100290EBF00286FF000006FF0000100F0E1F8BDE8F0815FF000085A
:207450005FF0000E002C08BF8D429CBF2C1C0025070C47EA01470E0CB44208BFBD429EBF76
:207470005FEA044444EA15445FEA0545070A47EA01670E0AB44208BFBD429EBF5FEA042405
:2074900044EA15645FEA0525470847EAC1774E08B44208BFBD4200F29380870847EA81773B
:2074B0008E08B44208BFBD427CD8C70847EA4177CE08B44208BFBD4266D8070947EA0177D5
:2074D0000E09B44208BFBD4250D8470947EAC1674E09B44208BFBD423AD8870947EA81672A
:2074F0008E09B44208BFBD4224D8C70947EA4167CE09B44208BFBD420DD8E60146EA55663A
:20751000EF01B14208BFB84201D3C01BB14158EB08085EEB0E0EA60146EA95664FEA8517B7
:20753000B14208BFB84201D3C01BB14158EB08084EEB0E0E660146EAD5666F01B14208BF42
:20755000B84201D3C01BB14158EB08084EEB0E0E260146EA15762F01B14208BFB84201D33E
:20757000C01BB14158EB08085EEB0E0EE60046EA5576EF00B14208BFB84201D3C01BB14151
:2075900058EB08084EEB0E0EA60046EA9576AF00B14208BFB84201D3C01BB14158EB0808FB
:2075B0004EEB0E0E660046EAD5766F00B14208BFB84201D3C01BB14158EB08085EEB0E0E09
:2075D000A14208BFA84201D3401BA14158EB08085EEB0E0EA34208BFAA423EBF2D0A45EA43
:2075F0000465240A89D3734642461E4617460B46024631463846BDE8F08170472DE9F04FD6
:20761000DFF8CCB19BF8A100ADF1240D05909BF8C00006909BF897000790002008909BF879
:20763000CC0001280BD16E4991F85C703FB1694891F85D10C219445C1579641D01E0089DB6
:207650002C4665480678082EA8BF07269BF8A010F000C0B2401824189D34A4B22819801C76
:2076700080B20FF0EFF9DFF87491D9F80480071C08BF089C00F0A68008998C2210F074FB4E
:20769000E4197C609BF8A0203D81DBF89C107868841A801A0FF0B6FF3C62C047641EDFF8A7
:2076B00044A1DDF82080DAF82450049016E0687EC00911D369684878C0F3810003280BD131
:2076D000E41F491D204610F02BFB761EF6B2641E08F110005FFA80F855F80C5C002E18BF53
:2076F000002DE4D1D9F8081004988847D9F804008047DAF824500DB36968491C0A78C2F335
:207710008102022A16D16A7ED20906D2297E890910D3012108916EB910E0497904F8011962
:2077300069684979761E08F10103F6B25FFA83F804F8011955F80C5C002DDDD1D9F808100A
:20775000884704F8018900202749079E059D04F80109069B9BF89520097841EA420146EADF
:207770008101090141F00F0104F8011945EA0311217079683A89091BC9B2891839817C60C8
:2077900004463C65F882164EBC650B22387506F154018DF80C0007F180000FF033FF0898EF
:2077B00018B1F88A40F00800F8820FF0BFFE01AA2346014600943846FCF7BEF818B13846A3
:2077D00010F0BBF82746384609B0BDE8F08FC046D8110020B0900100D61000200018002090
:2077F00048340020A8100020C8160020F0B542F20400ADF11C0D0DF115010CF0E9FD42F239
:20781000050005A90CF0E4FD664C67489DF81510A0666420414321666449C4F884109DF886
:2078300014104843E0676248C4F8A0006148007880B942F2020069460CF0CAFD68460FF08D
:20785000B1F904F15C000CF0EDF904F134000CF05BFC27E042F2030069460CF0B9FD0EF022
:20787000BBFF0546684629460CF026F82D1A04F1780084F85B500CF0D5F904F134000CF0F2
:207890007BF9012742F20200694684F854700CF09FFD68460FF086F904F15C000CF0C2F94B
:2078B00084F85870E8200DF116010CF077FF9DF81600032804BF012084F8B40094F8B800B7
:2078D00000286DD13C4D0021302205F10C000AF0F8F82046002133220AF0F3F83748286280
:2078F000374FAF6105F114000CF09CF942F21B000DF117010CF06CFD9DF817000DF11701BB
:2079100085F8300042F21C000CF062FD9DF817109DF8170085F8311095F83010012641B1F3
:2079300048010EF01DFF686308B910F003FA95F8310040B100EB800080B20EF011FFA863E6
:2079500008B910F0F7F91F4905F13C000A270A684B6802607F1E436000F10800F7D10021F2
:2079700095F8307085F88C1047B1686BFF220346C2777F1E997703F12000F8D195F831708B
:2079900047B1A86BFF22034602717F1ED97003F10500F8D1281D06220AF093F884F8B860C1
:2079B00007B0F0BDA03100204943010065FC0000CB7C0100C81600200414002029B9000014
:2079D000002A7515E09001002DE9F041714B724ADFF8BC810C46D128014610DCD12879D0DF
:2079F000713800F0B280401E00F0AA80401E00F0A380113810D04C3800F0878007E0D2382E
:207A100053D0401E40D0401E33D0401E28D008460FF08AFF0B2802D1F420BDE8F0815B4D60
:207A300005EB8005A97809B9E87850B1E878884208BFFB2000F0A880227891426ADC9042D4
:207A500068DB564E7068804729786A7807464046401821460FF0D6FDB1683846884792E0D1
:207A70002178022956DA1846641C042200EB810086E0207832284DDA1746C100241D18227A
:207A900001EB001178187BE026783046022841DA2C2505FB0680611C102239300FF0B2FDF8
:207AB000616905FB0680C1646DE022786178022A30DA02292EDA40462C2301EB42064F1CA4
:207AD00003FB0205022285F8387000EB460000F5DE7018E022786178022A1BDA322919DAFA
:207AF0002C23404603FB020595F830309942A4BF4B1C85F83030322303FB021101EB410199
:207B1000032240189030A41C3AE020786778022800DA17B1E820BDE8F08141462C22C5192A
:207B30007E1C02FB00136A0083F8286002EBC50288180A227C30E6E72CB3184608221FE0BF
:207B50000CB310464FF496621AE0B4B9404600F17C04A0F1080200F1900300F5DE710220E2
:207B700042F82C4F9360401E116104F10A0403F1960301F10401F3D105E0404658222430F9
:207B900021460FF03FFD0020BDE8F081FC7E010050250020C42B002014270020001800204B
:207BB0002DE9BC4305466D4800880021820804D2B5F89A20D20828BFE82110F0600F04D122
:207BD000B5F89A00800828BFE8212889B0F5006FA8BFE82195F8980030B995F8940000284A
:207BF00008BFF52100F0B480002940F0B180DFF87091D5F8A800DFF8708199F8381010B933
:207C1000012903D02BE0002900F0A1800FF076FC68B9D5F8A8104046BD3041F002010078DC
:207C3000C5F8A81018B141F00801C5F8A810D5F8A81011F0FF0F05D02A2085F83C0001F0EA
:207C5000FF072F6411F47F0F07D00420D5F8A87085F82C0007F47F00286399F83810002061
:207C700061B3404995F894700968042267B925232B75C98AC90934BF98F8B91098F8E21034
:207C900085F86A10891C08E015232B75C98AC90934BF98F8B91098F8E21085F86A1085F811
:207CB0006B2005F18C0785F869003B6805F16C010B607C684C603B890B8101E001212975C8
:207CD00095F89C70EF760446AC65B5F89A102C6595F89D30E9826A682B7795F82C702A6265
:207CF0000F2F09D00246B5F8A40005F12C0100B90122284601F0D0FC28BB95F83C10FF29B6
:207D100001D1AF6D27B105F13C01284606F0C6FCC8B9009495F89810B5F8963005F18C02F3
:207D30002846FBF709FE071C0CD12889B0F5006F03DA284606F0DCFD04E0E52068702846BE
:207D500009F0ACFF3846011C02D1BDE8BC831821284608F05FFFBDE8BC83C046941800206A
:207D7000C8160020A8100020D81100202DE9F843644C0746207808B10FF00AFEA046012067
:207D9000614988F800000978012902D00021FEF73BFE614E5E4D5F495C4C012F06F13800D4
:207DB0002A68D1F800900078A77034D9BF1E51D07F1E13D07F1E02D0781E46D042E092F8E7
:207DD0006900607192F86A0020710020A07103F00DFA2A68002A63D1BDE8F88300285FD042
:207DF000D6F8981021B1032088472A6896F83800002855D0776D002F52D0D06D20B102212E
:207E10000023B8472A68776D106E002848D008210023B84743E000206071D18A3F48C909E9
:207E300034BF90F8B91090F8E2102171A77837B990F897701FB10229C4BF0220207103F020
:207E5000D5F92CE00FF0A4FD29E0002060710FF093FF24E0324F38788600D9F83C0080477E
:207E700079683C22401AB0FBF6F0B0FBF2F151436278401A9101A1EB8201091AD9F83C00A1
:207E90003C318FB28047274906FB0700086791F8740000F0F00040F0020081F874002A68E8
:207EB0002148007878B912B90FF072FD2A685168087800F02000E0708878E07108788009E2
:207ED00001D20FF063FEA078042819D0174D68688047A17802290CD015490F7817B9154904
:207EF0000F7837B1022188F80010A9688847BDE8F883832188F80010A96888470EF0D2FF6D
:207F1000BDE8F88300360020EA1D00206C1C0020A810002068190020C8160020D81100208C
:207F30006C1D00200C150020F835002000180020FC350020FE3500202DE9F04389461446AC
:207F50000546ADF12C0D69460DF0CAFC5FEA000800F0C480AD1C0226284602A90CF083F877
:207F7000071C00F0BB809DF80900814509D0F6197D1908F10200B61CAD1CB6B2B042EBDC0A
:207F9000ACE0401E05F1020500F08B80401E52D0801E38D0401E2BD0401E24D0401E18BFE9
:207FB000622040F0AB80202F40F0988028686F6805F10801206004F10806676001F108058E
:207FD0000A684B68326004F1100773602A6868683A6005F108067860306804F11801086015
:207FF00073684B6089E0022F78D12888208084E0202F73DC20460021202209F062FD3A4615
:208010002046294677E0042F68D12888AD1C208015F8010BA070287800F00100E0702878F5
:20803000C0F3400020712878C0F38000607128784011A07161E00A2F50DD0DF1120000212E
:20805000162209F03EFD28682D1D20602988271D42F20B00398004A90CF0BAF9BDF810003C
:20807000A18888423ADCA81C10F8011BA17110F8011BE17110F8011B217210F8011B012378
:20809000C1F3C202A2720DF1120200F0D7FA28B39DF82700A0819DF81670E78104F1100031
:2080B00026E0042F1ADD0DF112000021162209F008FD15F8010B207015F8010B607015F87A
:2080D000010BA07015F8011B0DF112020023C1F3C2002071284600F0B1FA08B967200DE0D1
:2080F0009DF82700E0809DF81670278104F10A000DF11601112208F065F900200BB0BDE874
:20811000F083FEE72DE9F04F6D4C2068ADF12C0D002840F0C78004F124063068002800F01C
:20813000C18062480078022800F0BC80614D281D006880470A90606AB046074678B35C4ED8
:208150004FF0000A4FF01D093B7D0820711E11F8012F9A421ED0401EF9D14046394652462A
:208170000DF0DCF9787E30F07F0005D194F82F00401E84F82F0004E094F82E00401E84F876
:208190002E0087F8019057F80CBC384609F086FD5F4602E0BA4657F80C7C002FD4D13520F9
:2081B00008F0F8F9444EA968002849D1452008F0F1F9A96800283DD1D8F8000038B1017D1C
:2081D000252904D050F80C0C0028F8D110E078B196F8580050B3684601A907F08BFD3748C4
:2081F00000990078001F884213D8012086F85500152008F0CFF9A96848B10A98884720689E
:208210000DF106016C3000F0A5FC58B10FE00A9847E0252008F0BEF9A9680A9888470020C5
:2082300086F855000420FFF7A1FD3BE0192000F003FF37E00A98884708200CF08BFA31E01B
:208250000A98884796F8B400B8B10EF00BFD317800290EBF0921491EC9B201EB810171184A
:20827000D1F802100FF068FD42F21071814292BF00206431081AC0B200E0002069680028A4
:2082900008BF0620D9D0C6F8980088470446D6F8A010D6F8980006F1A8020DF071FBA968CA
:2082B000204688470BB0BDE8F08FC046FB190020F090010000180020A03100208B320020D9
:2082D000A81000202DE9F843664C002605466676687D0628A4BFE8216176A97D0E2903DDD3
:2082F00003281CBFE8216176032805D15E48008840083CBFE820607695F8280008B1E820C2
:208310006076E87D092801DB0A2801DDE8206076287E08B1042805DB802801DB862801DB9E
:20833000E820607604F11807294638460DF0ACFC291D112207F12C0008F044F895F8280023
:2083500004F11809002804BF84F86060A87D04D095F8290084F86000688DA4F85600687E78
:2083700084F85800A87EDFF8048184F85900E87E822784F85A00287F98F8D76084F85B0098
:2083900098F8E63084F85C70394F84F85D6005F11D01E763042684F8406098F8E72084F867
:2083B0005E3009F1490084F85F200B220FF02AF9607E00284ED1687800284BD1287EA77E7E
:2083D0008DF800000FB1EA20607605F11701E720FEF71EFC94F8600028B1287E022808BFE8
:2083F00001208DF8000098F8E7009DF80010884203D0E8206946FEF70BFCA77E1E4C601C50
:20841000007808B10FF0C4FAB8F8BA0019490880C7B1032F12D0052F05D0012F03D0022F41
:2084300001D00FF0B5FA022060700CF031FC4FF6FF70A8F8BA001149088005E00CF028FC9D
:20845000032000E0012060702720287030460EF0B9FC01E02A20287028460BF009FBBDE83B
:20847000F883C046DC33002094180020D8110020217A0100161C0020583500209A190020F9
:208490002DE9FE4F694C064694F83D00002800F0BA80DFF89C81B6F84210B8F8BA00884225
:2084B00040F0B18006F128000EF01EF9002800F0AA80002798F8BD0084F83D7010B1022055
:2084D0000EF080FC5148007810B101200EF07AFC307C400905D310200EF074FC80200FF0A1
:2084F00097FA20200CF084FF494D05F120000BF0D3FE7268517810782B4600EB0120C0F349
:208510000321C0F3003584F8391000F00F0184F83A50C0F3031584F83E1098F8E30088F8EC
:20853000C0500F2804D0884202DDD57805B9014688F8A11098F8A1A083F84070BAF10F0F1F
:2085500009D194F83B0002285DD10DF007FD06F0ABFBBDE8FE8F2F480078012803D0012037
:208570003946FEF751FADFF8CC90D9F80400804700900EF055FA28482F4DDFF8A0B00768FE
:2085900098F8A1202B786868391A980091FBF0F05BF822100CF084FD6F605BF82A000191D0
:2085B0001F4DA860E8600BF0D1FF019829680DF0D1FA08F0C3FE0098D9F80810884794F89D
:2085D0003B0002280DD118480BF066FE98F8A10034F810204FF4707181401348891A0EF01B
:2085F000ABF8318902200AF07FF804F1200528460BF052FE0B48A062616B28460EF09CF887
:2086100010200FF005FABDE8FE8FC046A3330020EC340020EA1D002088190020F08E010047
:20863000C81D0020FD300100FC340020641B0020D8110020001800206C1D00202DE9F04FC9
:20865000154601F00708C1F3C2074FEAA119044683460C22ADF1240D0021684609F031FA3C
:208670006248B8F1000F36D0B8F1010F7ED1228801A9A6780A80E41C8E7014F8011B01F067
:208690000F018DF8081022880DF10A031A80BDF80A30A41C4FF0000C6B75019ECDF818C0B8
:2086B0004168B14207D1017A9DF80820914202D14189994208D006990C30491C06290691D5
:2086D000EED96046614601E0017840788DF800108DF8010022E014F8013B14F8016B8DF802
:2086F000003000228DF801600C38079210F80C1F994202D14178B14207D00799491C0629BD
:208710000791F3D91046014603E04168027A4089687501918DF80820ADF80A0003A807F00A
:20873000FFF89DF800109DF80100B8F1000F11D0B8F1010F1AD1019904989DF808209DF832
:208750001460484086EA02010918BDF80A20BDF8160004E09DF80C2051409DF80D20504047
:20877000401803D1EF701FB1022F05D0002039E02188281DA41C0180B9F1010F27D0B9F1C5
:20879000020F2CD1BDF80A10281DC91DCA10214607F018FEBDF80A00C11D04EBE104F0B161
:2087B000401E811000EB5171C910C9B26D182B798710012600EB577121F00701401AC0B23A
:2087D000401C06FA00F0FF301840287107E0291D20460BF01FFC207804EB8004641CA4EB5A
:2087F0000B04A0B209B0BDE8F08FC046A01900202DE9F04FADF1840D209002F093FD0EF098
:2088100011FC0026012804D10EF0F4FD022808BF01265B490868C0F38150012806D151F82F
:208830000C0C0127010E07FA01F00643554800780EF054F8544D2C46286038B1FF2204F1A5
:20885000400107467F1E01F8012BFBD1209909684FF0000901F0FF02FE2A1DD0DDF880C05E
:2088700001F0FF074A460123FF2F0ED0B84203D903FA07F73E4201D002207EE001F0FF019E
:2088900047EA0909611881F840205CF8041F521C01F0FF07FE2FE7D1092006F031FC20986E
:2088B000002124220823606017A80FF0F7FA4FF0010804F1240017AA8DF8748041460FF086
:2088D000E9FA236843B3002794354FF0040BBA4608FA07F0064219D119EA000F04BF07F0EF
:2088F000FF0141F4C04105D0E019209B90F8401053F82110254804F02BFEF8B24FF0FF31B2
:208910000EF0BAFB2368C5F800A001E0C5F800B07F1C2D1D9F42DBD301A8002130220823A3
:208930000FF0B4FA1A4E30780025102101AB0990184A009504F108000FF0A4FA0DA828223F
:20895000082329460FF09AFA0DAA7068124914952B46139004F160000FF08CFA0F4951F8B8
:208970000D0C474620F4F85040F4005041F80D0C0B4EC1F8FF7F2846376021B0BDE8F08F85
:20899000B43F0050F9350020FC2E0020007FC767F8900100A5700100914B01000D3009403D
:2089B000080009402DE9FE4F544E0746301D00688047534C00258346A01C05701FB10DF0FD
:2089D000DFFC0AF093FE94F83800B04610B1E06B00B180470AF058FBDFF8749109F11C00A4
:2089F00090F900000EF00EFF0DF0E0FC0EF000FF0EF0B4FD0EF0A6FDDFF808A107270AF104
:208A1000240656F8040B00B180477F1EF9D13E480560456005614FF470018160C1600AF139
:208A3000040007680FB10CF01BFB38484E4600688AF80E50BA3EC0B112E048460CF0E0FEC2
:208A5000029002A80CF00CFB21E048460CF0D8FE019001A80CF004FB14E068460CF000FB98
:208A700008F0B0FC00280090F7D129480078012803D028460146FDF7C7FF2648264F057016
:208A900007F12409786A0028DFD109F10409B86A0028D2D17D62BD622048A06187F82E508F
:208AB0001F4BE36187F82F501E4A22621E49616287F830501D4BA362204B1D4A63601D497D
:208AD000E2621D4F25701E4A2163204BA2601D4967631D4FE16058462761D8F80810636139
:208AF000884706F1BD015220FEF792F896F8D7000BF0AAFB2846BDE8FE8FC046001800200E
:208B1000C816002088180020C81D00200C300020EA1D0020FB350020A810002033F50000AF
:208B30000D7D010035690100B17B00007DDA0000B56D0100017A0100C1BD0000E7EE000086
:208B500035AE00002D3E010085FF0000D12F0100921200202DE9F04F0546824660480E4609
:208B70000178ADF1140D0EF0C9FC5F4C00283FD0DFF8808108F104000068012914D0287A1B
:208B9000022835D15749504602220F4620310DF06BFF38B903208DF8080007F116016846D0
:208BB0000FF0BEF8EA4623E095F8089014F809A080470A274FF0640B8E340390207A4845C1
:208BD00006D15246204629460EF01CF9012804D07F1E04F10C04F1D104E00027F772A07A3F
:208BF000BB463073D8F80810039888475F4672E021464FF0000864278B468D6B91F83100BC
:208C100086F81E804446D9460AE099F800106D1C2034ADB234E099F83100641C6D1DA4B282
:208C3000A04217DDE8780028F5D028790BF086FF514608220DF018FF0028ECD1E878B0779F
:208C5000288800047060287986F80B80F077A87847463073DBF83440002F08BFBB46C5D04C
:208C700086F81E8042F219000DF10A010BF0B0FB0EF018F883461D4801786427454681463A
:208C9000A94228DDA07F0028BFD0E07F0BF056FF514608220DF0E8FE0028B6D1E07A022878
:208CB00003D0E07A58B1612710E0616858460FF043F8BDF80A200E495143814201D9474661
:208CD00004E0A07F6C2740F00800A07730462146202207F077FB384605B0BDE8F08FC046BA
:208CF000C81600206C1200200414002034140020808D5B00001800202DE9F04F0746880F4F
:208D1000ADF1140DC0F0BC8000200AF085FE62485D4E4FF0000900F11408C8F800900120E0
:208D300048F81C6C0DF0FEFF58480EF0E1FE584DBC68CB4640F60A0605F1140095F82010FD
:208D50002A7995F82130A5F816908246C5F818B001F0F0010680012A85F8201003F0F000CF
:208D7000A4F8029040F0010085F8210001D17B7CC3B1B8680088A6F10801814208D0B0F521
:208D9000C15F05D0218B4FF60F400840208304E0218A4FF60F4008402082B86887F8119056
:208DB00004F0F8FDB868694604F036FF68460EF007FE3346D91F4A1C00E03446666836B12B
:208DD0003088834203D0814218BF8242F5D1C4F804A0607B00F0F000607305F13C000EF0F1
:208DF000B5FF8068008881421FD082421DD03E8D06B397F8340097F83560C7F82CB000F0E6
:208E1000F00087F8340006F0F00040F0010087F8350007F12803AB619AF80D00A7F82A90AD
:208E300000F0F0008AF80D0004E0DA4605F1580080E80006B9680A8A4FF6FF3010400882F0
:208E5000D8F800000028FBD0A87AC8F8009070B901200DF0E5F901280FD0607B00F0F000E5
:208E700040F0010060730B480EF042FE05E00CF047FA0028FBD00CF061FAB86848F81C0C59
:208E900005B0BDE8F08FC04601010E0415350000D80D00203D2A0100081004402DE9F84F5F
:208EB000884605460EF094F801464FF6FF70884210D042F21C0BAB4509D0ABF10100A842AF
:208ED00005D01A38A84202D0001DA84205D10EF015FB10B16820BDE8F88F534C480000EB6D
:208EF000C1002418D4F8027017B9D4F8066016B3D4F80610B94208BF692000F09380607854
:208F1000401E12D0401E09D0801E14D1D8F80000874200F2818081427ED30CE0B8F800000B
:208F3000874279D8814277D305E098F80000874272D8814270D33D4F78688047ABF11A0A79
:208F50002B463B4E0090A3EB0A03012B25D90A3B012B14D9DB1F3DD1207862780021301871
:208F700008F0AFFD637840460EF07EFC834298BF181C02D940460EF077FC02462BE00DF0F2
:208F90002BFCBF68B8F80010884243DD207862784146301807F016FA23E00DF01DFC8146A1
:208FB000404649460AF088FCBF68A9EB00005FFA80F9B9F1000F2DD020786278414630188A
:208FD00007F000FA1B485146A94218BF401C80F8009006E0627820784146301807F0F2F967
:208FF000BF680AF11900A84204BF002086F887005846A84213D196F8870096F88610421855
:20901000322A01DC08430AD1022086F88600302586F887500098B8476A20BDE8F88F00982C
:20903000B8470020BDE8F88F2C860100001800205C320020FA3100202DE9F8435F4D80462E
:2090500095F83800002798B12A6F8AB1D5F8900070B142F21A0069469047D5F89000804781
:2090700030B19DF8000018B1B8F1E10F08BF0127534A02F1E70000780CF088FF407B0228C2
:209090000CBF05260126524C2068002800F09380B8F1000F914676D0B8F11B0F02D1017D59
:2090B000052970D1B8F1E90F2CD05FBBB8F1E10F16D10EF057FB90B12068C18AC9080FD2E4
:2090D00099F8C810817699F8B6104A1C89F8B620406881703046FEF749FEBDE8F883206819
:2090F000B8F11C0F1DD1216A002951D08847354900200978206001295DD00146FDF784FC49
:20911000BDE8F883F1200EF006F921688F7E57B90EF028FB20B12068C18AC90801D2CFE74C
:209130002068474630E04868098908F0D1F9216848680088000905D395F8387017B10CF05B
:20915000CFF92168C88AC00811D3087E00F07F000876087D032803D1487E40F00400487601
:20917000F0200EF0D8F82169206888470FE0887E401E887614490127F0200F700EF0CBF8FA
:2091900012480078A7E70027477008F087FD2068C08A000A0AD395F8380018B999F8D7004E
:2091B0000BF052F899F9D6000EF02CFB0020206010200EF02DFCBDE8F883C046C8160020B2
:2091D000D8110020EA1D0020F83500206E1C0020A81000202DE9F843634C5C4D5C4EDFF856
:2091F0007881604F94F8E4100846401E0B2864D8DFE800F07E2C43062343062343067967BA
:20921000042907D001220A2945F8212C14BF0220032004E0202045F8210C0120024684F8CF
:20923000E200002045F8390C0827C5F8FF7FC5F8F37F45F8392CBDE8F883052914BF092015
:209250000620002784F8E400376078E094F8E170383D0120002FC5F81B0004BF06200021DE
:2092700002D00021F160032084F8E400032045F8010C31603068800861D294F8E4103548C9
:20929000012703290ED00068456800216022052300914046A84794F8E400062814BF0A200B
:2092B0000720CFE700684568002160220523022000904046A8470420C4E70EF0D7FDBDE874
:2092D000F8832648264F0026012506600E203D6005F02EFC02200CF0BBFB84F8E45084F884
:2092F000E360BDE8F883002038600C25786024E04FF08059D9F8A0010168202088472C3DCB
:209310000F2045F8010C41F61D56C5F80360D9F8A401466800214FF4C07207230225404669
:209330000095B047D9F8A401C66800214FF4C07207234046B0470120386084F8E45004F152
:2093500078000EF0C3FDBDE8F883C04639400C4038600C40A401001000A00C402C500C408F
:2093700004800C4034600C40F01200202DE9F04304466668A7680D46ADF1340D0EF0B2FDBC
:209390003178012903D10EF0A9FD0020A9E04FF0010886F800800EF0A1FD28787070687887
:2093B000B07068687060A868B060E868F06028693061287D3075687D7075A87DB075A8698C
:2093D000B061287F3077687F7077A87FB0774FF00009C6F82090C6F830904D46756275638C
:2093F000B562B56386F82C50102386F83C3086F82D5086F83D50786805F082FE204605F061
:20941000F5FB204607F05EF970B937480068C16838688847786805F08BFB0EF063FD357092
:209430000EF05CFD2C465BE001A82946302208230EF02CFD0694387BCDF800902B4A0990AC
:20945000B96801AB06F180000EF01CFD01A82946282208230EF012FD05942549386901AAB4
:209470002B46079006F19C000EF004FD01A82946242208230EF012FD8DF81C80B07838B972
:2094900006F1D000294601AA0EF004FD19483061707838B906F1EC00294601AA0EF0FAFC20
:2094B0001548F06001A82946242208230EF0DAFC0695ADF814501149079406F584700A22DE
:2094D00001AB0EF0CBFCB969FA6906F140000EF022FA0B4A06F16C00042123460DF0B4F846
:2094F00020460DB0BDE8F083D001001045C5000069570100A97C0100A17C0100B90C01006B
:20951000517A01002DE9FE43604C614D0E46B00959D35D4800F1280980464DE00178D02959
:209530000EDBD02909D181783970C17879700179B97085687D60C168B9600EF0FEF947E0D0
:2095500004F1080528600AF093FA28460BF088FD3EE0884798F83010491E88F83010A96807
:209570008847009801788DF80410A0604778CFB1DC2F0DD0DD2F0BD0E42F09D0F32F07D06F
:20959000DE2F05D0DF2F03D0E82F18BFDB2F0BD104F06CFA9DF80400162805D168460BF074
:2095B0005FFD01E00AF064FA9DF80400162803D004F108000BF054FD48460CF021F9002847
:2095D00069680090C5D1F00BA846C00305D0314F07F0F8FE00280090A0D1700905D32E20CE
:2095F0008DF8040001A80AF043FA700805D325208DF8040001A80AF03BFAB00805D3262026
:209610008DF8040001A80AF033FAF00805D327208DF8040001A80AF02BFA300905D329201F
:209630008DF8040001A80AF023FAF00908D300208DF805002D278DF8047001A80AF018FA51
:20965000300A08D300208DF8050030278DF8047001A80AF00DFA6068D8F8041080B1884795
:20967000616800270091D8F8081067608847009804F1080630600AF0FBF930460BF0F0FC65
:209690000020BDE8FE83C046A81000208818002000180020EC1D00202DE9FE4F074610466F
:2096B000002F00910CBF4FF0E80B4FF0000B002900F0AB80BBF1000F40F0A98060B178684A
:2096D000401E7860F82101707868401E7860002606703889801C3881009C4FF000094FF0CF
:2096F000020ADFF83081CDF80490083C14F8080F00F00F010F2900F08580012820D0042894
:209710007AD1454D95F83800002875D0296D60688847061C26D03889B7F84C103018801C35
:2097300081421FDB78686D6D6168019B3A46801BA847B8B178683D89801B786076195AE0E8
:209750000098019E042309EB0001C91C11F8010FFF2841D021283DD13889B7F84C200B3002
:20977000824202DA1A20BDE8FE8F7868B8F8D020401E7860121202707868401E786098F8DB
:20979000D02002707868401E7860019D057098F8D2007A68107098F8CE2078681201401E9B
:2097B000786042F00F02027098F8C0C098F8A1207868401E786042EA0C1202707868401E9B
:2097D0007860212505707868F61DB6B2401E7860052505705B1EB9D17868C6F30121401E9A
:2097F000786041F0880101707868401E7860067038893618B61C3E81BAF1010A09F1080969
:209810007FF474AF7868B86501E04FF0E80B5846BDE8FE8FD8110020C81600202DE9F04F66
:209830005D4C054600208A46ADF12C0D80461746B4F952100A93DDF850B084F88901B4F906
:2098500050008BF80080401A40F6F87101400829A8BF012080F29280B4F95000401CC0F322
:209870000B030DF04DF80646D4F87C01B384854207D194F88801410824BF00F0FE0084F872
:2098900088010A98006800B940463062387B00F00F00022814BF4046B868BAF1000FF061F4
:2098B00075D00AF19C000EF065FA002865D128460BF036FF051C1AD1E36BC3B10AF0DCF9C6
:2098D000236C08902BB1216CE26B304606F062FA38B9236C5BB9E26B3046694606F05AFA83
:2098F00028B1012384F88931E06B3060E66394F88991B9F1000F4AD10DB9E56B95B12A6899
:209910003046294606F046FA18B92D68002DF6D108E00223286884F889312246306092F86D
:2099300089912E60B9F1000F31D10A980179504604F01CFD0146012926D094F88901002850
:2099500025D1012923D0E16B09B10868D0B9387B00F00F02022A1AD1C01118D141B9206CDA
:20997000A8B1216C3046424606F014FA28B10EE03046424606F00EFA48B902208BF8000086
:20999000464604E00968E0E7042084F8890130460BB0BDE8F08FC046D80D00202DE9F04F30
:2099B000504E7068ADF11C0D80474F4A934611784E4D04919BF80020B168012A0BD0012471
:2099D0008BF8004088472878012805D020460021FDF71AF800E08847464C454FDFF8189165
:2099F000E06807F1B001814206D1494691F90000002818BF002761D170688047404B05909C
:209A1000002003F13801A7F8B2000F78002F07BF4FF48601021C39492022804639489A4649
:209A30000378CDF808809B0904D20078000938BF012000D302208DF80C008DE806003649BB
:209A50003148324B006802AAFCF748F8B7680028A08030D4494691F900009AF800302C4AFD
:209A7000401C08702C49002B92F90000E16000F1010010700CBF40468020B4F84410254BC3
:209A90004FF67F720A4010430143A4F84410B3F8BA00B3F8BE10A4F852000822A4F85010BD
:209AB00003F1D80104F1470318460DF0ABFD0598B847012702E00598B84747467068804719
:209AD000B16817B9049A8BF8002088472878012803D000200146FCF797FF384607B0BDE817
:209AF000F08FC04600180020DE1D0020EA1D00200C15002048190020E71D002000004F8C96
:209B1000C8160020FD350020181C0020F1140000E61D0020D8110020BC1500202DE9F04F1A
:209B30008A4609AF4FF08051ADF11C0D90463D69059001F5D8700490D1F8B001D7F808B0D2
:209B50004169069327208847524C4FF00309143CC4F884970126C4F87C67C4F880970220D1
:209B7000C4F8FC06F868C4F8080430460EF0B7F8D4F808040008F8D2D4F88C07800F28BF4D
:209B9000B14655D2681E41460C238DF800000DF1010011F8012B5B1E00F8012BF9D1022D0C
:209BB00019BF0020011C98F80C1000208DF80D108DF80E008DF80F000099C4F83C15019BA9
:209BD000C4F84035029AC4F84425039BC4F848353968BAF1020F4FEAC542A1EB0A08A2F5DA
:209BF000002106D34FEA4A52A2F580026FF315021143264A0A43C4F84C258246C4F850855D
:209C1000BBF1000FC4F854A5214DC4F858B511D02E6078682060C4F808B030460EF05FF87F
:209C3000D4F88C078008F8D3D4F88C07000801D3CA4627E0C4F88497D4F88C0710F0030FC8
:209C5000FAD1D4F8800720F00200C4F880073F7D47B1049F3868016A2720884738680169FF
:209C700027208847C4F87C670598C4F8806748B12E6006982060C4F80880C5F80064206253
:209C9000C4F82880504607B0BDE8F08FC801042000004842184002402DE9F04F894609AFF2
:209CB0004FF08051ADF1240D9246059038683D69079001F5D8700490D1F8B001D7F808B098
:209CD0004169069327208847504C4FF00308143CC4F884870126C4F87C67C4F88087022073
:209CF000C4F8FC06F868C4F8080430460DF0F7FFD4F808040008F8D2D4F88C07800F28BF86
:209D1000B04653D2681E51460C238DF800000DF1010011F8012B5B1E00F8012BF9D1022D7D
:209D300019BF0020011C9AF80C1000208DF80D10019B8DF80E0000998DF80F00029AC4F8DA
:209D50003C15B9F1020FC4F84035039BC4F844254FEAC542C4F84835A2F5002106D34FEAB0
:209D70004952A2F580026FF315021143254A079D0A43C4F84C258146C4F85055BBF1000FE2
:209D9000C4F85495204DC4F858B511D02E6078682060C4F808B030460DF0A1FFD4F88C0723
:209DB0008008F8D3D4F88C07000801D3C14624E0C4F88487D4F88C0710F0030FFAD1D4F82B
:209DD000800720F00200C4F880073F7D47B1049F3868016A272088473868016927208847FF
:209DF0000598C4F8806740B12E6006982060C5F800642062079FA760A762484609B0BDE831
:209E1000F08FC046CC01042000004842184002402DE9FE4F524D286808B90DF0B9FD554CF1
:209E300004F13800DFF83C91DFF840A1DFF8408107789FB94D46686880474B490F7847B9D5
:209E50005246A96817782FB983234246137088476DE0A96802234246137075E0D4F89810FB
:209E700009B104208847676D2A685FB1D06D20B102210023B8472A68676D106E10B108218E
:209E90000023B8473C4E306A3C4F016CF86888474D46834668688047029033480578002D9B
:209EB00048D150460078002844D1D4F8841000208847F42001A90AF071FC9DF90400304DA3
:209ED00058451ADCAB79C3B9D9F8081002988847A878042801D00DF05BFD04214046AF79A8
:209EF0000170D4F88410781CA87109B1032088470320688100F0A8FB27E083214046346ABA
:209F10000170636CF8686A4600219847B6F90600BDF90010884214BF002001200AF05EFD33
:209F3000D9F80810029888470835287838700CF0B9FF0AE0022140460170D9F808100298FF
:209F50008847D4F88410042088470E480078012803D000200146FCF757FDBDE8FE8FC0461F
:209F7000A810002000180020FC350020FE35002000360020C8160020481900200C1C002000
:209F90006C1C0020EA1D00202DE9F8434E4E84460120002430704D484F4D04704C48DFF836
:209FB0003481047005F14E000088B14614EA03074FF0020606EA020608BF002E13D120461F
:209FD0004FF0E04710401F4008BF002803D11D2007F002FB54E0454695F90000401E287025
:209FF0000DF0F8FA4CE0424692F900303C4E5B1E137043F20842824207D06F8E931C8342E2
:20A0100003D0BA4218BFBB4217D1304608300068826C60469047008843F6030181420BD0C1
:20A03000204602F0F3F898F9000000283FD098F90000002838DD42E06F8EB5F86A1043F6B8
:20A050000400884205D0B84203D0B5F84E20904203D12248007803281AD1B1F5505F05D09D
:20A07000080B0BD31D2007F0B7FA07E01D480168304601F5C071016004F09CFC0DF086FA3E
:20A0900098F9000098B198F9000000280CDD16E0022811D0204602F0B9F898F9000030B1B8
:20A0B00098F9000000280ADC0DF072FC07E020460146FCF7A9FC02E0204607F08DFA89F813
:20A0D0000040BDE8F883C046EA1D0020E01D0020DF1D0020E61D00200C1500206E1C00209C
:20A0F000601900200C0100212DE9F0410C4601467138022840F29680133824D04D4F4C382F
:20A110007AD0401E61D0401E48D0401E36D0401E29D0401E1AD008460DF006FC06460B2E0B
:20A1300011D0424D6868804741498046B000425CBF1840184278394620460DF063FAA96831
:20A15000404688470CE0F420BDE8F0812278022A68DA3949601C01EB820104220DF052FAA0
:20A170000020BDE8F081217832295BDA334FCA00201D02EB0112B9181822EFE72678022E38
:20A1900050DA2C25601C05FB0671102239310DF039FA05FB0670C06C6061E1E72078022888
:20A1B00040DA2C2101FB0070667890F83800B04238DD23786278394602EB430201EB4201C2
:20A1D000022201F5DE71A01CC8E72078022829DA2C2101FB0070667890F83000B04221DD97
:20A1F000227860783223394603FB020000EB4000032209189031E6E72078022812DA2C210F
:20A2100001FB0070667890F82800B0420ADD6278207839468018420002EBC00289180A2214
:20A230007C31D0E7E820BDE8F081C04600180020FC7E010050250020C42B002014270020D4
:20A250002DE9F84F994692468B4606460DF04AFE4E4C0090B4F95210B4F950000AAF401A2F
:20A2700040F6F871014008297CDAB4F95000401C6FF31F30A4F85000B4F950800CF040FBBD
:20A29000054606F178000CF0FDFDC5F808B085F826A0C5F80490A5F824803D48EE6097E862
:20A2B0000C00202100271940104005F1100383E8030004F13C0085F827700368002B43D10B
:20A2D00029460BF0DFFB002844D0A6F8C08095F8270040F0800085F8270086F8C270E079FF
:20A2F00020B1207810B1E7710120207200980DF0F5FD206C002845D12078F0B96079012885
:20A3100040D00DF0EFFD0646A07988B9A86808F05DFD40B930460DF0E1FD04F1EC000421DC
:20A330000DF0D0F92EE004F1C8000DF0CFFD02E0184901200870304622E001200CF0D4FE70
:20A3500019200DF075FB1DE004F13C0029460BF099FB50B9B4F9500000F6FF706FF31F30FF
:20A37000A4F850006FF0010809E0A6F8C08095F8270040F0800085F8270086F8C270009862
:20A390000DF0ACFD4046BDE8F88FC046D80D0020FDEFFF9FF73500202DE9F04306460520BA
:20A3B0000327F08270683775401E7060411E716096F89610017096F89600ADF1140D18B1BE
:20A3D0004FF6FF70A6F89400B6F894507068411E7160291201707068411E716096F89440D7
:20A3F0000470337D7168481C3062581E0870308906F18B01001D308101A80DF091FC06F138
:20A410008B05002437488DF80C70DFF8DC8034650078B465002841D04FF0040986F86940EF
:20A43000F08A86F86B90C00932BF404640462930007886F86A00296806F16C0319606A6858
:20A450005A602889188186F874700DF057F828BB06F16C0029460DF063FC244D286810F424
:20A470007F0F0CD086F82C90286806F12C01012200F47F0030633046FFF70EF9286810F048
:20A49000FF0F0BD02A2086F83C00286806F13C0100F0FF003064304604F000F940460094FB
:20A4B000401C0388394601AA3046F9F745FA071C02D1304604F01CFA3946DC290BD0DD29FB
:20A4D00009D0E42907D0F32905D0DE2903D0DF2918BFDB2902D1304606F09CFB05B0BDE8D1
:20A4F000F083C04600170020911200201C8D01002DE9F0434D4CDFF8388194F83F6000276B
:20A51000ADF1140D002E57D198F89660002E53D0C768007A454600F00701C0F3021900E065
:20A53000BF1C0E46701EC1B24EB17A783878B5F8BE6000EB0220B042F2D1022710E005F19E
:20A550009406443600E008374846411E5FFA81F9A0B3304639460CF0C3FE0028F3D00327DE
:20A5700094F83F0040F0040084F83F0002A80CF0CFF801200CF026FC04F134018720FFF79E
:20A59000B3FD04F13C018520FFF7AEFD04F13D018620FFF7A9FD04F13E018820FFF7A4FD9B
:20A5B0000120009004F134060196B5F8BA30394602AA0520FCF72CFE002F33D198F8A1109C
:20A5D0000F292FD0404690F8C0208A422AD090F8BD0038BB1748007820BB17480078012896
:20A5F00003D001200021FCF70FFA144C606880472146134C94F83B20022A11D194F83820AC
:20A61000FF2A0DD00F4A176857B9576A47B98968884704F1200009F03FFE08F067FD01E033
:20A630008968884705B0BDE8F083C04664330020D811002096180020EA1D0020001800208A
:20A65000641B0020A81000202DE9FC414948484C494F4A490278A37865893878042B71D12C
:20A6700001F13C06337803F0F003337000268E630DB901256581884641490832554300FB54
:20A6900005F291F838500092002D50D00D46AA6F002A4CD0EB6F002B49D004F108016846C7
:20A6B00090478446374B2179DFF8E8E060791A68BCF1650F31D0BCF1000F28D1107D052842
:20A6D00011D13148017871B9186890F82C00042809D119686D6D906D096B3346A8470028D6
:20A6F00008BF1A2016D0294D6868804728490E68002E08BFA96807D0A96804F10C029642A6
:20A7100013D03668002EFAD1884738780FE0704606706046FEF790FC22E082F8690082F88F
:20A730006A107046E96F06701C20884718E01A49009E04F10C076161B6FBF0F138460CF031
:20A750007BFD0DE091F83C30083280005543884603F0F0036843886343F0030381F83C30D5
:20A7700098F8740000F0F00088F87400BDE8FC816C1C00200D1C00206C1D00200C150020F4
:20A79000C8160020A81000209512002000180020C81D002000360020219E0000F8B5071CEA
:20A7B00000F0A180B86840F6030120264A1C02E04068761EF6B260B15EB10388994218BF4F
:20A7D0009A42F5D1F9681CC828311CC149C881E849007868BA690026BE6168B3F968486815
:20A7F0000078022818BF42F0020297F82700002300F00700401E09D0401E04D0801E08D1EA
:20A810004FF0805304E04FF0804301E04FF00053324697F82700000908D397F8270010F0F5
:20A83000070F03D04FF0807032430343B7F92440084621467C68A0470DF054FB2A4C054694
:20A85000B4F95200401C6FF31F30A4F8520004F14C00016881F827600CF063FF28460DF07B
:20A870003DFBB4F95000B4F9521088423BD1F86890F8C20000280CBF0520072004F0A8FF2A
:20A8900004F5AA742568F868854208BF656890F8C240002C0CBF0468341C80F8C2604DB174
:20A8B00095F8C23023B92868A04228BF041C01E085F8C260A4B10D480068B4F1FF3F12D05D
:20A8D000B4FBF0F101298CBFB4FBF0F10121F86878300DF0BFFAF86878300DF0F7FAF8BD48
:20A8F00001200AF06FF9F8BDD80D0020149101002DE9FE4F514C814604F13C0A50460DF0D0
:20A9100025FA90468B46074608F0010000900DF0E9FA0325BBF1FF3F019015D1266C2EB1B1
:20A93000206CC068814508BF206C0BD00DF0DAFADAF8006074E0F168894570D10DF0CEFADB
:20A95000301C71D0B0F924B058460BF0EDFC00286AD0216C814248D0B84217D104F1C800F2
:20A970000CF090FAE06B0068E06397F82700394640F0040087F827000AF110000BF082F8BC
:20A990005FEA980022D3E76B01221BE017B9832D20D01CE03968884225D104F1C8000CF0DB
:20A9B00071FA39680868386091F8270040F0040081F827000AF110000BF064F85FEA9800AC
:20A9D00004D300224846394607F0FCFF832501980DF084FA6079012829D004F1EC000221B4
:20A9F0000CF070FE23E03F68D0E7009F90F82720012505FA07F13E1C41EA020180F82710BA
:20AA100014BF0C480C480BF00BFE5FEA980004D3E16B48462A4607F0D5FF832504E03668B0
:20AA3000002E88D10DF05AFA01980DF057FA2846BDE8FE8F0100020401000104D80D002095
:20AA50002DE9FF410646080BC0F092804A49C8680025012788460D70C3694F722BB1016AE0
:20AA7000C90802D304212A469847444908F170002A460DF058F942480DF03AF8D8F80C0063
:20AA90004168414C886808B9C86820B1A4F11C00C5613C490160384608F0BEFF25603B48C6
:20AAB00044F81C0CB1684D80B068028840F60200904208D0B2F5C15F05D00B8B4FF60F42F0
:20AAD0001A400A8304E00B8A4FF60F421A400A8200F1080C7774ACF10702531C00E0394626
:20AAF0004F6837B13888844503D0824218BF8342F5D12F464F60487B00F0F00040F001002D
:20AB1000487308F13C000DF021F98068008882421BD0834219D0308DC8B196F8340075855F
:20AB300096F83530F76200F0F00086F8340003F0F00040F0010086F8350006F128024A6095
:20AB5000487B00F0F000487301E0C8F86050B068694603F061F868460CF032FFB06802F03E
:20AB700019FF20680028FCD02560B06844F81C0C0090BDE8FF81C046D80D0020A17101005D
:20AB900015350000510007061C10044001010E042DE9F041494CDFF828814B4F4D4D0028C1
:20ABB00054D198F8A10022680F2852D0454E0F20118986F83900012007F096FD98F8970067
:20ABD00068B198F8BD0050B13846404998F89820376B01632830B91820310BF0ADFD98F8FA
:20ABF000C000716B0F2806D03948B06206F120000BF0A2FD01E00BF0EFFB206840680078EA
:20AC1000000956D3686880470646606A074670B10022387E800905D23A4657F80C7C002F19
:20AC3000F7D104E004F1240039460AF077FCA96830468847002F3CD0787E394640F010000D
:20AC5000787604F124000CF0EDF832E0226898F8A1000F282DD107F14001166D08784EB1BF
:20AC7000082298F8E76087F84220864202D0E820FBF7CEFF98F8BD0010B102200CF0C0FE97
:20AC90001548001D00688047676A6FB1397E01F0FD013976890903D3797E41F01001797625
:20ACB00057F80C7C002FF1D1A968884708200CF0AFFE20460AF0D4F9BDE8F081A8100020F0
:20ACD000D8110020641B0020A8340020137D01006D2F010000180020001800202DE9F04FCD
:20ACF0000546287CADF12C0DC0087FD34A4C05F12809B5F842806068CDF8249080470A9096
:20AD10004648A16800688A4610B90A9888474EE04FF0000B07465C46787E30F07F003BD013
:20AD300079684E464878367A4A46C446DE46CB1CC0F38100864219D1022806D0032815D182
:20AD5000491D48460CF0CCFA0FE0DE7899781288584601EB0621914207D119785A78ACEBE7
:20AD70000101B1EB022F08BF01208646BEF1000F12D044B1207D012812D16168087840F089
:20AD9000100008700CE03C46607E40F010006076207E40F08000207657F80C7C002FBBD143
:20ADB0000A9851468847B4B9BBF1010F1ED005F11C0106A80B220CF025FC0CF0B7FB014664
:20ADD0003020009006AF0197B5F842304A460120FCF71EFA0AE01249491E91F8380018B125
:20ADF000C86C08B1804701E003F0BAF810208DF8080005F128010DF10A000CF049FD0127BB
:20AE10008DF81670B5F84200ADF8140002A802F0D7FF0BB0BDE8F08F00180020CC100020EA
:20AE3000C91600202DE9F04106467478ADF1180D002C40F089804948B6F896100088884225
:20AE500018BFE82406F18C0101A80D460CF056FA01A80BF049FC424B40B996F8990040B1AC
:20AE7000A3F13700007820B9E8246DE0002086F89900002C68D196F8990000280CBF012076
:20AE90000520042737752946F0820DF10E000CF035FA706896F89840401E7060411E7160F2
:20AEB000B6F896800470327D71680024481C3062501E0870308934651A78B465801C308178
:20AED000A2B386F86B70296806F16C0001606B6843602A8902810CF011FB06F16C0228BB63
:20AEF00006F18C0110460CF01BFF1E4D286810F47F0F0CD086F82C70286806F12C010122F8
:20AF100000F47F0030633046FEF7C6FB286810F0FF0F0BD02A2086F83C00286806F13C01AE
:20AF300000F0FF003064304603F0B8FB0094304603210DF10E024346F8F7FEFC041C02D1C1
:20AF5000304603F0D5FC2CB174701A203070304608F08EFD06B0BDE8F081C046921200207D
:20AF700000170020208D01002DE9F04706464FF00108ADF1600D0922B07D8DF84C8006F150
:20AF900017018DF84D000DF14E000CF03BFB464D68688047814616A98120FFF7A5F8707D68
:20AFB000002854D09DF85800022817DA042000238DF80300347D8DF802809DF858708DF8C4
:20AFD000013069468DF80040781C8DF85800D220FCF7FAFC812016A9FCF7F6FC00274FF0C5
:20AFF000FF0A3C46307D8DF8217008A980F001008DF82000D120FFF777F8C0B99DF82200A6
:20B01000FF2814D08DF800006946D420FFF76CF820B1A96848468847192042E0307D69469D
:20B030000DEB80000461D420FCF7CEFC01E08DF822A08DF82440307D8DF8234008A98DF896
:20B050002000D120FCF7C0FC7F1C322FCADB307D00279DF84D208DF840000DF14E018DF812
:20B0700041700DF142000CF0CDFA8DF84B80D02010A9FCF7A9FC071C0FD1307D3146102222
:20B090008DF828000DF129000CF0BCFA30690AA90F90D320FCF798FC0746A96848468847FA
:20B0B000F8B218B0BDE8F087001800202DE9F04FFF25ADF1140D8DF800504FF6FF79ADF84B
:20B0D0000290ADF804900AF011FDDFF81CB104900BF1020000880027001F84B2082C64DBE0
:20B0F0004E46B046C246201F02A9082280B20AF05DFEBDF80800814508D1BDF80A1089451A
:20B1100006D1BDF80C20924502D107E0BDF80A1051EA000317D1BDF80C30A3B9BDF80E10C1
:20B1300008466FF30E0060B908460830844206DA0CF02EFC04980CF00FF800204FE008469A
:20B150002EE0241F2EE0C20BD30327D1BDF80C20854203D18E4208BF90451FD0C5B28DF812
:20B1700000500E46ADF802609046ADF804809DE80600384607F05CFE80B9BDF80E20A01AE5
:20B1900007F18851001F083280B292B20AF00EFEBDF80E003F180837BFB201E0BDF80E008B
:20B1B000241A083CA4B2082C9DDA09F019FF3FB10C484FF088513A460CF018FD0CF072FB95
:20B1D00004980BF0C9FF5A46507800281CBF0020011C03D1C7F58054391DA0B2518005B0C6
:20B1F000BDE8F08F04E00100741E00202DE9F8430020444C8DF800000CF01BFD2279484EB9
:20B21000424DDFF81091012191404FF6FF725218024096F83800628120B3326F12B342F2AC
:20B230001A0069469047384867790378A3B19FB99DF8003083B1D6F8940068B1804749460D
:20B25000491C2A78097830B1678908314A43B0FBF2F0C019608167799DF80010608907FB08
:20B2700001006081A078002847D1294F386AC06B80474E4680466489297870783B6A0830CB
:20B290004443D86B8F0080476968234D2A787578224E3C23401AB0FBF7F103FA02F0B1FB57
:20B2B000F0F205F108034243891AB1FBF3F25A43891A05F10803691A641896F8581096F81E
:20B2D0003C5098B2083401F0F00107FB048341F0020107FB0032736596F8744086F8581079
:20B2F00005F0F000B26340F0020086F83C0004F0F00086F87400BDE8F883FFF7A5F9BDE829
:20B31000F883C0466C1C0020F83500206C1D0020481900200C1C0020981200200C1500202A
:20B33000C81600202DE9F0434A4D95F8E700ADF12C0D00287AD13F4F387B01240021242294
:20B3500085F8E7407E6885F8E6000823C5F8106101A80CF087FD002605F10C00069601ABFE
:20B37000ADF814603449079632460CF077FD334905F1300001AB32460CF070FD304905F104
:20B39000540001AB32460CF069FDB96820468847DFF8BC802B4808F104037A7B00781868FA
:20B3B000C0F3815922B1B9F1030F04D185F8E140B9F1030F1ED0B9F1020F1BD0B9F1010FE4
:20B3D0002DD14FF08059D9F8A4011F4F456831464FF040521C23032000903846A847D9F83E
:20B3F000A40131464FF400720923456800943846A84714E002200AF069FDB9F1030F0CBF95
:20B410004FF47A7142F21071104800685435B1FBF0F128460CF01EFD28460CF057FD40469A
:20B430000068C00802D230460AF050FD0BB00020BDE8F083909001004FC600006515010097
:20B450003D120100F935002000A00C4014910100B03F0050F01200202DE9F84F06463079F9
:20B470008028D4BF0020E82071790027092901DB0A2900DDE820B17909B1042903DB80298A
:20B4900075DB862973DA002871D1DFF8E88098F8A1000F286BD0B8F8BA104FF6FF7088420C
:20B4B00065D0B8F8B410884261D0F079324C01280BD040B1FF285AD194F83B00002856D194
:20B4D00001252F4602E0012500E00225DFF8ACA00AF12000834608F0DFFE0AF1100008F0D3
:20B4F000DBFE04F1200008F0D7FEDFF89C9009F1040000688047224B84F83B500246FF2175
:20B51000002060631D6884F83810002D0CBF0121011C012F84F83D10554684F83C7008BF35
:20B53000032085F840004846816810468847B11DE820FBF76DFB711DE720FBF769FB311D16
:20B55000E120FBF765FB94F83D00012802D120200CF056FA0B4898F8A1104FF47077A8626F
:20B5700007FA01F000F2636158460BF065FEBDE8F88FC046D8110020641B0020EC340020FD
:20B59000A8100020752B0100001800202DE9F84F05464448DFF8109183462E18093699F85F
:20B5B000380034788846B0B1D9F8501099B10BEB8507786B00F0FF0088478246D9F85010D1
:20B5D000786B00F47F008847504480B218B131784018001DC4B23548007801280CD198F888
:20B5F00008704FB1324898F80930C1190E79C05C0019401DC4B200E000260D2D09D106EB0C
:20B610000408B8F1F80FD8BF2A4F1CDD0CF0C0F905E030198046801C0BF014FA074697B96A
:20B6300002200BF00FFA011C0AD00BEB050090F825001A270870204E4F70307807F03EFF73
:20B650000020BDE8F88F08F10202384600210CF08BFB07F10C00002174220CF085FB07F141
:20B670003C00FF2110220CF07FFB07F12C000F2110220CF079FBE0197860022D3E810BDB1B
:20B690000B2D09DA7868401E78606D1E05703889641EE4B2401C3881A7F84C403846BDE82D
:20B6B000F88FC046DC8C0100C8160020A4120020B0900100DC1000208818002070B5ADF1E0
:20B6D000380DFFF72FFE3E4908682822082340F00200086001A800210CF0D0FB394D3A4E4D
:20B6F0003A49A878002301AA079006F1EC000CF0C1FB00213022082301A80CF0C7FB2878F2
:20B7100000241921ADF81C40314A099001AB009406F170000CF0B6FB2822082301A82146CD
:20B730000CF0ACFBE8782B4901AA2346079006F590700CF09FFB01A82146302208230CF0BD
:20B75000A5FB01206A78ADF81C001A2101AB099206F18C00204A00940CF094FB1F49224617
:20B7700006F1C80013460CF079FB1D480CF0C0F91C4A2346042106F128000AF065FF25463B
:20B790004FF6FF70A6F8C400052386F8683006F1580181E830004FF4FA70C6F85C01C6F8D6
:20B7B00060012B4686F8C73033717371B371F37133727372B372F3720B4A13700EB070BD4B
:20B7D0000020094008910100D80D0020757601000508010071040100313D01000D5F010005
:20B7F00051BA00002D440100F63500202DE9F84F81463E48067899F8010000286DD13C4CC9
:20B810003D4DDFF80081607820B14746381D00680F2E5AD1374F786C417A0F290FD103F0AB
:20B8300013FC786C90F83000002856D094F83800002852D0206C00284FD080474DE003F037
:20B8500003FC0AF087FDAC6B0F2E2ED1786C2C4A417A2A4E52F82110B160407ADFF8ACA012
:20B8700052F820000AF10803F0601868203CA04201D80CF08DF8200801D30CF089F8D8F897
:20B89000040080475146834609781F4889004C430168641A446002F09BFCD8F808105846D3
:20B8B0008847B06808F052FEAC6B19482146286205F118000AF040FF786C90F824000F28D2
:20B8D0001CBF012085F8420007E08047114920352960B9688847BDE8F88F2D2089F80000CD
:20B8F000484608F0C5F8BDE8F88FC04679120020C816002048340020A8340020C81D00207D
:20B91000F08E010000180020043004406C1D0020853D0100A54901002DE9FE4F0BF0C2F974
:20B93000434C04F10C020290116820614FF40050491C1160694608F04BFDDFF8FCA0DFF837
:20B95000FC9094F8330000285FD0A66B94F8310000254FF0FF0BA0462F4654E0B07F8008B3
:20B9700021D3F07F09F0EAF80146082268460BF07BF8C0B1716802980CF0DEF92D498142FC
:20B9900011D8F07FB7770AF0F9F986F81FB0DAF80000804794F8323013B15B1E84F8323036
:20B9B000D9F80810884798F830006D1C2036ADB236E0F078800822D3307909F0BFF8014626
:20B9D000082268460BF050F8C8B13088010402980CF0B2F91749814211D83079F7700AF0AF
:20B9F000CDF986F804B0DAF80000804794F8333013B15B1E84F83330D9F80810884798F853
:20BA100031006D1CADB2A842D3DC94F8320048B1A046666B98F8300000254FF0FF0B2F4653
:20BA3000A8429BDC04F1140008F0FCF8BDE8FE8F0414002000A493D60418002000180020B5
:20BA5000F8B5424C0D46A8085DD2E8087CD301260420E6720AF03AFA0BF08EFE04F1580283
:20BA700082E8030004F13C000CF070F90746E06877B1FD6850B1854208D0EB6933B1286A27
:20BA9000C00803D328460421002298472846E06041682F4A0978116041681268097891422B
:20BAB00007D087692FB16FF0FF0100224FF00073B84702200AF00AFA112003F021FB667166
:20BAD000E168087C10B12079012803D00E2003F017FBE16849681F488F680FB9CF681FB1D9
:20BAF0000021C1611C4F07601C4A40F2FF711160002787611A4941611A480BF0F9FF192006
:20BB10000CF0A4F9F8BD04F14C0630460CF01EF9FEF744FE30460CF019F925F0020504F12B
:20BB30003C0158B9E80803D208460CF00FF958B104F1C8000BF0A6F9042101E045F00201F2
:20BB500004F1EC000BF0BEFDF8BDC046D80D0020D02108400010044051000706000004602F
:20BB70000A000040098D0000F0B5454C454A322100274FF6FF75ADF1340DA4F10C0636F829
:20BB90000C0F854206D07089430803D3C30B6AD202421DD1491E07F10107F0D10C3C3220C5
:20BBB0006FF0310734F80C1F8D4202D06189490804D2401E07F10107F4D102E0204608F072
:20BBD000FFF9002F52D14EF660200AF0A7F84DE02D49014228D009A800210C2205F071FF6B
:20BBF000022033888DF8080003A9ADF80030684604F0B0FA28B104A90A680AA80260496841
:20BC100041603088214BADF82600981DBDF8261000881022ADF8240015A008F053FD71896A
:20BC30004FF6FE4008407081718944F6FF700023084070813946312914BF491C191C8F4222
:20BC50000ED0880000EBC1002218205A854202D05089400802D2002BEDD003E0164600E079
:20BC700003B933461E46304608F0AAF90DB0F0BD21526573706F6E64696E673A2030780064
:20BC9000800B002000B0FFFF0090FFFF681700202DE9F041414C0746206800287BD0DFF81B
:20BCB0000081002F18BFE92F17D10AF0CBFF4546297801EB81016918C1F8020095F8B560B1
:20BCD000287800EB800029184E702878401C2870C0B20A28A4BF00202870324D68681C2F5D
:20BCF00032D0314E4FB1F079032806D1E12F04D0002088F8B200072000E0052008F02AFDC7
:20BD10002468F07903280ED06CB1002084F86900E18A2648C90938BF2938007884F86A0092
:20BD30003846FDF789F998F85700012833D168688047044606F042FDA9682046884700206F
:20BD500088F85700BDE8F08180470646A96894F82F0002281ADA216804F124000BF062F8F2
:20BD700094F82F00A968401C84F82F00304688472068007D252819BF012088F85600012059
:20BD900088F8550000202060BDE8F08130468847F120FDF751F9BDE8F081C046A810002080
:20BDB000A031002000180020F4190020BA1200204549B0B5044601F13800007800287FD0DB
:20BDD00094F88B00002871D13520207504F18D01112204F16C000BF015FC04F13C00FF2174
:20BDF00010220BF0C1FF04F12C000F2110220BF0BBFF94F88C0004F13C0500283ED0401E2C
:20BE100029D0401E14D0401E58D12A20287002272764042305F8103C4FF41022226303212C
:20BE300084F86B10204607F0F7F9071C3BD137E02A200A272870042327644FF44C1205F805
:20BE5000103C02212263204684F86B1007F0E4F9071C28D124E02A200227287004232764D0
:20BE70004FF4102205F8103C01212263204684F86B1007F0D1F9071C15D111E02A200227C2
:20BE90002870042327644FF4502205F8103C00212263204684F86B1007F0BEF9071C02D1A3
:20BEB000204602F025FD381C0BD1B0BD01280AD1886C8047002808BF002002D0192000E0A2
:20BED00018200BF0BDFCB0BDC81600202DE9FC410746BE6833687D68986B20F4FA60986349
:20BEF000AC6B44B13168886B40F4FA6088634FF0FF30BDE8FC81AA6329630024EC776C63A2
:20BF10000CE09DF80000296B08706B6B286BAA6B401C2863581C6863501EA863A86B90B90B
:20BF30003168886B40F4FA6088636A6B6878296B0128A1EB0201296303D1EB6838469847DB
:20BF50006A6B144646E005F14000694609F0C8F80028D6D50BF0C6FF204F8046387820B98D
:20BF7000022009F0B3FF0120387040460BF0B6FF1B49086840F4007008603168886B40F445
:20BF9000FA6088636878D8B9696805F1EC000BF089FF90B9AC630BF0A5FF0646387818B1E9
:20BFB000022009F055FD3C7030460BF097FF1027696B286BEF77401A2863686BBDE8FC8173
:20BFD00095F82D0030B1686B20B1AC6305F19C000BF038FF2046BDE8FC81C046F435002068
:20BFF000301000402DE9F04F09AF9A4616460D46ADF1440D3C89D7F80480109000203F8887
:20C010008DF83C00BC4201DAC24501D30BF0C0FC002E69D0364810F80690042EA4EB090493
:20C030004FF00000A4B2B8BF01205FEA000B0EBF3F1BA04400242F49082307A8A7EB09074C
:20C05000BFB211F801295B1E00F8012BF9D1290E00F8011B2B0C00F8013B2A0A00F8012BB7
:20C070009DF83C1000F8015B234D06702868109A4369686898470646B6F1FF3F24D00120BA
:20C090008DF801009DF83C608DF802600BAA04928DF800B08DF80390CDF80880CDF80CA09C
:20C0B00002218DF81410ADF8164007ABADF818702E686868326A01936946904706462868D2
:20C0D000826968680FA99047002E18BFE4200CD1B9F1000F08D0444448460BA911F8012B90
:20C0F000401E04F8012BF9D1002011B0BDE8F08FB4900100B7120020E435002070B5424CC1
:20C110000646683C607800287DD0B4F95200B4F95010884213D0304609F002FB38B9216C2F
:20C1300021B1216CC9688E4208BF206C38B1B0F9241002224FF0E043304604F0D7FE0BF0B6
:20C15000D1FEA178002943D0491EC9B20029A1703ED10BF0C3FE002565702078E66058B1E3
:20C17000012008F02FFD022008F02CFD06F140004FF0FF310BF096FE06F140000BF05EFE64
:20C1900006F178000BF056FE06F19C000BF052FE04F1EC000BF04AFE04F170000BF042FE2F
:20C1B00004F590700BF042FE04F18C000BF03AFE04F1C8000BF03EFEE56004F128000AF037
:20C1D000C1FD307C012817D10E2002F0B1FC13E00BF084FEE068864204BF0020E06006F16D
:20C1F00040000BF02BFE06F178000BF023FE06F19C000BF01FFE002504F5AA742068B042DF
:20C2100014BF6560256070BD400E00202DE9F0473F4C8246A07830F0010708D0042806D09C
:20C23000032804D0052802D00BF0B2FBA078394F667904210528DFF8D090DFF8D080397070
:20C2500006F10101CDB265711ED1022D57DCBAF1010F54D04E4631684868098905F038F9BB
:20C27000306840680088000905D34146087810B109F036F9657928460BF07EFD8320387008
:20C2900009F02CFFBDE8F087234EE73E96F8B810A94234DB032832D008F032F9A0780428D4
:20C2B00009D14146383991F8380020B1D1F8841009B102208847207996F8C510421C9142D5
:20C2D000C4BF401CC1B24E46217131684868098905F0FEF8306840680088000904D34146E1
:20C2F000087808B109F0FCF8FEF780FFA078042808D08320387008F095FBBDE8F087E12088
:20C3100005F06AF9BDE8F087A8100020001700206C1C002000360020BF1200202DE9F04352
:20C33000404C054660781F4690460E46ADF1440D012803D0FFF7C2F901206070AEB1364845
:20C35000337801684FF0010909FA03F001420CD0B8F1000F6E6008D0C5F808800BF0C2FDFE
:20C37000A178022903DB0BF0B9FD002051E004EB8102491CC2F85451C9B2A1700BF0AEFD21
:20C390004C461FB909A80BF00BFA09AF386828607868E860387C2874B86868617869E86107
:20C3B000B8696C742862788A6882F86800B1A8610021A02205F1280005F083FB6846002199
:20C3D000242208230BF06AFD8DF8184005F1400000216A460BF05EFD684600212422082300
:20C3F0000BF040FD0D49069505F1780000226B460BF034FD68460021242208230BF032FD2D
:20C410000749069505F19C0000226B460BF026FD284611B0BDE8F083D42108403171010077
:20C43000017D0100D80D00202DE9F8430AF0FAFF3E4E054615F00A0F4ED0376C002F4BD024
:20C450003869B9693A4A34464FF0000840F00A0028400843B8613B69C4F84080A2F11000FB
:20C4700000F108021168994307F11003116093E806000168121C91430160394604F14C00D3
:20C49000814609F0FFFA022104F1EC000BF01AF9A06C08B3F8684068007802281CD197F8D4
:20C4B000270040080CD297F8270080083CBFA06C20640FD3A06C2730017841F0020104E080
:20C4D000A06C2730017841F001010170A16C484609F0D8FAC4F84880326C05F0020005F058
:20C4F0000807074316D102F1100003C8002301EA03072840002F08BF00280BD0106997692C
:20C51000054072644FF4804106F1EC003D4395610BF0D8F8306C30B906F13C000BF016FC03
:20C5300008B103F0A1FABDE8F883C046D80D00201C1004402DE9F8438146D9F80870386808
:20C55000066CD9F8045046646A6CAB6CA86B16F4F06F0146A2EB03082AD1F00911D27009F2
:20C570005DD301B395F83C40641EA14298BF0C1C4846214609F060F9A86B001BA8630DD07D
:20C590004DE081B1484609F057F995F82D10A86311B9002843D101E00020A86305F19C00DC
:20C5B0000BF050FC3BE04846414609F037FD36E0F20A19D24FF00008444602E0A86B401EA6
:20C5D000A86340B34846012109F036F93868446814F00F04C0F80480F0D0286B401E28639A
:20C5F000686B401E686316E0386844680022202904F00F044260CCBF20270F1C48463946CF
:20C6100009F01AF9C7F12007B845C8BFB8464846414609F003FDEC77484606F06BF9B0098B
:20C630000BD3A96A49B10F46484609F03DF9A86218B94846391D07F057FEBDE8F88370470B
:20C6500070B53F4C0646A07EADF1200DF0B994F85C0082281AD0394B40F2016046F25C0510
:20C67000ADF8080034491868ADF80A50426A086802A99047812814BF6FF07F009DF90C0067
:20C690000AF0E3F894F85C10226B505494F85C00822814BF401C002004F1180584F85C00C1
:20C6B00094F85C0005EBE00292F82C00411082F82C10400807D294F85C00401C84F85C00B6
:20C6D000C0B28128ECDB94F85C0081282CDA05F14401E120FAF79CFA02204FF6FF738DF8B0
:20C6F0001800A17EADF8103031F0020018D0012919BF07208321082080210022493500923B
:20C7100004AA0195FAF784FDDB2807D0E52805D0F32803D0DF2818BFE8280AD1607603E027
:20C73000304605F0F7FA04E02A203070304607F09FF908B070BDC046181C002068190020DA
:20C75000DC3300202DE9F04707467D68D7F8089090460E460BF0C6FB8246A86A002864D197
:20C7700005F584700AF08EFB0024EC772E6250466C620BF0B3FB0BF0B5FB2F4E3378824679
:20C7900023B9022009F0A2FB0120307050460BF0A5FB2A49086840F480700860384641468F
:20C7B00009F082F8A862C0B93846414607F09CFDA878D0B9A96805F1D0000BF073FBE8B954
:20C7D000AC621020E8774946284605F01BFB0BF089FB8246307840B323E0D9F80010886BEB
:20C7F00040F020008863A87810B12046BDE8F087A96805F1D0000BF055FB10B1686ABDE831
:20C81000F0873846414607F06FFD1020AC624946E877284605F0F6FA0BF064FB82463078E0
:20C8300018B1022009F014F9347050460BF056FB4FF0FF30BDE8F087F5350020301000401D
:20C85000B0B505463C4C2878616BE1281BD0A16BE92815D0A16CF0280FD0E16CF12809D0EB
:20C87000E16B20B92969002004F08AF90DE0481CE0630AE0481CE06407E0481CA06404E001
:20C89000481CA06301E0481C6063697831F07F0050D0C8092AD24FF48050014609F018FD43
:20C8B000F0B12F78BFB14189CA0B38BF41F4804106D342894BF6FF711140418141F4004146
:20C8D000418142894EF6FF71114041814FF4FA6009F024FA04E042894BF6FF7111404181CD
:20C8F000287838BBE069401CE061B0BD4FF440704FF4807109F0ECFC071C16D0287858B980
:20C91000788940F48070788140F40071798140F6B83041F0010105E078894FF6FF6101402D
:20C930004FF47A70798109F0E1F9287810B9A06A401CA062B0BDC046681700202DE9F043C1
:20C95000DFF8E0808946054617464FF0FF31ADF13C0D40460BF0A6FA334C04EBC50466689D
:20C9700025680BF0BFFA2168096800290BD42968002905DCB9F1000F09D04FF0FF3108E0E0
:20C99000B9F1000F03D00BF0A9FA002442E02968491C29600BF0A2FA286802283ADA1FB95B
:20C9B0000DA80BF055F90DAF38686860B76800213022082301A80BF069FA4FF0000906949F
:20C9D00001AB307B194A09903946CDF8009005F12C000BF057FA01A82422082349460BF00E
:20C9F0005DFA012705F1640001AA8DF81C7049460BF050FA05F1480001AA39460BF04AFA17
:20CA1000706802F07DFB0A4A05F118002346042109F01AFE40460BF05DFA20460FB0BDE821
:20CA3000F083C0469C3500208090010081680100997C01002DE9F04106AF3D793E68984635
:20CA500004460B1CADF1180D074611D0012B15D130797379641C3870B17904F8013B337A86
:20CA700004F8011BB17A04F8013B7389181201E03178707804F8011B04F8010B8AB9002D03
:20CA90000CBF42F20C0042F20D00694607F0A0FC9DF80000BDF8003004F8010B181204F850
:20CAB000010BB8F1010F34D0B8F1020F39D1002D0CBF42F2020042F203000DF1020107F07C
:20CAD00087FC7589CDB1681E01468B100DF1020201EB5371C910CBB2811000EB517121F088
:20CAF0000701401AC0B20121401C01FA00F0D15CFF3080F0FF000843D054E81D0DF10201A9
:20CB1000C210204603F05EFC7089C01D04EBE00407E0002D14BF02210121204602F0AEFDA8
:20CB30000419E41B06B0A0B2BDE8F0812DE9F04390460A68D8F800401678814600271D462B
:20CB50003846ADF1140D531C242E0B6053D112F8016F5B1C4C2E0B600ED1AA68E41C24F05D
:20CB70000304241D54F8040C494606F077FE2968EF600127091A2960462E1AD1E41C24F0E0
:20CB90000304241D54F8040CE41C029024F00304241D54F8040C002749460390AA68ADF897
:20CBB000047001A803F086FA2968EF600127091A2960532E1FD1E41C24F00304241D54F808
:20CBD000040CE861C8F80040288B0090A968EA69D9F800004346F7F787FDD9F80040002741
:20CBF00014B10119C9F80010D8F800402968EF60091A01272960662E0AD12B8B23B9E41DAF
:20CC100024F00704083403E0E41C24F00304241D1FB9E9690E700127EF60C8F8004005B096
:20CC3000BDE8F0832DE9F041074602240D46ADF1380D78888DF82840391DADF820000320B1
:20CC50008DF832000A680DF12A0002604968416008A803F0CDFA00283ED50DF12A0003F0FF
:20CC7000C7FA002838D502A839460C2203F0AAFBAE8805A8868029680160254E0024A04667
:20CC9000306A0794E0B103A804F0E2FDB0F1FF3F20D107F03BFD0546322D11DA06208DF801
:20CCB00000000523ADF8023006F078FBADF80400306A46699DE80300182202ABB04728B1CB
:20CCD000B8F1010F06D009A0012406E06D1CA8B208F074FF08A000E00AA07988102207F057
:20CCF000F1FC20460EB0BDE8F081C0464661696C65643A20307800C04A6F696E65643A203D
:20CD1000307800C044656E6965643A20307800C0EC1500202C4870B50568B5F1FF3F08BFBE
:20CD300000250AF07FF901284DD108F0B9F8142849DB26482649002601230660254A0B6095
:20CD5000254C136020680028FCD1264A131D2349186820F00300014321480068C0080CD208
:20CD7000106810F0030F0AD041F003001860106800F003000328FAD101E041F001011A48BC
:20CD90001960006820B1194800682846F5F718FF174818490660184D0A686FF35B4245EA6C
:20CDB0000200086015490868C0F30130012806D10A681348104040F400320A60086020686A
:20CDD0000028FCD170BDFEE71C130050840460425C600C40082204430C0068420400002040
:20CDF000B03F00500040034080012843000120438C210840482003400000390104000940EA
:20CE1000FFFFFCFCD0B5071C68D0F96B002965D0B7F84000002861D00E78002017F1300143
:20CE300003D097F83810052901D0002856D0387A032809D1384609F081F94FF6FF718142CB
:20CE50004CD0388002213972294C206BB61E22D0B61E04D0761E3ED0F61E39D0D0BDB7F8B7
:20CE7000400001283AD1384608F092FC78B14289510B0CD34EF6FF711140418141F40051AE
:20CE900041814EF6602008F049FF09F091FC206A401C2062D0BDB7F840000D281ED13846B0
:20CEB00008F076FC38B142894FF6FF611140418141F400714181398809A0102207F002FC93
:20CED000201D04210AF01EF9E06A401CE062D0BD401C2063D0BD3846F9F79CFFD0BDC04652
:20CEF000436F6E6669675273703A20307800C046681700202DE9F04F09AF3C897D681646DD
:20CF10004FF0000A0246002EADF1440DA04610933C888DF83CA05CD0304810F80690042E31
:20CF300003DAA8EB0900C8462D18F868A4EB080407AB0827A4B2C01D10F801C97F1E03F89C
:20CF500001CBF9D1080E264F03F8010B080C03F8010B080A03F8010B386803F8011B9DF819
:20CF70003C101E704369786898478346BBF1FF3F2AD0042E04DA03208DF80000022002E0F3
:20CF900002208DF800008DF8140002959DF83C608DF8026001218DF8011038688DF8039022
:20CFB00007ABADF816800BADADF81840026A0193109E049569467868039690478346386810
:20CFD000826978680FA99047BBF1000F18BFE42000D1504611B0BDE8F08FC046B4900100BA
:20CFF000E4350020394833492DE9F047012500240570DFF8C480DFF8C8900C702F4901F1AF
:20D010006A06378882460220104014EA030608BF00280FD120464FF0E04710401F4008BF7F
:20D03000002832D0424692F90000401E10700AF0D1FA2AE0424692F90000401E1070BFB98D
:20D050004A8E43F2084320464646934204D191F84010090938BF281CFFF7D8F848460470DE
:20D0700096F90000F0B196F90000002817DD1DE0B7F5505F07D114481249006800F5C07051
:20D09000086001F097FC0AF081FA48464246047092F9000030B192F90000002806DC0AF09A
:20D0B00077FC03E020460146F9F7AEFC8AF80040BDE8F087E01D0020E61D00200C15002064
:20D0D000DF1D0020601900200C010021EA1D00202DE9FE4F83460020304E00907068019172
:20D0F00080472F4C0290E06804216A4605F0C6FA2C4DDFF8B4A0DFF8B490DFF8B8802C4E32
:20D110002BF0010725F00105BD4213D0504620F00100B8421CD1494691F9000010F1020F26
:20D1300018D03068826B91F90010E068904781280ED10FE0414691F9000010F1020F09D046
:20D150003068826B91F90010E0689047812801D00AF01EFC3068C66A1749019AE0685B4647
:20D17000B047061C01D50AF013FCBD4207D0504620F00100B84204BF49460E7001E04146F8
:20D190000E7001200090E06804216A4605F076FA0249029889688847BDE8FE8F00180020BF
:20D1B0000C1C0020E1E5000039030100DD1D002068190020DC1D00200C1500202DE9F84FA2
:20D1D00007463248DFF8C89000EB4706183699F83800348890468B46B8B1D9F85010A1B1AB
:20D1F0002C4D05EB8705686B00F0FF0088478246D9F85010686B00F47F008847504480B2C5
:20D2100018B131884018001D84B225481230007801280CD198F808604EB11F4898F809307D
:20D2300081190D79C05C2418641DA4B200E00025281980B209F006FC0646184890F8009058
:20D25000D6B13046002122460AF08EFD4FF00008A41937700D4986F8018006F18000746068
:20D27000CA5D358159460AF0CDF94846314606F025F94046BDE8F88F8DF8007068461A21B9
:20D2900003F0C8FC1A20BDE8F88FC046F0880100C8160020DC8C0100B0900100881800207A
:20D2B000921200202DE9F04F364E0025ADF1340D07464FF0010AA846A9460C93DDF858B0CD
:20D2D0000B914AE017F8020FAD1CADB2401E1BD0401E09D0401E04D0401E36D1022C34D1E6
:20D2F00038E0032C31D135E0072C2ED1B9787878FB1C40EA0120A6F84400186806F1480268
:20D31000106086F859A025E0052C1ED1CDF80890B91C0A8802A80280897881700B9803A9C0
:20D33000FBF718FC9DF82A00A0B1029B40F0020000F0F7008DF82A0006F15002039310680B
:20D35000049003A805F0DEFC04E008EB0400801C1FFA80F8E7196419A5B23846694608F0AE
:20D3700061FC041CAED1022D03DC4D466720A84600E048460C990D800DB0ABF80080BDE866
:20D39000F08FC046A03100202DE9F84F0D46064628684FEA900A3248504502D3287A0228F8
:20D3B00002D00320BDE8F88F0AF09CFDDFF8B4800090D8F8580108F5AA79B04214BF0024DC
:20D3D0000124A00080F0040059F8007006F19C0083460AF0CFFC68B957B107F19C000AF06B
:20D3F000C9FC38B93846022100F0C0FF074602E0022700E000271C4800686FB998F88801AB
:20D4100040F0020088F888010098C8F87C610AF065FD0020BDE8F88F2A68A10001EBC40100
:20D4300049440A612E7A0E76BAFBF0F1012998BF012158460AF00EFD58460AF047FD009868
:20D450000AF04CFD012F07D1D8F88001B8F9841198F886210AF008FC8320BDE8F88FC046D0
:20D4700040420F00D80D0020149101007CB5354C054694F8A1000F285ED03348697E0078F7
:20D49000890959D2297E002841F00201297639D069684A1C1078801010F0030F32D000F0C1
:20D4B000030002280ED1B4F8B4304FF6FE70984208DD56791179002001EB0621994208BF20
:20D4D000012004E004F1AA00491D09F009FFC8B9687E696840F0010068764A78C2F38102F0
:20D4F000022A2DD1491D4A7809784FF6FF7601EB02218E4224D1297E00F0EF0041F02001E3
:20D5100029761CE0687E114E40F0030068763078B0B994F8D7008DF80000FF238DF8033037
:20D5300094F8E6608DF8016094F8E7508DF8025068460AF095FB7CBD687E40F00100687623
:20D550007CBDC046D8110020C91600209F1B00202DE9F0470D4606465FFA85FA280824BFC3
:20D570002E4845402E494FEA8A03C85885EA00023240C2F300672B4A06EA0504B043224081
:20D5900006F4E0240243B4F5E02F01D1500E14D306F4E020074310D002F4E027B7F5A027D5
:20D5B00007D0B7F5803704BF22F4003242F4A02203E022F4803242F4C022DFF86C80CA507E
:20D5D00008F1D00739680122002002FA0AF40C4218BF101C5FEA000906D1F00D04D34146B8
:20D5F000C5F3805001F80A00300E0BD30AF07AFC290E34BF0021211C3A68A2431143396008
:20D610000AF06CFCB9F1000F06D0F00D04D34046C5F3805100F80A10BDE8F087006000A0F8
:20D6300000100840007F077F002002402DE9F04117460D460AF056FC324C80462078832653
:20D650006DB16D1E04D06D1E55D0681E11D00EE0B4F8C4004FF6FF71814202D005E0206C0D
:20D6700008B9802648E0206C808C388044E0032642E0386800215022054604F022FA022795
:20D6900004F5AA7C04F5B272A5F110015CF8040B41F8100F137A0B735068486052F80C3BE0
:20D6B0007F1E18448860F1D1206C002808BF02200ED0206CC068276C286297F82600236C27
:20D6D00085F82C00D869226C6862106AA8620320E76B8FB105280FDAFA6801016A5097F8FC
:20D6F00026204C192273FA6962603A6AA2603F68401C40B2EDE7387040460AF0EFFB3046BE
:20D71000BDE8F081D80D0020F0B52A4A2A491778ADF1140D002F44D02C48077837F07F0721
:20D730003FD1488C2A4F254D2A4B401C0024488407F16806012097F87410287001F0F00135
:20D7500087F8741019783C67012902D02146F9F75BF90AF0DFFA1C4D281D006880470746DE
:20D77000029402201C4A164B8DF80C0021468DE803001068314602AAF8F7B0F917490028EF
:20D79000A1F12001088008D40E49154C91F90000401C0870A4F114000660A96838468847DF
:20D7B00006E0888C401C88840020107009F028FD05B0F0BDFE3500206C1C0020DF1D0020C0
:20D7D000D5190100E61D002000180020003600200C150020EA1D0020181C00205C1C002045
:20D7F0006819002070B5344C611C09780225ADF1280D032958DB01A902F0ACFC002853D0ED
:20D8100007AA012313700AF0A9FA8DF81D000AF0A3FA0021264E8DF81E0030460AF02CFAFC
:20D830008DF81F00194630460AF026FA8DF82000294630460AF020FA8DF821003046032167
:20D850000AF01AFA1B4E8DF82200002130460AF013FA8DF82300194630460AF00DFA8DF8F9
:20D870002400294630460AF007FA8DF82500032130460AF001FA00929DF81320BDF8061036
:20D890008DF8260018460B2301F09CFD012802D008F08EFF08E024342068401C20604FF450
:20D8B0007A7008F023FA002528460AB070BDC046905F0100804F1200681700202DE9FC4710
:20D8D000314CA11D0888401C088009F0EBF90026B046354681462846694604F045FB824635
:20D8F000BAF1FF0F4CD09DF80030606B23B900EB4A104068010402E000EB4A104168484687
:20D910000AF01AFA864203D29DF800700646D0466D1C0A2DDFDB1E4D281D0068804794F800
:20D9300033106FB9A26B08EB88030026FF27491ED218D67013791771C9B284F833100CE0C4
:20D95000616B0022FF2701EB48118A77CB7FCF7794F83210491E84F832100C4A643BD9B25A
:20D97000136804EBC1013C310B6052684A6094F88C10491E84F88C10A9688847BDE8FC8780
:20D990000AF0D8F9BDE8FC8704140020E090010000180020E0B501880025A1F6020159B1BC
:20D9B00043F20402891A04D0491E57D190F8246000E00226C76901E0C67B4769002F4DD0B4
:20D9D0003F1F052044F2380357F8041F0A04120C934203D0401EF7D13F1D01E0C1F303459E
:20D9F000002D3BD01F4B3046401F18D01C4A401E10D0001F0CD0801E0DD0C01E06D00F38A3
:20DA100019BF1A1C6032184A443204E0121D02E0121F00E0083A1068C0F3834003E01A4605
:20DA30001068C0F303200F2806D0A84216D921F4702141EA004110E0761F0AD0761F08D0C4
:20DA5000761F06D00F3E1CBF21F4702141F4802103D121F4002141F4E0213960E0BDC0462B
:20DA70000011005020130050C4100050F0B5064600210B22ADF1240D0DF119000AF074F902
:20DA90002E4F2F4C3078C01E14D0801E04D0143810D0801F01282DD801208DF8180006F1F4
:20DAB0008B0103A80AF03CF9032538788DF8145068B112E000208DF8180006F18B0103A839
:20DAD0000AF02EF9032538788DF8145028B9B4F8BE000225ADF8020005E00DF1020004F161
:20DAF000D8010AF01DF98DF80A50B4F8BA00ADF8160017E002208DF8180006F1320103A8A2
:20DB100009F0C6FE0DF1020006F1280109F0C0FEBA34208806F11C01ADF816000DF11900E5
:20DB30000AF0FBF80B208DF8000077788DF80170684600F045F909B0F0BDC04600170020D4
:20DB5000D81100202DE9F84F8A463149044601F1B400007828B920465146F7F7CFFBBDE862
:20DB7000F88F0A25884642F2107B20465146F7F7C5FB98F8B410002848D19AF80060D4F854
:20DB90000090002937D023480168C88AC20832D280094FF0000702D3087D15282BD009F067
:20DBB00061F898F800308446002B0EBF09235B1EDBB20A2003EB830208EB0201491C0A78CE
:20DBD000964207D0002B0EBF09235B1EDBB2401EF0D110E0D1F8011060460AF0ADF86421A9
:20DBF00001FB09018B4505D942F242706426401AB0FBF6F717B90020BDE8F88F20686D1ED0
:20DC100007442760B1D10AF095F86120BDE8F88FA0310020A810002080B50288A2F6020743
:20DC30003FB143F20502BF1A14BF002090F8240000E0C07B2C4AD2F88832401F0B6048D039
:20DC5000401E3CD0001F30D0801E24D0C01E18D00F380CD0D2F890024860D2F89402886064
:20DC7000D2F8BC0220F0784040F080503AE050694860D06A8860506C20F0784040F0704043
:20DC900030E010694860906A8860106C20F0784040F0F04026E0D0684860506A8860D06BFA
:20DCB00020F0784040F0C0401CE090684860106A8860906B20F0784040F0A04012E05068E1
:20DCD0004860D0698860506B20F0784040F0405008E01068486090698860106B20F07840FC
:20DCF00040F02050C86080BDC41000502DE9F8432E4D686A002856D000202D4E0090301D87
:20DD1000006880476C6A009F8046A74223D0607E30F07F001AD0608A401E80B2608210B129
:20DD3000607EC00812D354F80C9C05F1240021463A4607F0F3FB6846214607F025FF95F8B1
:20DD50002E004C46401E85F82E0002E0274654F80C4C002CDBD1B1684046884795F82E00F6
:20DD700078B1144800780F2802D01348007840B9124C204606F090FA4FF47071204609F0FA
:20DD90005BFAF026E92509E002F080FD607EC00834BF66706570204603F080FF684607F0E1
:20DDB0002FFD041CF0D1BDE8F883C046A81000200018002079120020C91600207C34002096
:20DDD00070B50646304930780D5C401F1CD0083851D0401F4FD0284608F034FE041C0DD178
:20DDF00030780C2808D1706830B1301D07F038F9284608F027FE0446002C43D02A46204646
:20DE1000314609F0FFFB37E0B07810BB327A307C51005410401901F00E01091804F03800CB
:20DE300040182430C0B208F00DFE041C2AD03146182209F0E7FB04F118006060716824221F
:20DE500009F0E0FB6068243060617169327C0E46D6E7012816D12435E8B208F0F3FD041C5D
:20DE700010D03146182209F0CDFB04F11800606071682422EBE7344624B104480078214608
:20DE900005F01CFB70BDC04658900100EC1D0020F8B509F039FE04F0F9FC09F04DFE0446CD
:20DEB00004F00C000C284BD0E0081ED208F0ECFA264E376805460120014609F031F83168CC
:20DED0006943884211D2224C8220B0FBF7F0291A204609F0BFFF204609F0F8FF0120F8F771
:20DEF00057F9204608F0CEFF2CE0200928D2194809F0DBFD0428FAD0174A610905D220B1CD
:20DF10001168104621F0010103E01046016841F001010160983210684FF0805540F0030050
:20DF30001060D5F8B8018169202088470B4CD5F8B8712068B86B804701202060206801E019
:20DF500009F0F4FE09F0E6FDF8BDC04614910100FC120020004003408C2108402C2009404E
:20DF7000F8B5324D6868804706462E4CA9682068002853D1A0698047676A40F01000002F13
:20DF90004BD00022797E0140884205D03A4657F80C7C002FF6D140E004F12400394607F061
:20DFB000BDFA002F39D02760787E30F07F0005D194F82F00401E84F82F0004E094F82E000E
:20DFD000401E84F82E00A9683046884723681889D98A05F04DFFA0851348007807F0D6FF3F
:20DFF0000546D88A000A08D3D87E06F02DF9206890F91C0009F006FC2368687B012803D07B
:20E0100002280DD1052005E0187E401080F0010000F00100F9F7AAFEF8BDA96830468847F3
:20E03000F8BDC046A8100020BF120020001800202DE9F047294E04463078ADF1280D012862
:20E0500049D1DFF8B09009F120000068244F436CF868022108AA98479DF82000002831D1E8
:20E07000DFF8948008F10400006880470024022582461C48059404A90490F8688DF81850DB
:20E09000FFF782F93570029417498DF80C50174B4C8126468DE86000F86802AA0831F7F7E0
:20E0B0001DFD002801D509F073FC114991F90000124E45464F46401C0870A968FE60504693
:20E0D000884708E03078012805D10020012C307001D009F073FA0AB0BDE8F087EB1D0020B0
:20E0F0000C1C002000093D000C150020D53E0100E61D002048190020001800201415002008
:20E1100098B50446E07A002709281CBF0A28E827207B08B1042804DB802801DB862800DB1E
:20E13000E82794F8340018B126483830007850BBA07A8028C8BFE827607B1028A8BFE827FD
:20E150000F2804D01E490988090938BFE827A17B884202DA0F2918BFE827E07B50B194F8CC
:20E1700028000F2818BFE827608D43F6FF71814218BFE82714481D3000884FF6FF71814262
:20E1900008BFEC271AD0CFB904F10C01E820F8F73FFD04F10B01E720F8F73AFD342008F074
:20E1B000DFFA0A4901F144020028106008BF1A2704D0486C3422211D09F024FA384698BD45
:20E1D00094180020C816002079120020483400202DE9FF412E482D4F00683E78C06B8047C6
:20E1F0007968401AB100B0FBF1F4B868FF680025A8464146BC4271EB080101DAB84206D85C
:20E210002946424684428A413CDA074600E0294638463246F317001BA94109F017FA272757
:20E2300004464FF47A7200230D46ADF802700820ADF800002046F8F7D1F901901548016885
:20E2500068468847029843464FF0000100F6FC02A41A9D416042A94111DA0F480268294697
:20E270002046F8F7BBF90D4604464FF000016042A94104DA204606F0F3FD002000E00120D1
:20E29000064908700090BDE8FF81C0466C1D00206819002024180020F81B0020FF350020BF
:20E2B0002DE9F84F2E4C012683461D4690468946C4F87C670320C4F880670AAFC4F884071A
:20E2D000D4F88C0710F0030FFAD1387A58B14FF0805ADAF8B001016A27208847DAF8B00197
:20E2F0000169272088470220C4F8FC063868C4F80804304609F0F3FCD4F808040008F8D23E
:20E31000D4F88C07800F28BF301C26D22868C4F83C056868C4F84005A868C4F84405E86811
:20E330001049C4F848053879002814BF081D081CC4F84C05C4F850850020C4F85405C4F8E7
:20E35000580509490E60C4F800B0C4F80880C1F80064C4F82090C4F82880BDE8F88FC046C1
:20E37000044002402800002000004842314A2DE9F0410446106C002301261F4687420CD059
:20E39000106CC068844208D1106C90F8260009F0B9FA3E46031C18BF176CD56BDDB1D56B49
:20E3B00017E0C868844205D191F8270040F0080081F82700096826E0E868844208D195F80F
:20E3D000260009F09FFA002608B10BB92F4603462D68002DF0D1002E18BF022027D1002B47
:20E3F00014BF002F002022D0106CC0683946844209D1106C884206D1106C2730017841F09C
:20E4100008010170D16B0029CBD1C2F87C4192F8880140F0010082F88801BE8CC2F88041EE
:20E4300003F00103A2F88461012082F88631BDE8F081C046D80D0020F0B50446ADF1140D35
:20E45000FFF75EFE071C50D1637B0F2B30D02C4E96F83B0002282BD1E77B274837BBA438F6
:20E4700090F8C02036F813304FF4707101FA02F562685B009BB2EB18934215D8677B03463B
:20E4900036F8176093F8A1006768760001FA00F0B6B2861BBE4207D3401BA57BA94088425A
:20E4B00028BFC3F8A42003D2FD271EE000210160607C0027C8B194F83400B0B90F480078F9
:20E4D00098B904F112010920FDF760F868B102218DF80C104FF6FF72ADF80420A77A00974A
:20E4F000238901A901F0D2FE03E067702046FDF77DF905B0F0BDC0467C120020001700201E
:20E51000641B0020F0B506460F4600251446ADF1240D8B200DF10E010095FBF7E5FD8A20ED
:20E5300001A9FBF7E1FD707A00282ED1387AA0B9BDF80E104FF6FE70884205DCBDF80E1031
:20E55000884220D101A90DE020489DF80E700488BDF80E008DF812700CE0022807D0032870
:20E5700011D1394604A809F0DBFB09240BE038888DF812008DF81040211200128DF8111080
:20E5900005248DF81300284611E002280CBF05240924012818BF311C04D1892007A9FBF793
:20E5B000A3FD07A9224604A809F02CF8B07A04EB0D01C8736A4604A8214603F05FFC00282F
:20E5D00014BF281C009809B0F0BDC046921200202DE9F041294D012001462870F8F714FA92
:20E5F00027496FF0010008702B480068C06B8047244C074621786068A2688B003E1AB6FB3A
:20E61000F3F05843361A88001F4902FB03F8B1FBF0F0904201D209F0BBF9B91B1B4861605E
:20E630004144FEF755FD1A4CA06867682168404207F090FA002F08BFA16808D0A168786875
:20E650008142DCBF401A78603F68002FF7D1E068884202D0A06005F079FF02F06FFE0D4C73
:20E67000606880470646FFF7B3FDA1683046884708F0D4FD00202870BDE8F081EA1D0020FD
:20E69000DC1D00206C1D0020FFF6C2FFE1E50000C81D002000180020681900202DE9F84FF1
:20E6B00007460E1C14BF4FF000094FF0E809002F4FD0B9F1000F4ED17868401E78603F21EC
:20E6D0000170BD6D002D0CBF802000207968DFF890A00224083E491E7960DFF880B00870C4
:20E6F0003889A7F85440801C388116F8080FFF282CD02A2828D1706830B35546296D884773
:20E71000804678689BF80020A0EB08007860716829B96D6D3A460023A84748B10BE06D6D40
:20E73000786871688DF800206B463A46A84710B9EB20BDE8F88F3889B7F8545040443881FA
:20E7500008EB0500A7F85400641ECED17868386501E04FF0E8094846BDE8F88F58350020A8
:20E77000C8160020F0B52F4C0546A07EADF13C0D022806D0012804D005281CBFE820607638
:20E7900049D194F8600000284AD1002109A81822617609F0E9FACDF828D009A8294600F094
:20E7B000F7FB94F82E0094F85810814220DD266B70B10746BDF80A007189884204D130461C
:20E7D000694607F04BFE98B97F1E06F12406F1D194F82E00276B8100242201EB4011781889
:20E7F000694608F00FFF94F82E00401C84F82E000D48007828B19DF8340010B994F8580078
:20E8100028B909A8FFF7DCFA94F8580040B194F82E10884204D12A202870284605F028F9E6
:20E830000FB0F0BDDC3300206E1200202DE9B841804607F0D1FFC01DC51098F82300002864
:20E8500049D198F87E4007F0C7FFA04243DD264A1368E010191891F86C1004F0070421410F
:20E87000CFB207E0401CC0B21918C40091F86C7088F87E4047B9691E8142F3DC1068002108
:20E8900088F87E10417029E098F97E10C0000830884226DD401A79080BD298F87E10401E88
:20E8B0004FEA670701F1010188F87E10F3D1BDE8B88198F87E000D49087098F87E0088F893
:20E8D000810098F87E00401C88F87E000320F9F74DFABDE8B881002088F87E00072005F0CD
:20E8F00039FFBDE8B881C046A81000200C1C00202DE9F041054608F067FF287E000904D257
:20E91000287D012808BF022700D00527DFF89C80464670688047264C04F124010B68002BE5
:20E9300008BF0D600CD07F1E0026FFB202E07F1E1346FFB253F80C2C22B92FB143F80C5CD9
:20E95000012601E0002FF2D1D8F8081088471EB3616928468847E88AE168C00818D2D8F8E1
:20E970000400804794F82F10491C84F82F10D8F8081088470C4991F8380028B10846C06CB1
:20E9900010B18047BDE8F081FFF7EAFABDE8F08128468847BDE8F081F1206870284603F03C
:20E9B0007DF9BDE8F081C046C816002000180020A8100020F8B5264C236813B908F0E8FF52
:20E9D000236824480068044608F008FFD860204608F0FAFB264C18826068804706461E48A7
:20E9F000A1680278832A30D11C4DEF782FB386210170082008F0E6F9E88C1B4F1949401C71
:20EA1000E88417483A7881621849812A09DB0978842A07DA40F6485292FBF1F101F6B83167
:20EA300006E0097840F6485292FBF1F101F2A321203008F001FCA16807E0852202703046A5
:20EA50008847002002F0C8FDF8BD30468847F8BDA810002060190020003600206C1C0020E2
:20EA70003C1C0020A9450100BF1200206C1D00200018002003B42DE9F0472C4C4FF0000989
:20EA900008AF84F801903968ADF1100D02A80160B988818002A803C89A46164602F00AFC50
:20EAB000A046051C14D04C4686B128466946012207F07CF91AF804009DF80010884205D18B
:20EAD000641C6D1CE4B2ADB2A642EEDCA64227D0B8F80200F61C4FF6FC7440F6F87134400B
:20EAF0002018814203DA08F09BFFFCF7DFFA396802A8BE88016002AD868095E80300224641
:20EB1000534601F087FA98F80100B8F80210002818BF814604D10919083188B2A8F80200B5
:20EB3000484604B0BDE8F04702B07047741E00202DE9B043044609F0D5F981462748021921
:20EB500092F8EE10491ECFB2002F82F8EE703FD1254901EB84014A880C78904634F07F0769
:20EB700018D1E1090FD24FF0805000F5DC75D0F8B8018169104688472868416B404688475B
:20EB90000228F9D11EE000EB8800D0F804110020884717E04FF08055D5F8B801016A1046E2
:20EBB0008847D5F8B801816A40468847D5F8B801016B404688470A490120086009490868CB
:20EBD0008008FCD304F03F003F2801D0FFF7B0FF484609F083F90020BDE8B083F0120020A1
:20EBF00028200860282008401C8E0100F0B52B4D05F12C0158C9ADF11C0D02AA58C20AC959
:20EC10004FF0805682E80A0047688468D6F8D001C16820688847216821488A6B104088637F
:20EC3000206840F2F271416497F83C0097F83D10C0100DEB800080680843216848636846FE
:20EC500009F0ECF8D6F8D001397F466805EB8101BA698B68797F206855F821101943BB7FA6
:20EC700005EB8305AB690B430199B0470D490A1F106840F010001060086840F00100086069
:20EC9000A07D0027FF2802D0E07DFF2800D11FB1086840F44040086007B0F0BDB08E0100D3
:20ECB0000DF8FFFF3010004029482DE9B0410025DFF8A080294C0570ADF1140D88F83B5079
:20ECD000012088F83800201D006888F83D508047234924310F686FB1797E8A0806D341F0E7
:20ECF00001017976397E01F0FD01397657F80C7C002FF1D1A1688847102008F089FE082047
:20ED100008F086FE98F83C00E0B90920124C8DF80000B4F8BA108DF80F50E027ADF80210DE
:20ED300094F8D7308DF8017094F8E6208DF8043094F8E7108DF8052068468DF80610FFF783
:20ED50003FF801E088F83C5005B0BDE8B081C046C9160020641B0020D8110020001800200F
:20ED7000A810002030B50446ADF12C0D08F05EFD002818BFFC2050D168462146112201F0DD
:20ED900021FBA57C617D8DF81250607C8DF81510E37C8DF81100227D8DF81330A57D8DF8D8
:20EDB0001420002105B10121257E8DF8161094F825208DF81850E07D8DF8252094F8243003
:20EDD0008DF81700E58C8DF8243004F119010B220DF11900ADF8265008F014FC607C1A25AC
:20EDF00050B9812007F0BCFC04460A94A4B1FF21812208F0B9FF09E09DF81510880000EBE4
:20EE1000411080B207F0ACFC04460A9424B10720694603F073FE002528460BB030BD10B5C9
:20EE3000401EADF1380D28D0401E09D0801E4FD0401E43D0401E3FD0401E3BD0002048E006
:20EE500001A800F06DFD04460CA942F2090005F0BFFA9DF83000002808BF002203D00220EA
:20EE700007F0B1F9024601209DF83010009001AB204605F01EFE0A3028E001A800F050FDC8
:20EE900004460CA942F2080005F0A2FA9DF83000002808BF002203D0012007F094F9024600
:20EEB00000209DF83010009001AB204605F001FE001D0BE020200CE002200AE042F2130030
:20EED00004A905F085FA04A808F0CEFC80B200E004200EB010BD70472DE9FC4107462A4809
:20EEF0003988C180797B012904BF0121C17005785FB3DFF89880D8F82000012470B1466969
:20EF100066B106208DF80000ADF802400023ADF804309DE803000E223B46B04788F801404B
:20EF3000002D14BF0CA00FA008F0D0FC787B28B9397B0EA00A2205F0C5FB02E00EA008F003
:20EF5000C5FC0020214603F005FC4EF6602006F0E5FEBDE8FC81C046526573746172746556
:20EF70006400C04653746172746564004368616E6E656C3A2000C046467265712E20486F94
:20EF90007070696E6700C04668170020EC150020F8B505460E460520287096F849006968CC
:20EFB000E870F06B4861686806F1280108F070FCB6F842006968488196F8460069684874A6
:20EFD0006868002404761F4869680078C873686806F11C01193008F0A0FE307C696888738D
:20EFF000706810F8011B6A68918110F8013B6A68918941EA0321918107786A68F91117F02E
:20F0100007071174214607EB470218BF012189184018401C10F8011B297201F00702E8605C
:20F03000491001F0380101EB420140187268318968618B18834239BF2C72211C801A091A61
:20F050002974F8BDBE120020F8B50646294F2B4D786C294C90F8300010B194F83800C8B95E
:20F07000717A2846A13880F8A110B17A80F8C010317B80F8971006F124015F20F7F7C8FD99
:20F0900006F126016020F7F7C3FD06F125016120F7F7BEFDF07A207007F088F906F108015B
:20F0B000E820F7F7B5FDF11DE720F7F7B1FD207838B1311D5020F7F7ABFDB11DE120F7F755
:20F0D000A7FD284601210022007861700F2818BF0A1C87F8482007F1490006F10E010B22F2
:20F0F00008F090FA07F1540006F119010B2208F089FAF8BD48340020C8160020791200207F
:20F11000F8B5064608F0EEFE264D0746A91991F8EE00421C002881F8EE203ED1224C04EB90
:20F130008604267806F03F003F2801D0FFF7E8FF648836F07F0018D1F0090FD24FF08050EA
:20F1500000F5DC75D0F8B8014169204688472868416B204688470128F9D11EE005EB84051E
:20F17000D5F804110120884717E04FF08055D5F8B801C16920468847D5F8B801416A204626
:20F190008847D5F8B801C16A20468847074901200860074908688008FCD3384608F09EFEA8
:20F1B0000020F8BDF01200201C8E010028200860282008402DE9F84F294C8A468346211DB4
:20F1D00008880A254FF0FF09002604F13C084746401C088038465946082207F045FC30B1E9
:20F1F0006D1E07F1080706F10106F3D100E0B146B9F1FF0F05D1207A401C2072FF20BDE8FA
:20F21000F88F4846694602F0AFFE0546FF2DF5D09DF80000012806D0A06B05EB85014018D2
:20F2300080F804A004E0606B00EB451080F81FA009490A6808EBC900026049684160074EF3
:20F250007068804794F88C10491E84F88C10B16888472846BDE8F88FE0900100001800202D
:20F27000041400202DE9FF47DFF8888001270446214E88F800703078012803D038460021F7
:20F29000F7F7C2FB204606F0D1F8214D68688047002482468DF80C701849029418484C8376
:20F2B00002238DE81800174B006802AA18318946F6F714FC1449AA680028C8800AD4134BE6
:20F2D00093F90000C1F80C90401C1870504690473C460AE040460470504690473078012848
:20F2F00003D020460146F7F78FFB20460090BDE8FF87C046E01D0020EA1D00200C1500205A
:20F31000181C0020B941010048190020E61D0020001800202DE9F047274D284E234C0020EC
:20F33000383DA13E85F83D0096F8A18094F84000401CC0B2042884F8400031D0202006F047
:20F3500057F896F8E3200F2A18D095F83E0096F8A110814212DD1A4F86F8A10081467868B1
:20F370009046804782461248124950F829008860C86005F0EBF8B9685046884794F84010A8
:20F3900096F8A13035F818504FF4707204F11000491C9A4001FB152107F0CEF9BDE8F087F4
:20F3B00006F0DCFDFFF780FCBDE8F087EC340020F08E0100C81D00209C1B0020791200209A
:20F3D00000180020F0B50C46164607461D4600213822ADF1540D684602F073FBADF8004075
:20F3F00002208DF80800214C8DF80C00E01C007880B168460EA900F0ADFE002833D003215C
:20F410000FA88DF8081003686A461360406850608DF80C10E088A178ADF80A003F29B4BFF6
:20F43000481C0020012F41F08001A07008BF41F0400101248DF80D10012E8DF80E4018BF6D
:20F450008DF80F40ADF828501A9809900BA807F0A3FD07496A4618200FF0BAFEC0B200288D
:20F4700008BF201C00D0002015B0F0BD68170020395D000010F47C1F70B51CD110F00F0F13
:20F490001CD001460024012202EA010091435200401E0BD0401E07D0801E03D0001F07D1F9
:20F4B000093404E0241D02E0E41D00E0641DA4B20029E9D133E010F00F0F01D0002070BD0E
:20F4D000064602244FF4803505EA0600AE436D00B0F5803018D0B0F5803013D0B0F5003015
:20F4F0000ED0B0F5802009D0B0F5002004D0B0F580100FD1072008E0062006E0052004E02E
:20F51000042002E0022000E00120FFF788FC2418A41CA4B2002ED7D1022CD8BF00242046C1
:20F5300070BD704738B51C481A4C20601B4860601B48A0611B48E0611B4820621B4860626B
:20F550001B48A0621B48E0621B48A0601B48E0601B4820611B4800256061606C256308B151
:20F5700007F040FB082384F840306564164884F848502946154BE0630B221D7004F14900ED
:20F5900008F0F2FB04F1540029460B2208F0ECFB38BDC04648340020DD180100B55401001B
:20F5B000A9A3000079440100C5690100EDAC00000D6A0100FDDC0000092F01005D1401006D
:20F5D000CD5F010029780100217A0100C916002090B5044600214022ADF1440D684602F010
:20F5F00070FAA0788DF80000E0788DF801009DF8000000BB616811B101A805F0AFFB217A58
:20F6100001F007028DF82820E0689DF82870C1F302118DF8301027B19DF828100B9000EBE7
:20F6300041009DF8307007B10D90207C8DF8380067690F9719E0616811B101A805F08EFB75
:20F65000677A8DF82970A37A8DF82A30207A8DF82800E27A8DF82B20217B8DF82C10677BED
:20F670008DF82D70E389ADF82E300348006801696846884711B090BDBC1D0020F0B5012979
:20F6900004460546ADF1140D04D0022941D142F2030001E042F20200694604F099FE04B1B8
:20F6B0006D1C07F099F8C01DC010C0B2002830D000230646ADF1010C1F4618461CF801EF01
:20F6D00000224EFA02F101F00101884211D028B97F1CBFB25CB102EBC30103E03CB102EBB7
:20F6F000C301491E05F8011B091205F8011B80F00100521C082AE4DB761E03F10103DDD178
:20F7100030B12CB1D800401E05F8010B001228700FB9002005E004B12770012000EB870086
:20F7300080B205B0F0BD70472DE9F843254C80466068804781466946722006F049FF3225BA
:20F75000FF27002600994046091D07F0C9FD012808D000986D1E06F1010600F11800009090
:20F77000F0D100E03746A16848468847FF2F18BF381C22D1144DD4F804900A2700263C3520
:20F7900012492846082207F06FF930B17F1E05F1080506F10106F3D10DE04046016829605F
:20F7B00040686860C847064A92F88C10491C82F88C10A16888476436F0B2BDE8F883C0468F
:20F7D000041400200018002004140020E09001002DE9B841044608F085FBDFF898800546F5
:20F7F00008F5C4710878A04308F5AA7408702068002808BF002706D020689C3008F0BAFA5D
:20F81000002700B10127606838B19C3008F0B2FA0024384318BF0124274698F8880120BBBB
:20F83000012F22D0D8F87C0110B3C76917B1016A890811D24069D8B10746284608F04EFB81
:20F85000D8F87C0100214FF400030A46B8470020C8F87C01BDE8B881284608F03FFBD8F8EA
:20F870007C0102210022B847F1E7284608F036FBBDE8B881D80D002038B504F041FE03F052
:20F8900009F9204D05F13800007820B11F4808380168012088471E48007810B91D480078EE
:20F8B00008B108F075F81C4C606880471B4AA1681378022B1CD1144CA31C1B78042B1CBF54
:20F8D000832313708847A17831F0010008D0042906D0052907D10020607108F04DFA01E0F3
:20F8F000FBF784FCA178042903D007F0DBFA00E0884795F8380020B1E86C10B1102008F01F
:20F9100087F838BDC81600206C1C002060190020FC350020FE3500200018002000360020F2
:20F9300070B50446E820ADF1280D09A904F036FF9DF82400694607F0D5FA00280CBF0098D9
:20F950001E480DF125016060E82004F027FF9DF8250004A907F0C6FA58B90599C820032251
:20F97000B1FBF0F0401EB0FBF2F15143401AC0B200E00020207206F02FFF0021608165681A
:20F9900021700F4B61700A4608925968A9420CD1197A267AB14208D15989814205D118781E
:20F9B00020705E786670104606E008990C33491C06290891E9D901200AB070BD38C40D00DF
:20F9D000A01900202DE9F047254C01258246984691460E46C4F87C570320C4F8805708AF8D
:20F9F000C4F88407D4F88C0710F0030FFAD1387858B14FF08057D7F8B001016A27208847A4
:20FA1000D7F8B0010169272088470220C4F8FC06C4F80894284608F062F9D4F808040008FD
:20FA3000F8D2D4F88C07800F28BF281C15D2B8F1010F14BF08200C20C4F84C051021C4F812
:20FA500050150020C4F85405064A1560C4F800A0A160C2F800542662A162BDE8F087C0461F
:20FA70000440024000004842B0B50546264CE968E06888423FD1A86803F0A8F9A0B1E9688B
:20FA90004968A06C0978022900D168B9012005F099F8832835D1E068783007F0F3F904F1DB
:20FAB000C80008F013FAB0BD16492869A1F10802136805F110071843106097E80C0051F849
:20FAD000102C181C104341F8100C00270F60A86841F81C0C0F68002FFCD004F13C0007F05D
:20FAF00020FE2564206CC06840680078022808D14FF4004101E04FF4806104F1EC0007F017
:20FB1000E1FDB0BD1C100440D80D002070B52248204D686521484FF080562865D6F8D8019A
:20FB30001F4C036801210A46ADF1400D20469847D6F8D80142680121204690471948F8F73D
:20FB500057FE05F00DFA2E1D304607F08FFC05F11C044FF4E13031462060002005F020FA71
:20FB700011493C22082308600021684608F052F9F0344FF4707000230C4908906A46079476
:20FB90000120069005F15C0008F040F908F03AF910B070BD080200201F7D010031510100B9
:20FBB00000400340308F0100D8060020D91D00002DE9F041DFF8948006460C4636F07F0089
:20FBD00015D1002E3ED1224D243D686880471E49096831F81620144321F81640A9688847AE
:20FBF00041461431086807F07DF8BDE8F081042006F028FF071C25D04FF6FF7038807C8076
:20FC100007F0D0FF41468C78A7F10C05FF2802D0C96A40184478FF2C06D1384607F08DFE98
:20FC300007F0E4F9BDE8F081304607F013FB01463A46FF20A872204605F088FE10B138462F
:20FC500007F07BFEBDE8F0810C300020DC1B00202418002025483EB50078002843D042F2F8
:20FC70000100694604F0B4FB42F2050002A904F0AFFB1D4D95F8540010B39DF808000024D0
:20FC90009DF80810009B2864642285F85440581A02FB00F1E96705F1780003F0C3FF01A86D
:20FCB00005F07AFA124801992E300078B1FBF0F2451E4243891A01918D4214D9204610E044
:20FCD0009DF8081064204843E86705F1780003F0A9FF288F401C288700242C64012085F8EC
:20FCF000540004F037FD3EBDA0310020951200205C3200202DE9F041224C064604F15800C9
:20FD100005780F46002D04BF0020011C1CD0204D1D49281D0B780068D3B91C480568E06C3C
:20FD300007F0DEFD228FB0FBF5F1B0FBF5F3891889B203FB05F2236C3980801AC0183060F1
:20FD500085421CD8401B491C30603980BDE8F08180475FFA80F804F1780007F091FE226CA0
:20FD70004FF47A73410001EBC001B1FBF3F0238F3060A9683B808018306040468847BDE896
:20FD9000F081C046A0310020951200206432002000180020F8B50F46002302B90123DFF85B
:20FDB00090C00021EFB13D6ADDB1C669CEB1FC68C768A74207D0DCF854110CF5AA77A142AE
:20FDD00014BFF968B968B4086FF05047A4EB9504641AA74225DDB4F1704F01DB002C20DD12
:20FDF00001210AB3D769FFB1066AEEB1D268C068824208D0DCF854310CF5AA70934214BFFB
:20FE1000C068806800E00020C0EB97006FF05042A0EB9600824204DDB0F1704F03DB002863
:20FE300001DC0020F8BD012301EA0300F8BDC046D80D002030B50546ADF1240D294607A811
:20FE500007F0EDFE214CE08BADF81800284606F075F94FF6FF71ADF81A0081421AD1022005
:20FE700023788DF81600581CADF81A00E06838B142682AB105F1080106A890478DF8160034
:20FE90009DF8160048B905F1080106A8002202F09DFE02E000208DF81600684600210B22B1
:20FEB00001F00FFE0DF10B0007A907F0B8FEBDF81A006A460649ADF8140018200FF088F98F
:20FED000E16D09B12846884709B030BDDC0A0020117C0100F0B520480127F84201D004F05F
:20FEF00081FB204D204F214EBD4206D203CD0478A4003459401CA047F6E71D48002800D05A
:20FF10008047164D164FBD4202D210CDA047FAE7F0BD03251BE0416808300A1C2A400BD1AD
:20FF30001A1C2A40AB4305D0046804300C600431043BF9D1131C05D0047801300C700131A5
:20FF5000013BF9D1021C2A4001D0A84304300368002BE0D17047C046FFFFFFFF0000000013
:20FF700000000000C00E0000200F00007C0E000055C5011070B504466068254E4078ADF1BF
:20FF9000480DC00921D3B4F842003546E63DB5F8BA10884219D11D480078A0B995F8C40001
:20FFB00098B104F1280006F09FFB70B9012000901C340194B5F8BA3005F1AA0203210620F9
:20FFD000F7F726F91FE007F0F1F80BA80021182201F077FD02A821460C900BA8FEF7D8FF86
:10FFF0002C208DF82C000BA803F042FD3546503D17
:020000040001F9
:20000000287810B19DF83C0028B105208DF82C000BA8FDF7DDFE12B070BDC046C81600208A
:20002000BE12002003B426482DE9F041058806AF1446ADF1080D98464FF6FF70ADF80000DE
:200040000222ADF802006946ADF8040044F40040ADF80600601986B2304602F03BFABDF857
:200060000600022269466FF3DF30ADF80600304602F030FAA1102846CAB2414602F02AFAC1
:20008000387840F40040ADF800007888ADF80200B88802226946ADF80400304602F01AFAB8
:2000A000BDF80000022269466FF3DF30ADF80000304602F00FFA02B0BDE8F04102B0704740
:2000C000761E00202DE9F843002A894607464CBF47F6FF75151C002F08BF002033D038880F
:2000E000002808BF002403D02A4600F0BBFC0446281B002826DD388828B1291B484613A22B
:2001000004F012FE0419B868E0B1D7F804802E1BB8F1000F0DD0404607F0AEFB401DB04267
:2001200007DC291B48460AA2434604F0FDFD04192E1B122E06DBBB68291B484606A204F0CF
:20014000F3FD04192046BDE8F883C0463A2000C0222573222C2000C06C696E652025643A79
:20016000200070472DE9F047244C0746203C206A8A46ADF1280D00283CD0BAF1000F39D01E
:2001800004F0CCFA5FEA000834D0062000250523A1468DF808002E46ADF80A30642D29DA82
:2001A000D9F82000ADF80C5004AB02AA0469009392E8030018230022A047B8B9387A0228E4
:2001C00004D1BDF812103A88914207D003280CD105A93846082206F04FFC30B904A950463C
:2001E000182200F0F7F8012005E0761CB04505F10105D3DC00200AB0BDE8F0870C16002076
:200200002DE9F043244C0746206AADF1240D00283DD0002F3BD0387A002838D004F07AFBC5
:200220005FEA000833D0062000250323A1468DF808002E46ADF80A30642D28DAD9F82000AE
:20024000ADF80C5004AB02AA0469009392E803000A230022A047B0B9387A9DF818108142F4
:2002600010D1022804D1BDF810103A88914207D0032807D104A93846082206F0FDFB08B956
:20028000284606E0761CB04505F10105D4DC4FF0FF3009B0BDE8F083EC150020BCB50446BC
:2002A0000920207560680D461112401E00F8011906AF00F8012939781D4A00F80119B2F827
:2002C000BE10091200F8011992F8BE1000F80119191200F8011900F80139411C2162217DCC
:2002E000491E017061682289091AC9B289186060287A2181032814BF002001200D490B22AD
:200300004931E08204F1800007F084F90020032120654FF6FF73A0652A4600902046F3F743
:2003200013FB071C02D12046FEF7EAFA3846BCBDD811002048340020F8B5234D0120014659
:200340002870F6F769FB6FF00100204C1D4927690870381C28D0A1684268914203DA07F0D4
:200360001FFB27693846C8B105F036FA7968884224BF2769381C11D200F0E8FF14E0266908
:200380007068002802D507F00BFB2669304603F08BFFB168307B88472769384620B105F0A0
:2003A0001BFA79688842EAD2094C606880470646FDF716FFA1683046884706F037FF0020EE
:2003C0002870F8BDDD1D0020EA1D0020C81D002000180020002A4AD05FEA000C8B071CD13A
:2003E000830722D1102A08D370B4103A78C978C0103AFBD270BC103238D0042A2CD3082A98
:2004000005D30C2A24BF08C908C008C908C008C908C092072AD0920F22E00B780370491C8F
:20042000401C521E22D08B07F7D1C30714D18307D8D0121F12D308C903801B0C4380001D52
:20044000121FF8D20AE008C903701B0A43701B0A83701B0AC370001D121FF4D2121D05D013
:200460000B780370491C401C521EF9D160467047F8B507F03FFD234C0746D4F8C00010F402
:20048000602F33D0D4F8C000400CC6B2700807D2B00803D2F00828BF022602E0012600E0AC
:2004A0000026751D002168B203F084F9D4F8C03006F111010120884023EA00013846C4F8E3
:2004C000C01007F013FDB00004F1A8010A18D7682FB1085800224FF000632946B8470A48D2
:2004E000006830B9022004F075FB02E0384607F0FDFCD4F8C00020B104F59070002107F067
:20050000E9F8F8BDD80D00200C1004401CB51F4C04F1780006F028F804F15C0006F024F8BE
:2005200004F1940006F020F80021882204F1340007F022FC07F014F906F056F984F85A00FC
:20054000134984F85B001348086001200DF1010184F8B30042F2040003F042FF42F20500B0
:20056000694603F03DFF0C489DF80110A0666420414321660949C4F884109DF8001048433C
:20058000E0670748C4F8A0001CBDC046A0310020581900205D5D01004943010065FC00005F
:2005A000CB7C0100D0B5244C04F124010F68002F3FD0002215280AD13B7D0126022B08D011
:2005C000032B06D0052B04D0042B02D000E03B7D0026984200D016B17B7E5B0905D23A462F
:2005E00057F80C7C002FE5D123E00846394604F09DFFF88A2760000A03D397F91C0007F053
:2006000009F9387D022818BF052802D1012006F0E1FB2068407E30F07F0005D194F82F00B9
:20062000401E84F82F0004E094F82E00401E84F82E003846D0BDC046A81000202DE9F843D1
:20064000234D884606464FF0FF3105F12400814607F030FC00200CE0FF2909D02A688A4232
:2006600004D905EB8101D1F894700FB1002627E0401CB8F1000F03D018F82010FE29EBD167
:200680000024346074600127B46011E0FF280ED005EB80000B787268C0F8946007FA03F02F
:2006A000104370600A680949304605F0BFF9641CB8F1000F04D008EB84010878FE28E5D150
:2006C000484607F00FFC3046BDE8F883007FC767FC2E0020B0B5456884682349607DA27D97
:2006E000ADF1180D40F000400090207D0027FF2A41EA000001904FF0020002D0E27DFF2AF3
:2007000000D13FB1E37DA07D1943039140F0004002900420FE214DF8201005F158006946F4
:20072000FFF78CFF6866002808BF381C1AD0617D0F2205F0A9FD686E217D102205F0A4FD57
:20074000A17D3846FF2902D0E27DFF2A00D140B1686E112205F098FD686EE17D122205F0C9
:2007600093FD012006B0B0BD0000C0A02DE9FE4F0290DFF88880007A022838D1029805F035
:20078000E5FC81464FF6FF70484530D01C4D444632264FF0060B4FF0050A3434203D2F6A29
:2007A00034F80C0F814520D12046FF210C2201F090F9D7B1FF68C7B1029801F051F8B0F131
:2007C000FF3F12D08DF800B02F6AADF802A0FA68ADF804009DE80300904730B903F09EFF01
:2007E00018B1401E80B205F0F1F9761ED7D14446216809B102988847BDE8FE8F400B0020B2
:200800000C1600203EB506F015FE0446204D2149286981422FD1204905F17000002207F03D
:200820008AFA0120287006F067FC00204FF6FF71B5F8C4306871994209D10220ADF8000057
:20084000684605F0F5FEBDF80800A5F8C400286C60B905F13C0007F081FA031C06D003F0AB
:20086000EDFF40B91846FFF707F904E005F1EC00022106F02FFF04F0804104F0020008433C
:2008800005D005F1EC004FF0005106F023FF3EBDD80D00201535000039C400002DE9F84361
:2008A000DFF88880054608F104000068804781461F48243004680027A7422CD0607E30F0EA
:2008C0007F0024D062686B68501D591D52785B78C2F38102C3F38103934218D1022A05D057
:2008E000032A14D106F004FD064609E00A78037800269A4204D149784078814208BF0126BC
:20090000301C04D0607E274600F0BF00607654F80C4C002CD2D11FB1787E40F04000787650
:200920004046816848468847BDE8F88300180020A810002098B5244C0746A8B1401E0BD01F
:20094000401E2CD1204690F8402042F0080202F0EF0280F8402022E094F84020204602F0B1
:20096000E70242F01002F4E7214601F17402107891F83C3000F0F000107003F0F0000022BE
:2009800081F83C0091F840308A6343F0080000F0EF0081F84000F420413103F007FF002F3B
:2009A00008BF44F620600CD007F050F94FF4FA670A2244F6206390FBF2F15143401A07FBAF
:2009C0000030A06498BDC0460C1500202DE9F8432020EFF3118780F31188214CA068012199
:2009E00007F014FA4FF001094FF0000865692168A4F81C906A1A2168A4F81E80461B401AC1
:200A0000904227D387F3118840464519361A4846294607F0F7F9B042F7D92021EFF3118762
:200A200081F31188E18B012903D14046294607F0E9F9B0F1FF3F06D0A169801B814238BF5D
:200A4000081C411901E0A069291807F0D7F9A4F820902560A4F81C8087F31188BDE8F883EA
:200A6000780100207FB503461F480D4601881F480088144614A6984205DB32462146284613
:200A800004F052F91DE0994206DB184606F022FA0028F2D04268F1E715480088002808BFAE
:200AA0000CA2EBD00095002C48BF47F6FF74114E0020114901946A46346802901846A047C4
:200AC000029800907FBDC0467B6D6F64756C652325647D007B6D6F64756C652D726F70659C
:200AE0003A25787D00C046C07E900100309101008E140000289101001D61010070B5194DA5
:200B0000194E482205F1500406F15C002146FFF761FC164828651648E8661648A86516484D
:200B2000C5F88400154828661548443CFF21A8661448F4604FF41672686606F1A40000F0AA
:200B4000C8FF5220012106F009FC318C532006F011FC0D4C0D49142204F1940003F092FE1B
:200B6000A06170BD68170020DC0A002045FE00009D6A01006D0701004D710100BD1B01004A
:200B8000BD21010065240100EC1500209D720100B0B5234C0A46ADF1280D0892276A002F6A
:200BA0003CD07969002939D0B0B9606A11461930884233D806208DF80000ADF802000025F6
:200BC000ADF804507D699DE80300042208ABA84708B90898606221E06946FFF7C3FAE8B1C7
:200BE000059908981931884218D30590206AA8B101A800F035FEB0F1FF3F0FD00621052763
:200C0000256A8DF8181006ABADF81A706C69ADF81C0093E8030018226B46A0470AB0B0BDAB
:200C2000EC15002090B50C46214A0178575CADF11C0D0B2F8DF8007035D0002F36D00C2FFA
:200C400004D0112F29D106F080FE26E01A2C22D090F899100190C7688DF80210038A029726
:200C6000C28AADF80C30510905D21249827EC8310978891A00E000218DF80E10877F8DF86F
:200C8000107090F91F308DF81130826A0592417F8DF80F1001E0002001908DF80140684649
:200CA000FDF796F802E04470FCF7E8FE07B090BDFC880100D81100202DE9F041074678683D
:200CC000BE68044600F5847006F0E4F830681C4980690968C0F3C00008BB07F00BF9194DFB
:200CE0008046287820B1022004F0BAFE00202870404607F0FBF83168134D886B20F02000AB
:200D00008863286820F480702860606A216A091A21622369626A38469847BDE8F0814FF4C3
:200D2000FA70B0FBF1F1012998BF012104F58474204607F097F8204607F0D0F8BDE8F08101
:200D400014910100F5350020301000402DE9F04180461E4800680D46416927208847012410
:200D600004FA05F61A4DC5F80064C5F87C470327C5F8807717480460C5F88477D5F8040444
:200D8000012818BFC5F80444C5F8FC6312480460C5F800801023AB60204606F0A8FFD5F829
:200DA0008C074008F8D3D5F88C17204611F0404F09D1C5F884770021C5F8FC16D5F80024B4
:200DC000164218BF081CBDE8F081C046B00100100440024000E04842000048422248F8B552
:200DE0000C460178012904D0417A012918BF012034D190F8C710CA080AD390F8C620A242E8
:200E000006D101F0FB0180F8C710002780F8C67007F070F8074607F055F806460121204626
:200E200002F0C8FC0E48210201F47F41084305F0FFFB0C4A1168054604F10C03012098407D
:200E400081433046116007F039F8384607F04EF805F0FF05012D0CBF81200220F8BDC04694
:200E60000100080408100440D80D00207CB515460E46044600E004192046694604F0DAFEFC
:200E800000282ED014F8021F8E42F4D1491E04F1010420D0491E12D0491E08D0491E18BF53
:200EA000622029D102281CD12078287023E0032817D114F8010B2870207868701BE007280F
:200EC0000FD161782078A41C40EA0120288020682E1D30600FE0052803D12078062828705D
:200EE00001DD67207CBD2D1D0020641C2860A678AE702088288000207CBD70472DE9F041FF
:200F00001E4615460F46044606F0DCFF8046384605F012FA071C04D097F8270030F07F0011
:200F200003D1404606F0CAFF28E097F8270010F00F0F1BD113487968884202D07968A16610
:200F4000786004F1600080E86000404606F0B6FF04F140004FF0FF3106F0ACFF04F17007BA
:200F60000020A06697E80300BDE8F081404606F0A5FF97F8270010F00F0FFAD102200021B1
:200F8000BDE8F081AD2C010070B506467468B568606E05F0BEFF29681C488A6B1040886352
:200FA000304600F037F8304601F0ACFC2968C86A20F01000C862296815480A6B1040086362
:200FC0006868FDF7BDFD04F1800006F033FF04F19C0006F033FFA07818B904F1D00006F099
:200FE00035FF607818B904F1EC0006F02FFF04F5847006F027FF06F07DFF0021217006F0EC
:2010000075FF04F16C0005F0A5FE70BD0DF8FFFFFEFCFFFF2DE9F04106467568B46806F0B9
:2010200069FFA96A39B921688969090903D206F05DFFBDE8F0810027AF6206F057FFA17DD7
:201040003846FF2902D0E17DFF2900D118B12846214600F0DFFE2168886B20F020008863BF
:201060000D49086820F48070086006F043FF0B4C8046207818B1022004F0F2FC2770404667
:2010800006F034FF686A296A091A29622B696A6A30469847BDE8F08130100040F535002077
:2010A00038B50C4644220546002100F012FD04F12801284606F012FA04F1320105F10A006A
:2010C00006F00CFAE06B6861B4F840002883B4F842006883B4F84400A88394F84600A87784
:2010E00094F84700E87794F9480085F8200094F8490085F82100B4F850006884E06C6862DB
:20110000A07B85F8280094F8520085F82900606D0B2204F11C01E86205F13000FFF75AF9C6
:201120002089A5F840006068E86338BD70B51E4DAC68064606F05AF94FF47A71001B484314
:20114000030C05F061FA2969401A48BF404240F6B8319B19994210D306280EDAE9688C42F5
:201160000BD8286848B1114A091B51438A0C02EB1141884288BF011C08E00D4948684008B7
:201180000ED208687D2100F0FF004143C82905D3B1F57A6F88BF4FF47A6103E0C82101E084
:2011A0004FF4FA61084670BDB835002040420F00AC3F00502DE9F8431F4C00264FF0010813
:2011C0004FF002093746A51E15F8020F03280FD0022824D168786368022820D0304606F00D
:2011E0002BFD0146384606F0C1FC85F8019011E0304606F021FD014663686878012805D0D6
:20120000384606F0B3FC85F8018003E0404606F0ADFC6F700246C9B2184604F06DFA761CB8
:20122000022ED1DB05F040FA18B104F1200006F097FDBDE8F883C046201B00207CB5042065
:2012400004F0F6FF022818D0032816D019480068C0F38150032814BF41F288324FF47A721B
:201260001649174C09684C342046B2FBF1F106F0F9FD204606F032FE7CBD4FF08056D6F832
:20128000A4010D4D446800214FF040521C23032000902846A047D6F8A40100214FF4007221
:2012A00009230126446800962846A047022004F0D7FB7CBDB43F005000A00C40149101004E
:2012C000F812002003B42048F0B505AF3E787D880088BF88ADF10C0D001F84B2082C2CDB9B
:2012E000201F6946082280B204F068FDBDF8000086420FD1BDF8020085420BD1BDF80400DB
:20130000874207D1BDF806006FF3DF30241A241FA0B213E0BDF80600C10BCB0309D100F11A
:2013200008018C4202DA06F03BFB06E0241A083C00E0241FA4B2082CD2DA002003B0BDE895
:20134000F04002B07047C046761E0020F8B51E4C002528462268A168256190420CD052680F
:20136000914209DD04F038FA0146206842689142C8BF41602061A168676837B118B1426866
:201380007B689A4201DD38462061C8B14068814216DD0F4D044605F108000068A04201D813
:2013A00006F0FEFA094E706880470746EC60204600F056FEFCF714FFB16838468847F8BDE5
:2013C00005F036FB2561F8BDC81D0020001800206C1D00202DE9F8431C481F4D0778686856
:2013E000804781461A4883680026344680469C4212D013F8020C874208D134B163B13846BA
:201400004FF40041FEF7DCFB13E01C4604B91E4653F80C3C002BECD15FB9686880470D4986
:20142000096831F817206FF3DF3221F81720A96888472CB108F108002146324604F076F819
:20144000A968484688472046BDE8F88388180020DC1B00200C300020001800202DE9F843DC
:20146000DFF87480054644466068804781461B48476AE726EFB100220446787E30F07F00B4
:2014800007D0387D012804D1287997F89910884205D03A4657F80C7C002FEED109E004F127
:2014A0002400394604F042F894F82E00401E84F82E00D8F80810484688473FB13846FFF7F0
:2014C000EDF93846F021FFF7ADFB002628463146FFF7A8FBBDE8F88300180020A810002025
:2014E0000829C8B50BDA00293BD00278491E92FAA2F24FEA226200F8012BF6D1C8BD46426F
:2015000006F00306891B37188AB2361802F00301864209D9361A0378761E93FAA3F34FEAF4
:20152000236300F8013BF6D122F00302D71987420AD93A1AD21C96100268761E92FAA2F271
:2015400012BA40F8042BF7D1CF19874209D93F1A01787F1E91FAA1F14FEA216100F8011BA2
:20156000F6D1C8BD2DE9B84106F0C4FC1C4C1B4D804604F1E000007848B92C46A1680220D9
:2015800088470746102003F0ADFB0FB31DE001F0F3FB70B9134800683221B1FBF0F101B940
:2015A00001213034204606F05DFC204606F096FC0EE0002084F8E0002C46A168022088472C
:2015C0000746102003F08EFB17B1A16803208847404606F08BFCBDE8B881C0469090010047
:2015E000F012002014910100F8B5074600261A481C4C067019481A4D067095F83800E0B12F
:20160000E86FD0B12168087D35280AD148680989FFF766FF206840680088000901D303F087
:2016200067FFE96F384688470F48007801280BD030460146F5F7F0F906E002F069FF01F009
:2016400031FA3846F7F700FD206810B1007D352801D005F0A3FFF8BDF83500200036002013
:20166000C8160020A8100020EA1D00201D491E482DE9F041352751F8048B51F804EB51F8A5
:2016800004CB51F8046B51F8045B40F8048B51F8044B40F804EB51F8043B40F804CB51F8BD
:2016A000042B40F8046B40F8045B40F8044B40F8043B7F1E40F8042BDDD151F8045B51F81C
:2016C000044B40F8045B51F8043B40F8044B51F8042B40F8043B40F8042B09680160BDE848
:2016E000F081C046EC02000000C0002170B51B4C05461022ADF1200D04F19D016846FEF79A
:2017000069FE0026049509208DF8146004F12D018DF8160001258DF815500A680DF117002C
:2017200002604A684260097A01720D496A4618200DF056FD0B4918208922631D0DF050FD6E
:201740007120314606F024F9D520214606F020F95D20294605F002FE08B070BD288C010088
:2017600079AF0000D97900002DE9F04F1C4C8246206A8846ADF12C0D70B3B8F1000F2BD065
:2017800002F0CCFF071C27D0062000250523A1468DF808002E46ADF80A30642D1CDAD9F8E0
:2017A0002000ADF80C500DF1100B02AB0469CDF800B093E8030000221823A04740B9B245AE
:2017C00005D1404659461822FEF704FE04E0761CB74205F10105E0DC0BB0BDE8F08FC046D1
:2017E000EC1500202DE9F0431C4E044600271D468846A2EB0409ADF1140DC6F8B07101201A
:2018000006F075FA3068C00FF9D3306A0090706A0190B06A0290F06A039044B12846234636
:20182000694611F8012B5B1E00F8012BF9D10320C6F838026CB108EB09016D1E491E11F82D
:20184000010F15F8012F904218BF042002D1641EF5D1384605B0BDE8F083C046504502402B
:201860002DE9F0431C4C8046203C206AADF12C0D68B3B8F1000F2AD002F050FF071C26D00D
:20188000062000250523A1468DF808002E46ADF80A30642D1BDAD9F82000ADF80C5004ABE7
:2018A00002AA0469009392E8030018230022A04748B905A94046082205F0DEF8002808BFA2
:2018C000281C06D0761CB74205F10105E1DC4FF0FF300BB0BDE8F0830C16002090B5044698
:2018E0006078ADF1140DF3282FD0DF282DD0E8282BD0DB2829D02046FCF70AFC071C23D1B6
:20190000607C08B394F83400F0B912480078D8B904F112010920F9F741FEA8B102218DF803
:201920000C104FF6FF72ADF80420A77A0097238901A9FEF7B3FC0746F32F05D0DF2F03D035
:20194000E82F18BFDB2F03D16770204603F0B2FD05B090BD001700201849B0B50546164C30
:201960000F7820781FBB164A8100B2FBF1F1A94202D206F015F820786168154F800005FBF7
:201980000014A7F10C000068C06B8047211AA1F54871090806D30B4A011B891A090828BFB5
:2019A00000F5487408482146FBF79AFBB0BD074901200870B0BDC0466C1D0020EB1D00209E
:2019C000FFF6C2FF00093D00E1E50000FF35002074190020F8B51A4E1A4D0120002414EA85
:2019E000030730704FF0020000EA020008BF00280CD14FF0E04004EA0201184008BF0029AC
:201A000004D11249888D401C888503E095F90000401E287005F0FCFB05F0C0FD0A4804704D
:201A200095F9000030B195F90000002806DC05F0B7FF03E020460146F4F7EEFF3470F8BD33
:201A4000EA1D0020E61D0020DF1D00206C1C0020F8B500680E4617464FF0FF310446483081
:201A600006F028FA4FF0FF35092E08D0217A0120B040084211D108433546207210E0227A10
:201A80000721012303FA01F0104202D0491EF9D503E0227A0D4610432072B5F1FF3F0ED03A
:201AA0006FB129463846FFF751F940B1217A0120A8404FF0FF3580F0FF000840207204F193
:201AC000480006F00FFA2846F8BD002213460A46194671B510F0030F0BD0002A82BF00F8FC
:201AE000011BB2F1010210F0030FF6D1002A08BF71BD11F0FF0141EA0121042A18D341EA9A
:201B00000141082A0FD30E46102A08D30C460D46B2F10F0312F00F0272C0103BFCD812F046
:201B2000080F18BF42C012F0040F18BF40F8041B12F0020F18BF20F8021B12F0010F18BF6A
:201B4000017071BDF8B5054606F0D4F91A4C0126074605F19C00E67005F09CF9207801281E
:201B600011D094F8880170B1B4F95000B4F95210884208D1384606F0B9F90720FDF730FE30
:201B800006F0B8F90746B4F95200B4F95010884218BF85F8C2600AD105F1780005F07AF954
:201BA000304603F017F8E17920780843E071384606F09CF9F8BDC046D80D00202DE9F0410F
:201BC0000646DFF86C80307848BB4546AF68341D57B1B27CB87C824203D16089F989884221
:201BE0001DD03F68002FF5D1282004F0D1FCB0B1AF68B4E80C10011DA1E80C10B4E80C10A8
:201C0000A1E80C101CCC81E81C000024046017B9A86004E00F4639680029FBD13860454660
:201C20006C35296809B130468847BDE8F081C046DC0A002038B51B4D95F8A1000F2824D0A3
:201C4000194C3B3C94F83810FF291ED094F83A0068B102290BD103F0BFFD216B0F4C95F8B5
:201C60009820401A2178083101FB12010BE003F0B3FD616B0A4B95F8C020081A1988401A38
:201C800034F81210411A002901D5002038BD4FF6FF708842C8BF88B238BDC0460D1C002004
:201CA000D4100020D81100209F1B002080B501460A7D012A05D0152A03D0252A18BF352AA3
:201CC00002D1087E000920D313480768087EC30916D2012A18BF152A01D1000909D24F78ED
:201CE0001B2F04D00D4807B10E30805C02E0232000E0312008700A48007801F0E7FB80BDF7
:201D000047B148783946884780BD4A7808461146FEF788FF80BDC046AC100020F38C0100FE
:201D2000881800201C4938B591F85C3001EBE304657F012203F0070302FA03F383F0FF033E
:201D40002B4063778B7E01F11800032B18D091F86030012B10D0022B08D0B1F856108A4012
:201D60009102A1EB821101F570710EE0B1F856209101A1EB820108E0B1F856108A4001E08A
:201D800004490A789102A1EB82111C3005F05CFA38BDC046A1120020DC33002010B504461F
:201DA00000213422ADF1380D6846FFF792FE002000908DF80C008DF80D008DF816008DF8A2
:201DC000250013490A90CA8BADF804208DF83040097F8DF8061009218DF8071001228DF844
:201DE00008200F218DF809108DF80A1018208DF8241043F6FF71ADF8261004498DF80B20DC
:201E00006A460DF0EDF90EB010BDC046697C0100DC0A002038B50C4621680546886B20F09C
:201E200020008863686E217D012202F0E3FC686E217D012203F060FC686E217D002204F0BF
:201E400023FA686EA17D002204F01EFAA878012806D005F1D0004FF0FF3106F02BF803E0F3
:201E6000216888690009FCD2686E217D102204F00BFAA17D0020FF2902D0E27DFF2A00D1E1
:201E800018B1686E112204F0FFF938BD2DE9F84F834689467120114604F0A2FB1746812023
:201EA0006946F8F729F94FF0F308002507E0B8F1000F23D038686D1CEDB22C3038609DF820
:201EC0000000A8421ADD3868066890F804A0002402E0641C0A36E4B2A245E8DD737A002BC7
:201EE0000CBF052009208145F3D14A463046594604F090FF0128ECD14FF000084046BDE8BF
:201F0000F88FFEE71A487CB5007880B342F2050001A902F065FA42F20100694602F060FAB3
:201F2000144C9DF80400216C88420BD80098884203D805F007FF01250DE00022012584F85F
:201F4000542004E001259DF8040084F85450401A64214143E16704F1340606F1440004F041
:201F600003FB06F1440001F065FE84F858507CBD95120020A0310020F8B50B461A4991F8D5
:201F800031708D6B4C7A6430C2B25FB100206D1F6D1DEE7816B12E79B24207D07F1E00F167
:201FA0000100F5D1641CE0B2487204E0FF281CBF0021197016D10120187091F830704C6B8E
:201FC0004B7A5FB10020203C2034A67F16B1E57FAA4207D07F1E00F10100F5D15B1CD8B2F3
:201FE0004872FF20F8BDC0460414002038B5054601201A4C68712879B0B90DF0C4FC21781D
:20200000002904BF6FF00704051C15D0491EC9B2217039B90DF0E1FC606804F0AEF80020A3
:20202000687118E0054613E00DF0ADFC05462078FF2805D16FF0060428460DF0CEFC0BE082
:20204000401CC0B20128207002D1606804F0ACF828460DF0C2FC0024204638BD001E0020E0
:20206000154998B50F7817BB144A1178144F52688B00890000FB0324B7FBF1F1814201D2F8
:2020800005F08EFC11480068C06B8047211AA1F54871090806D30B4A011B891A090828BF8E
:2020A00000F548740A482146FBF71AF898BD06490120087098BDC046EB1D00206C1D002049
:2020C000FFF6C2FF00093D00FF350020681900203903010038B517481749007818B908468F
:2020E000007828B906E00846007830F07F0001D005F056FC114D68688047114C0C3C2178F1
:20210000A278914207D10F4AA9681278D20803D28847012038BDA968884705F003FEA07884
:20212000FDF7A8F8012804BFA078207005F036FA38BDC04600170020003600200018002092
:20214000181C0020FD3500202DE9F84380461848077817B9174D287810B90120BDE8F88305
:20216000154E70688047814668880124B8F1000F0ED1214603464FF6FF72B9404A401040B1
:2021800068807BB170B9002004F016FA044609E018B9204604F010FA68882146B9400843DB
:2021A00080B26880B168484688472046BDE8F88388180020701E002000180020F8B505466B
:2021C0001A4C2878002818BFEA2823D1687801281ED010BBAB69DFF850C00021FF224FF0B6
:2021E000010E0846C6101CF8066000F007070EFA07F7374204D01E5CB242C4BF011C5A5C1D
:20220000401C8128EEDB04F11C000170032002E0022000E0012005F039FA7434216809B133
:2022200028468847F8BDC0466E8C0100DC0A00202DE9F8438146EFF31188202080F31188C6
:20224000174D154C134F012605F11C000660A4F114000660F86A016A14208847D9F81000F8
:20226000810C14BF000C04202060386802682321002090470948066054F8180C20F4C020EE
:2022800040F4803044F8180C2E6088F31188BDE8F883C04684010010182009408002244333
:2022A0000000244330B504460D4642F20900ADF12C0D09A902F094F89DF8240008B342F249
:2022C0000B000DF10E0102F08BF800230094BDF80E00029300040190684602F069FD04467D
:2022E00004A942F2030002F07BF804F07DFA024604A9B4FBF5F06843241AE0B202F0A0F99B
:2023000006E042F20D0003A902F06AF89DF80C000BB030BD2DE9F843194D064628780C4658
:202320009846012805D0687A012818BF6FF0010024D162600A20208001F0FAFB071C1CD405
:20234000A77005F0D7FD8146204604F071F90446484605F0CBFD04F0FF04012C06D0384605
:20236000012101F027FA6FF0010706E005EB8705A83545F8088C45F8146C3846BDE8F88357
:20238000D80D002038B50546FEF788FA164C04F11800006880471349012812BFB1F8C2002A
:2023A000B1F8C200401C6882254695F82E0060B991F8A1000F2808D10C4C204601F074FFD1
:2023C0004FF47071204604F03FFF094C243C6068804795F82E10491C85F82E10A16888473A
:2023E00038BDC046D8110020A81000207C340020241800202DE9F04107461748174CC01FA0
:2024000006786068804780461549A268087886281CD1104D05F12A021088401C10808720BC
:20242000087005F0BBFBA16840468847082004F0DBFAE879B04207D127B90020FFF7D4F83D
:20244000BDE8F0811B20F9E7E920F7E740469047BDE8F0816C1C0020643500200018002058
:202460000036002030B5044603202146ADF13C0D8DF838000A680CA80260496841600CA81B
:202480006946FDF76FFED0B10DF1230001A905F0CEFB00210B2206A8FFF71BFBBDF8020063
:2024A000012506AA8DF82E500849ADF82C0018200CF096FE03A968462A4600F08FFB0448C9
:2024C000016809B1204688470FB030BD1B7C01004C0B00202DE9FC4716460C46054604F0A3
:2024E00079FB164F814678688047804603F006FB8246B2002146484605F080FB504604F072
:2025000033FE02E02D1D241DADB23046411ECEB278B128466946042203F050FC68462146A9
:20252000042204F0A9FA0028ECD00549012048700870B96840468847BDE8FC870018002085
:20254000741E00202DE9F8430024002B16460F468046254606D5002FC3F1000302D57F42EE
:20256000761E2D2599463846494602F0A1FD0CA0405CB7FBF9F7002F04F1010408F8010DD8
:20258000F1D1A64205DD3021301B401E08F8011DFBD10DB108F8015D4046BDE8F883C04603
:2025A000303132333435363738396162636465660000704730B5401E4FF00004ADF12C0DA5
:2025C0000AD0401E04D0401E20D1F6F70BFE1DE000F026F8044619E001A8214624220823DB
:2025E00005F048FC06940D4DADF8144009490794012201AB05F1780005F038FC064A2346A9
:202600002C2105F19C00009305F044FC20460BB030BDC04645360100414D0000F0120020D3
:2026200098B5164C94F8E100002710B91448007860B105F05FFC94F8E310002906BF0121CA
:2026400084F8E310012705F051FC0FB1002098BD022003F043FC0E20FCF75AFD094A1068D5
:2026600048B909494020C86008600127D761002084F8E20098BD012098BDC046F012002046
:202680009E90010004800C402C500C40F8B516460C46054605F02EFC07461CB3641E1AD026
:2026A000641E15D0641E0FD0601E0BD1306828B1012807D1802002F08DFA15E0802004F0E4
:2026C0001BFD11E0032410E030780A4908700BE03088688208E00120EE68687406F1600048
:2026E000E86001E0306828608324384605F0FEFB2046F8BD400E002070B5194D95F8C040DD
:2027000003460846002101F0BBFB14490F2C15D095F8A16091F83920A64208D0521C6FF0E0
:202720000F06A2409401A4EB8204321907E0521CA2409401A4EB8202A03A00E0002281F879
:202740003830012B1CBF4A63086305D1D5F8A430181808639B184B6370BDC046641B0020AD
:20276000D811002038B5042903462BDA05F064FA0546084605F0FAF9134C5B0002460229E7
:20278000195503EB040012BF0329002141706068E9B202F0B1FF03F087FF50B904F120006E
:2027A000044605F01DF901280CD1204605F0DAFA38BD04F12000044605F012F910B920460C
:2027C00005F0CEFA38BDC046201B00202DE9F843174C241F04F1240108688846074628B36F
:2027E00000261D25387D35281BD140463946324602F09CFE787E30F07F0005D194F82F0044
:20280000401E84F82F0004E094F82E00401E84F82E007D7057F80C9C3846FFF747FA4F46DB
:2028200002E03E4657F80C7C002FDBD1BDE8F883AC10002038B5164D95F8B41001290FD0DA
:2028400003280BD013480078812804DB8428B8BF49F6404419DB4FF4FA5416E0002414E09E
:20286000032844F6206410D00B48006890F8690058B105F0EBF90A224FF4FA6390FBF2F1C7
:202880005143401A58432418A4B2A5F8B64038BDA0310020BF120020A8100020164880B548
:2028A00007683FB315498B6803EA5300C00E21D2134A106880081DD2486880081AD210687D
:2028C000096810F0050F4FEA114101F0F00101F5E0710AD1B9420DD2190F38BF40F00100BA
:2028E000D90E38BF40F0040003E0B94202D920F00500106080BDC04628500940AC3F005049
:2029000000000940F8B50646B06801687568886B20F4FA6088631349086820F40070086013
:2029200005F0E8FA104C0746207820B1022003F097F800202070384605F0D8FA05F0DAFA4C
:20294000A96B11B905F0D2FAF8BD0021A96305F0CDFA686B296BEB68091A29636A6B304686
:202960009847F8BD30100040F4350020F8B5844640F6FF741CF8013B002210E0481B401EB7
:2029800010F8015B7F1E01F8015BF9D103E01CF8010B01F8010B521C5B08082AEADA5808E8
:2029A000F5D21CF8010B1CF8015B05F00F07FF1CC5F30315122F45EA001508D11CF8016BEC
:2029C000300A24BF1CF8010B60F3DF16F719AC42D4D1F8BDB0B5184C05460F46101C28D08D
:2029E0000DE03868E06397F82700394640F0040087F8270004F14C0003F04CF8E76BD7B1A6
:202A0000F8688542EDD014E0386888B13868C06885420DD139680868386091F8270040F00F
:202A2000040081F8270004F14C0003F033F800E03F68002FE8D1B0BDD80D0020084610B59F
:202A400000F0005100F00400084321D0012003F0EFFB114C012813D00E4801683220B0FBE2
:202A6000F1F2012A8CBFB0FBF1F101212046A0F12404204605F0F6F9204605F02FFA10BD94
:202A8000064805F03DF806492046D8380839086010BDC04614910100C40E0020153500009B
:202AA000081004409EB5144C606880472146134C2289E38893421CD0114B1F78CFB9114B04
:202AC00089681F7837F07F0714D1E28088471027E088ADF8007001A9ADF8040009880DF115
:202AE0000203198008480068426AE068694690479EBD896888479EBD001800200C1C002010
:202B0000FE35002000360020681900202DE9F843DFF85880044608EB440000F11805008B51
:202B2000894603F097FF074611480678AFB12A883846002105F020F900253C7041467D7015
:202B40000A5D381D494604F065FD3046394600F0BDFC40B92846BDE8F8838DF8004068463C
:202B60001A21FEF75FF81A20BDE8F883F08801008818002010B5164A144C92F83D0094F863
:202B8000401048B91348006860B9012082F83D00202004F03DFF05E0481CC0B2042884F85D
:202BA00040000DD00C49A1310A784FF4707304F1200003FA02F101F2636104F045FB10BD6C
:202BC000202002F01DFCFCF777F810BDEC340020641B0020A8100020D8110020002A184A2F
:202BE0002DE990418846117804460AD0201D03F0ADFA4FF6FF7181421FD004F0C3FAE0B1F3
:202C000017E0322904DB4FF6FF7004F0BBFA07E088004F1C00EBC1001018F9B21170A43078
:202C200058B16188424601801368871C3B609288BA800121017200274781BDE89081C0464C
:202C4000DC0A002010B5044600212822ADF1280D6846FEF73EFF134911226846FDF7BAFB5B
:202C6000FF228DF8182005208DF812008DF8114000218DF815108DF8161009228DF813208B
:202C800001208DF817008DF814000B220DF11900FEF71FFF044918206A460CF0A1FA0AB001
:202CA00010BDC0466E8C010075ED00002DE998430446A76E9946904607B1B84700200221E5
:202CC00000EA090701EA0801002F08BF002917D104F1600106C909EA020708EA0101002FBB
:202CE00008BF00290CD161680978022910D100EA09000821002801EA080108BF002907D0B2
:202D000004F1700080E8000304F1400005F0EAF8BDE89883C8B50146164AC87AB8B992F8B6
:202D20003170906B2FB3401F401DC6781EB1CA7F03799A4202D07F1EF6D1C8BD8A7FC270B5
:202D4000CA880280CA7F0271097B8170C8BD92F83070506B6FB120382030867F3EB1CA7FFF
:202D6000C37F9A4203D12022FDF734FBC8BD7F1EF2D1C8BD0414002038B5012003F058FA07
:202D8000012820D0114DD5F82401C4681048342101220023A047002808BF002014D0286841
:202DA00003F06EFC04F022FB0B4A0A4D93681168D060C01AA1EB910105FB00F3180C88427C
:202DC00028BF011C1160012038BDC0468000001000A00C4040420F00B835002098B50446B1
:202DE000207B00F00F00022824D100F04DFFA168081A8108114800F10C021768002F14BF51
:202E0000FB6840F6C41303F57A728A4212D20A4A12686FF050448C420CD3C91AB1FBF2F3CC
:202E2000012B8CBFB1FBF2F10121C83005F01AF8012098BD002098BD14910100D80D0020D5
:202E4000001F06B480B290B5082803AFADF10C0D22DB3A78B0F5805F1EDA00F18851091F6C
:202E60000C686B461C6049685960BDF800108A420BD17988BDF80230994206D1B988BDF84A
:202E80000430994208BF012007D0BDF80610401A083880B20828DDDA002003B0BDE890409E
:202EA00002B07047F0B5174D286A4FF6FF77ADF12C0D20B301F032FC08B30620002605235B
:202EC0008DF808002C6AADF80C60642EADF80A3015DA04A80090246902AB93E803003246F2
:202EE0001823A04748B1BDF80C002C6A401CADF80C0080B26428ECDB01E0BDF81270384638
:202F00000BB0F0BDEC1500201FB5044694F8960038B304F18B0101A804F00AFF03208DF82E
:202F20000C00114890F8D7100091B4F89420B0F8BA3001A92046FDF7B1F90146DC290DD063
:202F4000DD290BD0E42909D0F32907D0DE2905D0DF2903D0E82918BFDB2902D12046FDF7E7
:202F600061FE00901FBDC046D811002010B5FF201349144C0870201D00688047124903464F
:202F800024310868014650B14A7E32F07F001CBF02F0EF024A7651F80C1C0029F4D1A168D5
:202FA000184688470948A13890F8A11090F8C000814201D003F018FA082004F031FD10BD89
:202FC0009C1B002000180020A81000207912002010B504460320ADF1180D04F128018DF8C7
:202FE000020000208DF8030001A804F0A1FE6068007804F11C018DF80C000DF10D0004F009
:2030000094FE04F1280003F077FB58B14FF6FF7453206946ADF80040F3F702FE0449204637
:203020000A3108800DF10200FAF7D2FE06B010BD8212002070B5164D286808B104F0A2FD71
:20304000144C606880470C3DE9690A68002616710968E961A16888470A4A0B49107810B93B
:203060000846007860B1167008460670FCF70CFC06480078012803D030460146F3F7CCFC03
:2030800070BDC046FC350020FE350020EA1D00206435002000180020F8B50025114C1348B7
:2030A000A5604FF4700665600068E660C06B80470D49C0F1FF3008600D48C76865700FB92E
:2030C0000C49C1600C480570012001F0D1FE08B104F066FC304601F041FAE068FEF7C0FF23
:2030E000F8BDC0466C1D00200830044068190020DC1B002059370100FF3500201649154897
:203100008CB5FF220F7890F83B30144980F83820012B08D091F8A10091F8C010884217D06E
:2031200003F062F98CBD002380F83B3087B18DF8032091F8D7008DF8000091F8E6708DF8C9
:20314000017091F8E7308DF80230684604F090FD8CBDC046641B0020D7100020D81100207A
:2031600038B5154C124D0121BD3C94F8A10085F83D100F2818D0114837380170202004F004
:2031800047FC94F8A1200E490A4835F81220886201F1200091F84010491C5143490001F28D
:2031A000A32103F0D1FA38BD02F0E0FE38BDC046641B002025F30000951200200017002018
:2031C000EC34002070B5164604460D1C08BF052426D034F07F0001D003F010FF002C18BF5C
:2031E000032407D155F80C0C18B915F8020CFF2804D00524284604F0A8FB11E0012E0948E5
:2032000005F8024C03D0294602F0C6FC02E0294603F010FE20464FF40041FCF7D1FC00244D
:20322000204670BDE41B002030B50446606800252062ADF1140DA5657820A4F84C0094F869
:203240002C0025650F2807D004F12C0120460122F6F72AFA08B116E0284694F83C10FF29D1
:2032600001D1A16D21B104F13C012046FBF71EFA48B92B4601208DF80C30032101AA009047
:203280002046F0F761FB05B030BD70472DE9FC41144C154F06468846700809D32068456872
:2032A000002101220B461FFA88F000903846A847B00809D3206845680021022201231FFAA0
:2032C00088F000903846A847F00809D320681FFA88F600210C220223446800963846A0476B
:2032E000BDE8FC81A401001000A00C400246F8B5084611464C68203821D0401E1CD0401ECC
:2033000018BF6FF001001ED18D6804F0F3FD0E4E07463068016928688847B0F1FF3FF8D1FC
:203320000025A564606C401EE06425653846A56304F0DCFD2846F8BD0021084601E001217F
:20334000002084F82D10F8BDD0010010012898B523D1012002F06CFF01281ED004F05EF8B5
:20336000114C012104F1D800017004F0EDFB800915D20C4800683222B2FBF0F707B90F468B
:20338000083C3034204603F085FD2046394604F069FD204604F0A2FD01E002F02DFB002057
:2033A00098BDC04614910100F81200202DE9F041154C206A0025ADF1280D08B301F0AEF965
:2033C000071C1DD0062005232E468DF80800A046ADF80A30642D13DAD8F82000ADF80C505A
:2033E00004AB02AA0469009392E8030018230022A0470A2804D000B9761C6D1CB742E9DC19
:2034000028460AB0BDE8F081EC150020F8B51549154A134D36395B320B681778E91C0978FF
:20342000002F0CBF1C695C6901EB810164182679002101E0491CC9B28E42D8BF4FF6FF70C2
:203440000DDD23680A4602EB42029B1893F900209042EFD1B3F801002881B3F80100F8BDCF
:203460000C1C00209A1900209212002038B5154C04F1180005461C3000F016FF03F07EFA0B
:20348000042003F0B1FAA07E032801D1607EA0B105F14501E120F3F7C3FB05F14601E720F7
:2034A000F3F7BEFB084894F85F100078884204D005F14701E820F3F7B3FB2846FAF788FC47
:2034C00038BDC046DC330020BF12002070B502460D4632F07F0004D110460022FFF772FEBD
:2034E00070BD04F067FB104908398C78A5F10C06FF2802D0C96A40184478FF2C02D103F0D2
:203500007DFD0DE0104603F0ADFE01462A46FF20B072204602F022FA20B1284604F015FAA2
:20352000012070BD002070BDE41B002080B501884FF6FF728A4224D002F032F9071C20D06D
:20354000788940F0010010F4407F788102D103F037F9788910F4A04F13D10A48008880084D
:203560000FD20948283004F03BFA50B94FF470404FF4805102F0B4FE18B94EF6602002F05D
:20358000D5FB80BD6C170020EC15002000B5ADF1240DADF80000ADF80210116801A80160F7
:2035A0005168002241600E49069391F836008DF80C202D318DF80D000B680DF10E0003605D
:2035C0004B684360097A017218208DF81C2005498DF81D206A460BF003FE09B000BDC0466E
:2035E000288C01006958000098B5154B1B1D18680004070C21D003F007F8104991F90720EC
:20360000824205DD10F1800FB8BF6FF07F00C8718C88BC4210D80A68D3F8D40F801A801C96
:203620001F2888BF1F203F1B4008C7404FF6FF70E719B84238BF071C8F8098BDEC350020A7
:203640003010094008B51348134A14490078801E0A2807D8DFE800F01814100614100614B1
:20366000100609C004F00AFC11E010688008FCD250688008FCD20AE008688008FCD306E00D
:2036800008688008FCD202E010688008FCD3F5F7A9FD08BDD413002034600C4038600C4091
:2036A00010B5114CE16B81B1104A106848B911600020E0630220F4F761FB022003F08AFBC0
:2036C00003E004F13C0001F0D3FC0948007850B10848A16B00780F2805D00748206204F1A6
:2036E000180003F031F810BDA8340020A8100020C916002079120020853D0100F8B5154C7A
:20370000124940F27C62243C2046FCF763FE002102220B46181932278D3000F8031F41707C
:203720007F1E8170F9D1521E03F19603F2D1084E04F5E275322728463146182203F06AFFF7
:2037400018357F1EF7D10220A070F8BD287F0100EC8001007425002070B5134C60688047EF
:2037600012490025064648784D70A168820808D2C00816D33046884728460146F3F74CF9B9
:2037800070BD304688470A480078012803D001202946F3F741F9606880470646FAF720FD54
:2037A000A1683046884770BD001800206C1D0020EA1D0020B0B50F46044604F09BFB0546AD
:2037C0001148EC3890F8C710C90803D390F8C610A14215D0B0F8C430012101FA04F21A4334
:2037E0000A4BA0F8C420181D026804F10C0399408A430260006818B917B1022001F0EAF956
:20380000284604F073FBB0BDC40E0020081004401549096821280ADC212819D00C380FD0CA
:203820000D380FD0001F0FD0C01E0FD01AE0253810D0001F10D0401E10D0401E10D011E006
:20384000086870474868704788687047C8687047086970474869704788697047C86970472C
:20386000086A704700207047F0010020F8B50646B08815460F46FDF7F5F80446002D02D428
:20388000281B0A2806DB3368291B38460BA201F04BFA0419B08978B1002D06D4B06803F001
:2038A000EBFF291B401D884206DCB368291B384603A201F039FA04192046F8BD257000C09E
:2038C0002827257327290000F8B50746C81D01F00705C610002F4FF0010000FA05F0A0F110
:2038E000010C14BF0029002019D00020BEB17F1E33460246941B17F8011FB4F1FF3F08D12F
:203900000DB10CEA010104E001F1FF04401C2140C0B20029F8D15B1E02F10102EAD1F8BD18
:2039200070B5F0F73DFD124D68688047064603F029FE104C94F9D60003F06CFF02F03EFD9B
:2039400003F05EFF03F012FE03F004FEA9683046884794F8D70000F07FFC04F1BD015220D6
:20396000F3F75EF904F014F908B9FFF795FB70BD00180020D811002038B50C4620B1416897
:203980000122A240114201D1022038BD914341600E480025231800EB8401C1F8945003F1BA
:2039A00040010978FF291ABF406850F8211044F020410548F9F7D4FD20464FF0FF3103F0B8
:2039C00063FB284638BDC046007FC767FC2E00201248134908B54FF42C72FCF7FBFC4FF0AC
:2039E0000451002081F89003012081F87903022081F87503032081F87703042081F8AE03B9
:203A0000052081F8AB03062081F88103072081F84D030448C1F8C00308BDC0461C04002173
:203A20003C000000CD05002198B5124CE2685168496839B110B102F011FCE26850684068A4
:203A40008047E2685268906808B9D7688FB10A491C310F68002FFCD000230B6010B180473B
:203A6000E0684268D06800B180470448503802F0DFFD98BDD80D00200010044051000706F6
:203A8000144BB0B5997B03EB81010A69017801F07F014D000170AC185219527803EB820555
:203AA0002F6907B19A732278141103EB84031F6C2FB90C290CDA1821FDF7B4F8B0BD02F0AF
:203AC0000F0257F8221011B903F06AFFB0BD8847B0BDC046881800202DE9F04105461248D3
:203AE0000E46002100782960012802D00120F2F793FF0E4C606880473768804630463FB105
:203B00006A687968914203DC38463F68002FF8D1056030682F60854201D1FDF717FCA168EE
:203B200040468847BDE8F081EA1D002000180020134A38B5B2F8C4504FF6FF71A9421BD028
:203B40000024012000FA04F32B4212D05940B2F8C4300C4D1940A2F8C410291D0A6804F1DC
:203B60000C03984010430860022003F0C5FA204638BD641C0F2CE5DB6FF0010038BDC0469E
:203B8000D80D00200810044038B5044642F209000DF1020100F024FC9DF8020050B19DF812
:203BA000020002281AD1A08894F82710FEF77AFB054606E042F20D00694600F011FC9DF8E6
:203BC0000050284600F048FB0020A4F87C5094F82130607013B1102003F022FF38BD38B5D5
:203BE000046845682068002808BF4FF0FF301FD004F080F92168002954BF491E002121609D
:203C000004F074F9206890B904F12C0004F012F904F1480004F01AF904F1640004F016F9B2
:203C20006868FAF78DFF04F1180003F093F8002038BDFEE72DE9B841124C0546201D006855
:203C40008047804603F026F86F7E002F08BF6B6807D069682A69AF68091A5218B9180B460F
:203C60006960E968286105F11402184601F090FE012768686F76A168A86040468847BDE8D0
:203C8000B881C0460018002010B504F033F9104C217829B10F490C6804F028F9204610BDE5
:203CA00004F024F903F070FD0B4A002303F0D6FC626A002314001B184FF07A024FF0905046
:203CC00044EB0104C11842EB04021046001C10BDD80D00200430044000093D00B0B5134CDE
:203CE0006068628800B325880021AA42C8BF01210B46AA42C6BFA91A01F58061A91A8FB29C
:203D00008FB1012B03D0A1183A46083109E0A118C2F58062083103F085FF606804F1080141
:203D20002A4603F07FFF6580B0BDC046D406002038B51248104C0168114D0C40E143016015
:203D4000A10907D34068800904D328464FF4005103F0C0FC14F4602F0DD02846EC3800F12F
:203D6000C0010A6804F4602400F5907014430C60002103F0AFFC38BD20000E00081004409E
:203D8000C40E002010B511480F4C0078A16BD0B10F484031206104F1080002F0D5FC03F0B7
:203DA0004DFD40B9F3F732FCE06360B1017E41F04001017610BD0749002391F8A800E36335
:203DC000401C81F8A80010BDA8340020C9160020A1360100D811002070B5124DBD3D95F8B2
:203DE000A100B5F8C6400F2810D00F483430066801F0F2FC2018864208D895F8A1104FF4EF
:203E0000707088402418A41B04F57074044D284600F04AFA2146284603F016FA70BDC04624
:203E20007833002095120020641B00201FB5014604208DF8000048788DF80100B1F8960008
:203E40000DF10203ADF80C008C31184603F05EFA02F052FC60B14FF6FF7453200DF10E01BF
:203E6000ADF80E40F2F7DCFE044920460A3108806846F9F7ADFF00901FBDC04682120020A6
:203E8000134A3D321278812A01DB842A0FDB00F11002490892B224BF00F129018AB21228A1
:203EA000CCBF05200220801880B2C0000DE04201490802F5C67292B224BF02F21E218AB260
:203EC0001228CCBF28200C20801880B27047C046821200202DE9F0410120104E104D3070AB
:203EE00028781F469046022801D003F059FD0024022114EA070001EA080108BF002902D1A0
:203F000003F04EFD07E0074991F90000401E08702C7003F05BFB3470BDE8F081EA1D002006
:203F2000EB1D0020E61D0020C8B5071C01D103F037FD79684878C6111FD03B89F9640020F5
:203F40004A78C2F3C3020F2A09D00A781018801C80B25218834202F10201F1DC01E0801C2C
:203F600080B2834206DB79683E8941187960311A398100E00020A7F85000C8BD10B5044607
:203F800000211C22ADF1200D6846FDF7A2FD60788DF80000A0788DF80100E0788DF80200DC
:203FA00020791122611D8DF8030001A8FCF712FAA07D8DF8150008B1A069069003480068C5
:203FC00081696846884708B010BDC046BC1D00201FB5044603208DF80E000DF10E01009184
:203FE000627921880123FBF7F5F9012809D002208DF80C002388ADF8043001A8FFF796FAD1
:204000000AE0608940F480506081044801F08EFE03498869401C886100901FBD009F24006E
:2040200068170020F8B504460D46084611220021FDF74FFD94F800C0BCF1000F1AD0641C43
:2040400000214FF0010EE078A37843EA0023207809E0C610AF5D00F00702401C0EFA02F27A
:20406000C0B23A43AA558342F3DA491C241DC9B28C45E8DCF8BD80B502465378107840EA5B
:204080000320C7130F7007BFC0F3062300F0FF00C0F3C323C0F30A004B70802848800DDAAB
:2040A00002280BDB012B0CD0022B0AD0042B08D0052B06D0062B04D0072B02D00022104653
:2040C00000E0921C4A6080BD70B5114C2068E8B1104D686880470646216894F82F0002281A
:2040E00006DBA96830468847F120F4F7ADFF70BD04F1240002F09EFE002394F82F00A9681E
:204100002360401C84F82F003046884770BDC046A81000200018002038B5044642F208001A
:204120000DF1020100F05CF99DF8020040B19DF80200022817D1204601F034FA054606E052
:2041400042F20C00694600F04BF99DF8005094F8200030B9284600F07FF8A4F87C50002065
:2041600000E00120207038BDF0B5124D00260C460746ADF1140DC5F8B061012003F0B7FD9B
:204180002868C00FF9D3286A0090686A0190A86A0290E86A03903FB13846694611F8012B94
:2041A000401E04F8012BF9D1032005B0C5F838023046F0BD50450240114898B501210170AD
:2041C000022111400F4A4FF0E0471F4008BF002903D092F90010491E1170044692F9000032
:2041E00030B192F90000002806DC03F0D9FB03E000200146F2F710FC0020207098BDC04638
:20420000EA1D0020E61D002038B50546687E00F0EF0068762846FCF741FB0C4C294604F120
:20422000240002F007FE0A4D6868804794F82E10491C84F82E10A96888470648A130007815
:204240000F2802D1082003F0EBFB38BDA810002000180020D8110020B0B50546802D01DD0A
:2042600003F09EFB0D4C606880470D4B0D490A4A1F780A390D701FB91778A1682FB907E032
:204280001778A16837F07F0702D088470120B0BD8847FDF71FFFB0BD0036002000180020CE
:2042A00000170020181C002070B505460F480078012803D001200021F2F7AEFB0C4C201DCF
:2042C000006880470B49064628460B4602F05DFE18B9191D284602F058FE1869A84201D109
:2042E000FDF734F8A1683046884770BDEA1D002000180020C81D002070B540680C46054655
:2043000000F5847002F0C6FD0D482A7F0168687F8018AA69C01D80B244430A4805F584762A
:204320006043B0FBF2F008186330B0FBF1F1491C304603F097FD304603F0D0FD70BDC04642
:204340001491010040420F000F4838B50078C8B10E4D0F4C95F82E106420503C484320664F
:2043600004F15C00FFF766FCE08EE26B95F82E10401C80B28918E08600B900210020E1633B
:2043800000F0F0F938BDC046951200205C320020F0310020F8B5114C60680D4680470E4B4E
:2043A000A16893F830705A6B97B10024203A2032967F4EB1D37F9D4206D100239377FF2381
:2043C000D37788472046F8BD7F1E04F10104EED18847FF20F8BDC04604140020001800203A
:2043E000F8B50E4602F0FCFD05464FF6FF70A84208BF682013D00A4C6068804709490A4B2A
:204400000746680000EBC50008180278991842783046FBF7DFFFA168384688470020F8BDC1
:20442000001800202C8601005C320020042838B51CD1104CEC3C04F1C800054603F0A2FCC0
:20444000A0B1284603F03AF909490968484364280CD2284602F01EFD052001F03FFD20468C
:20446000012181720421EC3003F034F9002038BD14910100C40E002010B5044610489530ED
:204480000078ADF1180DC0B1012000238DF8000004F128018DF801300DF1020003F048FC9C
:2044A0006068007804F11C018DF80A000DF10B0003F03BFC6846F9F78BFC06B010BDC0463A
:2044C000D811002038B5EB2002F02DFF0D48002505700B480078862802D1284600F064F8C8
:2044E000094C6068804709490C39CA6913681D711268CA61A168884702F0ECFE38BDC046B1
:2045000000360020FE350020001800206435002038B50D4C6068804705460C48007870B9EC
:204520000B48007830F07F0009D10A48007830B90948007830F07F0001D103F0F3FBA16860
:204540002846884738BDC04600180020FD350020FC350020FE35002000360020F8B50646A6
:204560000F4800680D4CC06B80476168401A21788900B0FBF1F0B04201D303F011FA094D46
:20458000243D686880470746A6603046FDF7E4F9F9F726FEA96838468847F8BD6C1D0020B9
:2045A000681900202418002038B50F49104C088D401C08856068804705460C480178862989
:2045C00003D0A1682846884738BD8721017003F0E5FAA16828468847082002F005FAE9207A
:2045E000FDF702F838BDC0466C1C00200036002000180020F8B506460F4D104F73880024C9
:2046000017E0A00000EBC400321851689068D26852B9AF420BD00A7855F822200346491C89
:2046200008461946904701E0FBF7D4FE7388641CA4B2A342E5DCF8BD7C0E0000880E000005
:20464000F8B5034600208C460446074613E01CF8015B082685F0010101F001014018C0B216
:20466000411E994206D0641C761E4FEA6505E4B2F0D100E00127A24203DC27B903F062FB21
:2046800001E0002FE3D02046F8BD3EB5054615F8060C03281DD12B681869009058690190D0
:2046A000986902906C6859689A681868DB68A0472968086015F8080C01F0A0FC0446012014
:2046C00002F0C8F9011C04D0422008702046FEF7FDFE3EBD2DE9F04117468846064603F05A
:2046E000CBF80D4C0546002128222046FDF7F1F931462A462046FBF76DFE40463A462919B2
:2047000000F0E4F8204602F01BFE02A002F018FEBDE8F0810D0A00C0303500201048B0B583
:2047200007680025ADF1180DADF810509FB106208DF808000424ADF80A40ADF80C5004AB53
:2047400000933C6902AA92E8030002232A46A04708B1ADF81050BDF8100006B0B0BDC046D0
:204760000C16002070B50F4C05462179E079814217DD6179A94214DDA3680B4E23B1294625
:2047800032469847E0796179A07101FB0050216800EB800009180878E071D1F801103046FC
:2047A000884770BDF4190020D4310020F8B502F0CEFB0D4607463B2F08BFF42012D00B4C25
:2047C000606880470646BA0007480949835C801842784E39C918284602F01CFFA168304610
:2047E00088470020F8BDC0460488010000180020BA12002038B50D460E49144660390A6862
